:020000040000fa
:080000000002040000000000f2
:020000040000fa
:040008004c030000a5
:020000040000fa
:04000c004c030000a1
:020000040000fa
:040010004c0300009d
:020000040000fa
:040014004c03000099
:020000040000fa
:040018004c03000095
:020000040000fa
:04001c004c03000091
:020000040000fa
:040020004c0300008d
:020000040000fa
:040024004c03000089
:020000040000fa
:040028004c03000085
:020000040000fa
:04002c004c03000081
:020000040000fa
:040030004c0300007d
:020000040000fa
:040034004c03000079
:020000040000fa
:040038004c03000075
:020000040000fa
:04003c004c03000071
:020000040000fa
:040040004c0300006d
:020000040000fa
:040044004c03000069
:020000040000fa
:040048004c03000065
:020000040000fa
:04004c004c03000061
:020000040000fa
:040050004c0300005d
:020000040000fa
:04005400146b000029
:020000040000fa
:04005800406b0000f9
:020000040000fa
:04005c004c03000051
:020000040000fa
:040060004c0300004d
:020000040000fa
:040064004c03000049
:020000040000fa
:040068004c03000045
:020000040000fa
:04006c004c03000041
:020000040000fa
:040070004c0300003d
:020000040000fa
:040074004c03000039
:020000040000fa
:040078004c03000035
:020000040000fa
:04007c004c03000031
:020000040000fa
:040080004c0300002d
:020000040000fa
:040084004c03000029
:020000040000fa
:040088004c03000025
:020000040000fa
:04008c004c03000021
:020000040000fa
:040090004c0300001d
:020000040000fa
:040094004c03000019
:020000040000fa
:040098004c03000015
:020000040000fa
:04009c004c03000011
:020000040000fa
:0400a0004c0300000d
:020000040000fa
:0400a4004c03000009
:020000040000fa
:0400a8004c03000005
:020000040000fa
:0400ac004c03000001
:020000040000fa
:0400b0004c030000fd
:020000040000fa
:0400b4004c030000f9
:020000040000fa
:0400b8004c030000f5
:020000040000fa
:0400bc004c030000f1
:020000040000fa
:0400c0004c030000ed
:020000040000fa
:0400c4004c030000e9
:020000040000fa
:0400c8004c030000e5
:020000040000fa
:0400cc004c030000e1
:020000040000fa
:0400d0004c030000dd
:020000040000fa
:0400d4004c030000d9
:020000040000fa
:0400d8004c030000d5
:020000040000fa
:0400dc004c030000d1
:020000040000fa
:0400e0004c030000cd
:020000040000fa
:0400e4004c030000c9
:020000040000fa
:0400e8004c030000c5
:020000040000fa
:0400ec004c030000c1
:020000040000fa
:0400f0004c030000bd
:020000040000fa
:0400f4004c030000b9
:020000040000fa
:0400f8004c030000b5
:020000040000fa
:0400fc004c030000b1
:020000040000fa
:040100004c030000ac
:020000040000fa
:040104004c030000a8
:020000040000fa
:040108004c030000a4
:020000040000fa
:04010c004c030000a0
:020000040000fa
:040110004c0300009c
:020000040000fa
:040114004c03000098
:020000040000fa
:040118004c03000094
:020000040000fa
:04011c004c03000090
:020000040000fa
:040120004c0300008c
:020000040000fa
:040124004c03000088
:020000040000fa
:040128004c03000084
:020000040000fa
:04012c004c03000080
:020000040000fa
:040130004c0300007c
:020000040000fa
:040134004c03000078
:020000040000fa
:040138004c03000074
:020000040000fa
:04013c004c03000070
:020000040000fa
:040140004c0300006c
:020000040000fa
:040144004c03000068
:020000040000fa
:040148004c03000064
:020000040000fa
:040208004c030000a3
:020000040000fa
:04020c004c0300009f
:020000040000fa
:040210004c0300009b
:020000040000fa
:040214004c03000097
:020000040000fa
:040218004c03000093
:020000040000fa
:04021c004c0300008f
:020000040000fa
:040220004c0300008b
:020000040000fa
:040224004c03000087
:020000040000fa
:040228004c03000083
:020000040000fa
:04022c004c0300007f
:020000040000fa
:040230004c0300007b
:020000040000fa
:040234004c03000077
:020000040000fa
:040238004c03000073
:020000040000fa
:04023c004c0300006f
:020000040000fa
:040240004c0300006b
:020000040000fa
:040244004c03000067
:020000040000fa
:040248004c03000063
:020000040000fa
:04024c004c0300005f
:020000040000fa
:040250004c0300005b
:020000040000fa
:040254004c03000057
:020000040000fa
:040258004c03000053
:020000040000fa
:04025c004c0300004f
:020000040000fa
:040260004c0300004b
:020000040000fa
:040264004c03000047
:020000040000fa
:040268004c03000043
:020000040000fa
:04026c004c0300003f
:020000040000fa
:040270004c0300003b
:020000040000fa
:040274004c03000037
:020000040000fa
:040278004c03000033
:020000040000fa
:04027c004c0300002f
:020000040000fa
:040280004c0300002b
:020000040000fa
:040284004c03000027
:020000040000fa
:040288004c03000023
:020000040000fa
:04028c004c0300001f
:020000040000fa
:040290004c0300001b
:020000040000fa
:040294004c03000017
:020000040000fa
:040298004c03000013
:020000040000fa
:04029c004c0300000f
:020000040000fa
:0402a0004c0300000b
:020000040000fa
:0402a4004c03000007
:020000040000fa
:0402a8004c03000003
:020000040000fa
:0402ac004c030000ff
:020000040000fa
:0402b0004c030000fb
:020000040000fa
:0402b4004c030000f7
:020000040000fa
:0402b8004c030000f3
:020000040000fa
:0402bc004c030000ef
:020000040000fa
:0402c0004c030000eb
:020000040000fa
:0402c4004c030000e7
:020000040000fa
:0402c8004c030000e3
:020000040000fa
:0402cc004c030000df
:020000040000fa
:0402d0004c030000db
:020000040000fa
:0402d4004c030000d7
:020000040000fa
:0402d8004c030000d3
:020000040000fa
:0402dc004c030000cf
:020000040000fa
:0402e0004c030000cb
:020000040000fa
:0402e4004c030000c7
:020000040000fa
:0402e8004c030000c3
:020000040000fa
:0402ec004c030000bf
:020000040000fa
:0402f0004c030000bb
:020000040000fa
:0402f4004c030000b7
:020000040000fa
:0402f8004c030000b3
:020000040000fa
:0402fc004c030000af
:020000040000fa
:040300004c030000aa
:020000040000fa
:040304004c030000a6
:020000040000fa
:040308004c030000a2
:020000040000fa
:04030c004c0300009e
:020000040000fa
:040310004c0300009a
:020000040000fa
:040314004c03000096
:020000040000fa
:040318004c03000092
:020000040000fa
:04031c004c0300008e
:020000040000fa
:040320004c0300008a
:020000040000fa
:040324004c03000086
:020000040000fa
:040328004c03000082
:020000040000fa
:04032c004c0300007e
:020000040000fa
:040330004c0300007a
:020000040000fa
:040334004c03000076
:020000040000fa
:040338004c03000072
:020000040000fa
:04033c004c0300006e
:020000040000fa
:040340004c0300006a
:020000040000fa
:040344004c03000066
:020000040000fa
:040348004c03000062
:020000040000fa
:10040000cfa221000e7f22000e0188000000000014
:10041000000020000000e000020032000001200087
:10042000200288000c000700e0e227000100200005
:1004300011000700000020000000e0000200320070
:1004400000000200000000002e7f020000000000fb
:100450000040da000000fe004440a900002b20000c
:100460000000e0000300320000002000a00188002e
:100470004440a80000000600910188008000780038
:100480000000eb0015003700e280400032a0b4000d
:100490009101ba00e280400032a0b4009102ba009b
:1004a000e280400032a0b4000002eb00472bde00e7
:1004b000f507b200602ce10004003a000059eb009f
:1004c0008301e900fdff3e00040037006128e100e0
:1004d000010032000082eb000b00070011c3ba00dc
:1004e0001101ba000604e00003003a000200e00037
:1004f000e5ff3a0000000600f607b200960188000a
:1005000082007800f5ff37003159ba008301e90015
:100510000c0032002159ba008301e90008003200c2
:100520000400e00003003a00e280400032a0b40082
:10053000f5ff370011d9ba008301e900faff3a004c
:100540008100e800e180400032a0b4000000060015
:10055000000000000000000000000000000000009b
:10056000000000000000000000000000000000008b
:10057000000000000000000000000000000000007b
:10058000000000000000000000000000000000006b
:10059000000000000000000000000000000000005b
:1005a000000000000000000000000000000000004b
:1005b000000000000000000000000000000000003b
:1005c000000000000000000000000000000000002b
:1005d000000000000000000000000000000000001b
:1005e000000000000000000000000000000000000b
:1005f00000000000000000000000000000000000fb
:1006000000000000000000000000000000000000ea
:1006100000000000000000000000000000000000da
:1006200000000000000000000000000000000000ca
:1006300000000000000000000000000000000000ba
:1006400000000000000000000000000000000000aa
:10065000000000000000000000000000000000009a
:10066000000000000000000000000000000000008a
:10067000000000000000000000000000000000007a
:10068000000000000000000000000000000000006a
:1006900000000000000000000040da000000fe0042
:1006a00003f0a200889fbe008a9fbe008c1f7800c6
:1006b0004a010700510133006450e1004f0032004d
:1006c0006420e1005200320003826c0007003b000e
:1006d0000905d0000306d000820f54000c065d000f
:1006e0000200390002003200890178000306780018
:1006f0008582550004003d000003fd008103fd00dc
:100700008502ea008b854200840f720002003b00e4
:1007100060001000e08018006011b8000005eb00d8
:100720007a28e1000a00390006007800c75ddd0084
:10073000f707b200878075002d00370082817100b5
:100740000a017800610560008180d1000080d3003b
:100750008502e900f9ff3b00060440008784480059
:1007600002003b0060041400e0841c000988a30020
:10077000070032008a81710082817100610164008a
:100780008904d1000884d3008b05e80017003700e6
:100790000978a30013003a000b00e00013003400b6
:1007a0008b05e9000804440089844c000a44740065
:1007b0000978a3000d003a000b00e00007003400a8
:1007c0008b05e9000804440089844c0001003a00cc
:1007d0000b0020000978a300f7ff32000001eb00b6
:1007e00002003700828171000a017800c000070012
:1007f0000cf0a70001f0a000090137006420e1001f
:1008000002003a00838f6c00090133000801be002a
:100810000200be0002013700889fbe008a9fbe0012
:100820008c1f7800ed000700f400330003866c0095
:100830006450e1002e0032006420e10033003200f9
:100840006150e1002f0032006120e10031003200f0
:1008500085855500eb07b000090020000804200042
:10086000050037000804440089844c000a00310068
:100870000603430087834b000001530081815b0026
:10088000f8ff33000203be000800a0000804440083
:1008900089844c00f6ff3900c639dd0083017300fe
:1008a00001003200130020008904d1000884d30025
:1008b0000998a300050032000800a7000300a0006b
:1008c0008904d1000884d3008b05e8008904d10095
:1008d0000884d3000001eb000281d20084000700ed
:1008e00001f0a1000cf0a70001f0a000cc0037003f
:1008f0006420e100ce0032000801be000200be000c
:10090000f7ff37006120e100c90032006000b80045
:10091000f3ff37000000200001f82700f0ff370048
:10092000140020000e023700f4ff2f000c023700e5
:100930000003be00940007006011b8000470a70017
:1009400007f0a10007f8a30017003a006509b100fd
:100950000d0032000d003500860220000628e1005f
:1009600003003500030028006000b8000200050005
:100970000000400081804800020149008381490055
:100980008502e900faff3a0000000600f88f4200f5
:10099000050034008100d1000080d3008502e8000a
:1009a000fcff3a00000006006011b8008000eb0078
:1009b000000005000001be00730007000470a700de
:1009c00003f0a10003f8a30013003a006509b10089
:1009d00010003200090035006928e10002003500ee
:1009e0000100280000000500000040008180480050
:1009f0008502e900fcff3a0000000600f88f420083
:100a0000050035008100d1000080d3008502e80098
:100a1000fcff3a00000006008000eb00000005002b
:100a20004f89de0082017800e8013700889fbe0010
:100a30008a9fbe000082700004027100048271006f
:100a4000260032000004be000200be006011b800a3
:100a50006b092000950220000182cf000a003900b6
:100a60000541b1000082cf00070039000541b10007
:100a70000982cf00040039000541b1000882cf008f
:100a8000010039000541b100054252001200320058
:100a90000a003b0082817100610164008100d10085
:100aa0000080d3008984d3000884d3008b05e8003c
:100ab0000442e800f7ff3a0007003700080444004a
:100ac00089844c0000004800818048008b05e900c3
:100ad0000442e900f9ff3a00050007004f05be0097
:100ae0004f04be00000006006011b800cfff3700c1
:100af00081002000618055000b003d000b002000ac
:100b000061fe2f000100e1001d00340082817100b0
:100b1000610164008904d1000884d3000000e8006a
:100b2000faff3a00710020006100640003007000c9
:100b3000020060000900320061044400e0844c00bf
:100b40000988a500050032008b05e8006808e1006f
:100b500002003a008904d1000884d300f20f20007b
:100b60000258e10005003d00c75ddd00f907b20055
:100b70008980750008007800000006000bf8270047
:100b80008b00780000000500c70ade00f107b20004
:100b9000f50fb20008003200e1cf4200020032003f
:100ba0000170a00024000500810f700001003200d8
:100bb0000408050044000500810f700002003a009f
:100bc000140005008502e9000000400081c04800d3
:100bd000fcff3b000170a000240005000004be00e3
:100be000e9ff07000003be000405be000200be00ce
:100bf000e5ff0700844f7500000006000200be00fc
:100c00006450e100050036006420e1000200360077
:100c10000968a30001003a000800be000160a000be
:100c20004f0678004f05be004f04be0000000600ce
:100c3000f0ff2f00f1ff2700f9ff3700889fbe006b
:100c40008a9fbe008c1f7800e4ff0700ebff330093
:100c500003866c006450e100240032006420e1004f
:100c6000270032006150e100220032006120e100e3
:100c7000210032008b854200eb07b1000134b8003f
:100c8000003ab8000804420089844a00013ab800da
:100c90000030b8008880400009014a000400330099
:100ca0000000400081804800020149008b05e900f6
:100cb000c909dd008301700001003200130020002b
:100cc000c814de004814dd004709de001200b2003f
:100cd000c808de000884700085ff070001f0a1004d
:100ce0000cf0a70001f0a000cdff37006120e1006b
:100cf000cfff32000801be000200be00f7ff370040
:100d00006150e100fcff3a00c9ff37006022b800e3
:100d1000060220000000d0008180d2000482d200b0
:100d20008582d2000000a0000202520083825a0095
:100d3000030031000202420083824a000000a10049
:100d40000603e900f3ff3a0000000600efff07008a
:100d50000400be0000000600889fbe008a9fbe00ff
:100d600030044200b0844a0030054b0090854b00af
:100d70006000b1000898be000a90be000440e10087
:100d800005c8e10006d0e10007d8e100020031000b
:100d9000680040001008e8004f05be004f04be0088
:100da00000000600889fbe008a9fbe003004be007f
:100db0002005be000418540005985c0006185d006c
:100dc00007985d00110020000440e10005c8e10023
:100dd00006d0e10007d8e100010039008000eb00f7
:100de000108810004f05be004f04be000000060032
:100df0001200fa00889fbe008a9fbe008c9fbe0032
:100e0000e0b79f00f1b79f0082bf9f0093bf9f0094
:100e10000605be000404be000000eb00d0b79f0032
:100e2000c0b79f00b0b79f00a0b79f0090b79f00ca
:100e30000006eb005fb19700cfb097008201410040
:100e40003fb097000200e00004003d0037000700bb
:100e50007e805700c0ff0700030037003300070003
:100e60007e805700cfff0700dfb697000d00e0003f
:100e70000c0035006fb29700ffb297000fbb9700d0
:100e80009fbb970010002000010020006011b800f7
:100e90000002720081827200020373008383730078
:100ea0001b0007000c06e80001042000810f56001b
:100eb000e0ff3a000d00e00004003d000802be0023
:100ec0000a03be007e805700a3ff07005fa89700bb
:100ed0000000e00005003a001fb29700afb2970093
:100ee0003fb39700cfb39700090007006fb097009a
:100ef000ffb097000fb997009fb997004f06be004b
:100f00004f05be004f04be000080fa00000006003e
:100f10000100070000000600a4b79f00b5b79f00be
:100f2000c6b79f00d7b79f00000006004f09de003c
:100f300082817100b3b79f004f01de0081804000c5
:100f400082807000a1b79f008fb097004f09de002c
:100f5000000040000200700090b79f007fa897003b
:100f60004f01de00818040008280700081b79f00c9
:100f70000d0007004f3ade00000040000400700042
:100f8000f0af9f00080007000402420085824a007b
:100f900006034b0087834b00dfff07000802be00fb
:100fa0000a03be00000006002fb29700bfb29700f0
:100fb0004fb39700dfb3970000000600881f78004a
:100fc00018002000881f780089ff07008f87e9003c
:100fd0004f04780000000600801feb0084ff07002c
:100fe0008f87e90000000600889fbe008a9fbe0030
:100ff000e00f5000e08f5800e00f5900e08f5900db
:101000000c003d006044b8006055b800000054007a
:1010100081805c0002015d0083815d00180020007a
:101020001500070008003d00180007000004eb0051
:10103000050037000004eb000f00070002003d0030
:101040001200070018002000dcff07000800e00085
:10105000060032006022b8006033b8000000520081
:1010600081805a0002015b0083815b004f05be0056
:101070004f04be0000000600e00f5200e08f5a004f
:10108000e00f5b00e08f5b00000006006044b800ea
:101090006055b8000402540085825c0006035d00c0
:1010a00087835d0000000600889fbe008a9fbe0007
:1010b0008c1f7800e00f5000e08f5800e00f5900bf
:1010c000e08f59000d003d006044b8006055b80045
:1010d0000000540081805c0002015d0083815d009e
:1010e0001c0020000820e10009a8e1000ab0e1008e
:1010f0000bb8e1000d003d00080037000006eb00d2
:10110000e00f5200e08f5a00e00f5b00e08f5b00c1
:1011100006003d006044b8006055b8000402540069
:1011200085825c0006035d0087835d00aaff0700df
:101130000c00e000060032006022b8006033b80006
:101140000000520081805a0002015b0083815b0035
:101150004f0678004f05be004f04be000000060099
:10116000889fbe008a9fbe00841f78009bfe0700f8
:101170004f00780011003300f0ff2f00838f6c00c8
:1011800006003b00040565000a00a70008003700c0
:1011900009f0a6001000200008003700820f54005c
:1011a000838f5c00030039001000200001003e0026
:1011b0000000200009f0a7000000ea004f05be0073
:1011c0004f04be000000e00000000600881f780009
:1011d000030478000300e00007003d0060001000f9
:1011e000e080180060011900e081190002003b0056
:1011f00001f02d00030037000cfe070008f0a700e7
:0c12000001f0a0004f0478000000060080
:020000040000fa
:10120c000d0a00002800000078000000293e0000b4
:10121c000008000020080000000000002e20000044
:10122c0000200000004300006c7500007463000097
:10123c006820000064690000736500006e670000a0
:10124c00616700006564000021210000210000009e
:10125c00546f000020660000696e00006973000086
:10126c00682000007365000074750000702c00008d
:10127c00207300007461000072740000207500007f
:10128c00702000007468000065200000706f000082
:10129c00776500007220000073750000707000000c
:1012ac006c69000065730000207700006974000011
:1012bc0068200000636f00006d6d0000616e00001f
:1012cc006420000027570000270d00000a000000d2
:1012dc00427500007320000050690000726100002c
:1012ec0074650000207600003300000020630000cd
:1012fc006c6f00006e650000207700002f6400000a
:10130c006966000066650000726500006e7400007e
:10131c002050000049430000004300006f6d0000a6
:10132c006d7500006e6900007479000020460000a5
:10133c00697200006d77000061720000652000008a
:10134c00763700002e300000202d000020670000b2
:10135c006f6f00002e6700006c2f000067430000c9
:10136c007a5100006e570000200000002028000079
:10137c0032340000464a0000363400004741000079
:10138c00303000000034000020000000322000004b
:10139c000041000033000000423400000042000015
:1013ac003500000042380000005500004e4b000094
:1013bc000029000000490000090000004f0900004e
:1013cc0000480000090000004c0900000045000026
:1013dc006e740000657200002072000061770000de
:1013ec0020760000616c000075650000206600002e
:1013fc006f7200002042000052470000003e0000c7
:10140c00001b00005b440000001b00005b000000a0
:10141c00440000001b5b0000430000001b5b00004d
:10142c00324b00000d000000430000001b5b00006d
:10143c003244000000570000617200006e69000029
:10144c006e6700003a2000006e6f000020760000ee
:10145c006f6c00007461000067650000206f000075
:10146c006e20000056700000756c00006c7500005a
:10147c0070200000706900006e000000203d00002c
:10148c0020000000436c00007574000063680000cd
:10149c00206500006e670000616700006564000055
:1014ac002121000021000000565200004547000099
:1014bc00207400006f6f0000206c00006f7700003c
:1014cc002c20000069730000207400006865000087
:1014dc00726500002061000020730000686f00003e
:1014ec00727400003f0000002e2000003c00000041
:1014fc000041000052540000310000001434000080
:10150c00040d00008206000040030000a001000052
:10151c00cf0000007f0000006700000044000000c6
:10152c002200000000000000000000002c01000060
:10153c00000000005802000000000000b004000091
:10154c00000000006009000000000000c012000054
:10155c000000000080250000000000004038000062
:10156c0000000000004b0000000000008070000034
:10157c00000000000096000000000000c0da00002f
:10158c000000000000e100000000000000c20000ac
:10159c000100000000f400000100000000e8000061
:1015ac000300000014340000040d0000820600004b
:1015bc0040030000a0010000cf0000006700000005
:1015cc0044000000220000007f0000003062000098
:1015dc0000300000303000002c00000030300000e3
:1015ec000000000014340000040d0000820600000e
:1015fc0040030000a0010000cf00000067000000c5
:10160c00440000002200000030780000303100005f
:10161c003233000034350000363700003839000012
:10162c0041420000434400004546000020480000b1
:10163c007a000000467200006571000075650000bc
:10164c006e63000069650000732000003c20000000
:10165c00314800007a200000617200006520000013
:10166c006e6f000074200000737500007070000035
:10167c006f72000074650000642e00000000000012
:10168c00436f0000756c0000646e0000277400004e
:10169c00206b000065650000702000007570000074
:1016ac000000000053500000493100000000000011
:1016bc00181c00001d0300000b1300001b00000091
:1016cc00181c00001d000000314100004c530000ac
:1016dc0001420000507600003300000021000000a1
:1016ec000010000000230000000f0000424000002a
:1016fc00400500004102000000000000002900002d
:10170c00002000005700000020520000004900009b
:10171c0032430000310000000808000008080000f7
:10172c00080000000000000042420000494f000089
:10173c003100000052410000573100000000000051
:10174c00003500003f620000610000004f430000c4
:10175c004431000000000000000000000000000008
:020000040000fa
:10176c00881f780013c4800003007800f007b200d3
:10177c000480210064407800f1ccb300814040002b
:10178c00e8cf500018003e000000fb000003b10041
:10179c008300e800f107b20064c1780006cdb30005
:1017ac0086424100e9cf52000c003e008381e800e4
:1017bc006a00b9000201fb00000041000003b10007
:1017cc0083007800f107b20064c178008301e8005f
:1017dc0086424100e9cf5200f5ff360011c4880063
:1017ec004f0478000000060001c3b300814f500085
:1017fc000700320011c0b300408821000148780076
:10180c000000eb004f04780000000600f6ff3700e4
:10181c008300e800f107b20064c1780025c6b3006c
:10182c00854f51001e00320025c4b300854f510076
:10183c001b00320085c7b300854f510038003200c1
:10184c0085c5b300854f51003500320080425100f0
:10185c000000eb00e9cf5200e0ff3e000201fb006c
:10186c0000fd2f00020040008381e80006cdb3008c
:10187c006a00b900000041000003b1008300780049
:10188c00f107b20064c178008301e8008642410090
:10189c00e9cf5200d1ff3e000201fb00f4ff3700fc
:1018ac008380e800f107b20064c1780006cdb30074
:1018bc00864241000000eb00e1cf5200c7ff3e0022
:1018cc00e3814100000040000201fb0002004000e7
:1018dc000003b10083007800f107b20064c1780006
:1018ec008301e80086424100e1cf5200bbff3e007d
:1018fc00000040000201fb00020040000003b100a8
:10190c0083007800f107b20064c178008301e8001d
:10191c0086424100e1cf5200eaff3600afff3700ac
:10192c008381e8000000eb0006cdb300f7cbb300d9
:10193c00f8c9b30083007800f107b20064c17800e5
:10194c0086424100e9cf5200130036008742410025
:10195c00e5cf52000300360088424100e5cf52002b
:10196c009eff3e000254a00002f278004400dd000d
:10197c007005b1000201fb00020040008301e80089
:10198c0083007800f107b20064c178008642410000
:10199c00e9cf5200edff3e004400dd000003b10032
:1019ac000201fb00020040008301e800f4ff370055
:1019bc0011c480000100e800f007b2000280210091
:1019cc00e241780010002000a2c3b30082cf510086
:1019dc0001003200000006008180e800f107b2002f
:1019ec0011c488005eff070011c480008100e9006b
:1019fc00f107b20011c488000000060011c4800079
:101a0c000100e800f007b20002802100e2417800fa
:101a1c000000eb00b2c3b30082cf510001003200d2
:101a2c00000006008180e800f107b20011c48800b4
:101a3c004bff070011c480008100e900f107b200e0
:101a4c0011c488000000060011c480008100e80069
:101a5c00f107b2000080210060c1780080c7b3009c
:101a6c00804f51000f00320040c6b300804f510030
:101a7c000800320020c6b300804f51000b0032002a
:101a8c000040eb0073c7b300834f510003003200da
:101a9c000000060011c488002000050011c4880055
:101aac004000050011c488001000050011c4880016
:101abc003000050010c4800002802100e241780053
:101acc0001c2b30081cf510006003a000000e800cb
:101adc00f007b200e240780083cf5000fbff3200e9
:101aec0010c4880000000600ee874700889fbe00e7
:101afc008a9fbe008c9fbe008e1f78000004be0023
:101b0c000205780003077800dcc2b3008dc7b30070
:101b1c000bcdb30060902800b265020000000000fd
:101b2c000800e0004300350008407800946802008b
:101b3c0000000000c0902800b26502000000000008
:101b4c000000eb00e0b79f00f0b79f00c66a0200f0
:101b5c000000000080407800edcf500016003200ed
:101b6c00edcf50003d003c00e8cf50005600320055
:101b7c00eacf5000100032000bc04000e94f50007b
:101b8c0044003e007fb19700e30f51005a0034002f
:101b9c0070c0b300d46a02000000000043002000b3
:101bac00f3b79f00c66a0200000000008040780076
:101bbc00edcf5000eaff3a0030912800d2650200c8
:101bcc00000000007fb097000000e0002a00320007
:101bdc008000eb000a0034007a805700ffb09700b9
:101bec00010240008000eb006a09b900b000fb0064
:101bfc000103b10082804000840f5000faff3a00cc
:101c0c00818f540002003c00810f55004c003d00b8
:101c1c00b101200080ec20006e7c0200000000006e
:101c2c0060902800b2650200000000000800e0008f
:101c3c00bdff3d00a0902800b2650200000000002e
:101c4c00c0902800b2650200000000000000eb000c
:101c5c00e0b79f00f0b79f00bcff37008ccf50005f
:101c6c00100032008dcf5000c3ff3a000e00e00090
:101c7c00c1ff32000084eb00080078004f077800a9
:101c8c004f06be004f05be004f04be00ef00b10072
:101c9c000000060070c0b300d46a0200000000000f
:101cac00aaff37007fb097000000e000f9ff3a0070
:101cbc000c407800d46a02000000000011002000e3
:101ccc00e1b79f00a1ff3700ffb097000100e000d3
:101cdc0015003a006fb197000200e000edff3200f2
:101cec00f0902800b2650200000000008001eb00bb
:101cfc00e3b79f0095ff37000140780081bf9f003c
:101d0c00d46a0200000000008fb89700814178006f
:101d1c007a8057007fb19700037079000201e800c8
:101d2c00f2b79f0089ff37008100e900f1b79f00ef
:101d3c00f0902800b26502000000000083ff37001d
:101d4c006fb197000200e000090032000104ea00c4
:101d5c00080078004f0778004f06be004f05be0004
:101d6c004f04be00ef00b10000000600c9ff3700b1
:101d7c00010078004f0778004f06be004f05be00eb
:101d8c004f04be00ef00b10000000600c1ff370099
:101d9c000e00fa00889fbe008a9fbe008c9fbe007a
:101dac0011c480008104e900f907b200180020007a
:101dbc00898f50000e0032000b8021008b067800ba
:101dcc006bc07c000004e00005003a000906e80046
:101ddc00fc07b2006d407e000004e00038003a00c1
:101dec008904e900f907b200818f5400f4ff3a002e
:101dfc0070912800d26502000000000071002000e4
:101e0c00107420006e7c0200000000001300200003
:101e1c0008017800830078000000eb0032ff070017
:101e2c008000e800e18f50004700360000004000c1
:101e3c00fa805700e101780003007800f007b20047
:101e4c000b8021006b4178000204e0004800320056
:101e5c0004c480000000eb0084004000f107b200d5
:101e6c0082f578000000e80083004000f107b20022
:101e7c006bc178000204e000f7ff3a000402e900ad
:101e8c00f407b20014c488000482e8000000420089
:101e9c00f007b20000c488000000e900f007b200af
:101eac008040eb00817578000000eb004f06be000f
:101ebc004f05be004f04be000080fa000000060073
:101ecc00084078009468020000000000409128004f
:101edc00b2650200000000006d407e000004e000ce
:101eec00090032000985e800d46a020000000000f5
:101efc000a007800f007b2006b4078000a05e80091
:101f0c000004e000f8ff3a00080044000c017800df
:101f1c00fa805700823078000804e800e70f54007c
:101f2c00b3ff320030912800d2650200000000009f
:101f3c0011c480008904e900f907b200818f5400b4
:101f4c009fff3a00aaff370030912800d2650200ab
:101f5c0000000000100020004f06be004f05be0020
:101f6c004f04be000080fa0000000600d4ff3700ca
:101f7c000000eb0004c480000402e900f407b20086
:101f8c0014c488000482e80000004200f007b2008c
:101f9c0000c488000000e900f007b2008040eb00ac
:101fac00817578000000eb00c0ff3700889fbe00f1
:101fbc008a9fbe008c1f780010c480000000e800cf
:101fcc00f007b20010c4880002802100e2417800c2
:101fdc0001c2b30081cf510006003a000000e800b6
:101fec00f007b200e240780083cf5000fbff3200d4
:101ffc0010c48800dafd07000000e0003f003a0042
:10200c000005eb000c8d21000b0320000a40e800ba
:10201c00946802000000000040912800b2650200a4
:10202c0000000000090320000bd0b9008002b000b2
:10203c00088d210000004600d2650200000000005f
:10204c000a05e800e40f5500f0ff3a00710120008a
:10205c00606d20006e7c02000000000040882100b2
:10206c000048eb00130020000a0178008300780080
:10207c00030078009cfe07000005e9000000e80062
:10208c00e10f50004c00360020cf80000980b900d1
:10209c002002b0006800780000000100147a0200f1
:1020ac00000000002acf880009d0b900fe044000cf
:1020bc0068807c000000010090912800d26502002d
:1020cc00000000000a00e00032003a00510020003d
:1020dc00505720006e7c02000000000000c48000fd
:1020ec000000e900f007b20010c488004f06780029
:1020fc004f05be004f04be00000006000004e900be
:10210c00e30f540016003c000a03200020cf80008f
:10211c000a80b9002002b000098d21006900780006
:10212c0000000100147a02000000000028cf880093
:10213c000ac5b9007e05450069007d00000001005c
:10214c000800e000e1ff3200c222a800510020008c
:10215c00505720006e7c020000000000dfff3700ab
:10216c0051012000c07220006e7c020000000000b3
:10217c0000c480000000e900f007b20010c4880021
:10218c004f0678004f05be004f04be00000006004d
:10219c00daff3700c222a800e0922800d2650200c4
:1021ac000000000051002000505720006e7c0200ff
:1021bc0000000000c9ff3700e1002000d06e2000b5
:1021cc006e7c02000000000000c480000000e900ea
:1021dc00f007b20010c488004f0678004f05be000f
:1021ec004f04be0000000600c4ff3700889fbe00ed
:1021fc008a9fbe00e0962800b26502000000000035
:10220c00e0c2b300d46a020000000000a09e2100ce
:10221c0010407800d46a02000000000031cf80002a
:10222c00f0442000808f5000ab0032003091280029
:10223c00d26502000000000030992800b26502004f
:10224c0000000000b0c5b300d46a0200000000001a
:10225c00190020000004eb000b8d21000a03200064
:10226c000800e00007003a00808f2100b2650200f0
:10227c00000000000804e8008904e8000800e00001
:10228c00f9ff320000c2b300d46a02000000000063
:10229c000ac0b9008002b00000804500b26502009f
:1022ac0000000000e38f5400f2ff3600d0c5b300ed
:1022bc00d46a020000000000d1002000a0802000a1
:1022cc00167c020000000000a1bf2a000000eb00f9
:1022dc00d869020000000000000478004840de00cd
:1022ec009468020000000000e0c2b300d46a02004f
:1022fc000000000008407800946802000000000014
:10230c0030912800d265020000000000610020001e
:10231c0030762000167c02000000000030cf8000d8
:10232c0040690200000000007100200010ec200049
:10233c00167c02000000000040cf800040690200c3
:10234c0000000000c09b2800b265020000000000e5
:10235c0031cf8000f0442000808f50003b003200d1
:10236c00c09c2800b26502000000000040cf800035
:10237c0021042300810f50003b003200810f5000dc
:10238c001300360031042300810f5000440032004a
:10239c00e3804000810f50001e003200b09d2800e9
:1023ac00b265020000000000f09d2800d26502001a
:1023bc0000000000e1012000907620006e7c0200fd
:1023cc00000000004f05be004f04be0000000600d8
:1023dc00f103b100810f5000f0ff3a00f09c28008f
:1023ec00b265020000000000f09d2800d2650200da
:1023fc0000000000e1012000907620006e7c0200bd
:10240c00000000004f05be004f04be000000060097
:10241c00efff3700809d2800b2650200000000002d
:10242c00f09d2800d265020000000000e1012000b0
:10243c00907620006e7c0200000000004f05be006c
:10244c004f04be0000000600e1ff3700909c2800fe
:10245c00b26502000000000040cf80002104230080
:10246c00810f5000c5ff3a00209d2800b265020084
:10247c0000000000f09d2800d26502000000000062
:10248c00e1012000907620006e7c0200000000002c
:10249c004f05be004f04be0000000600ccff370005
:1024ac00509d2800b265020000000000f09d28003d
:1024bc00d265020000000000e101200090762000af
:1024cc006e7c0200000000004f05be004f04be00f1
:1024dc0000000600beff3700c0972800b26502005e
:1024ec000000000030912800d265020000000000be
:1024fc0030992800b265020000000000b0c5b3009e
:10250c00d46a020000000000190020000004eb0057
:10251c000b8d21000a03200051ff3700c802b600c2
:10252c0003003a00409e2800b26504000000000041
:10253c00109e2800b265040000000000ca02b6001c
:10254c0003003a00a09e2800b265040000000000c1
:10255c00709e2800b265040000000000a10020005d
:10256c00400721006e7c0200000000006104200086
:10257c00c00c21006e7c020000000000a1012000b4
:10258c00e0072100167c0200000000000003200080
:10259c0021cf80000088b9004002b000018d2100dd
:1025ac006100780000000100a100200080092100da
:1025bc00167c02000000000000402000d7ff07003e
:1025cc0000102000d5ff070000202000d3ff0700db
:1025dc0000042000d1ff070000082000cfff0700f7
:1025ec0030912800d265020000000000410020005c
:1025fc0020112100167c02000000000021e3a8003d
:10260c00a0002000567a020000000000926902002f
:10261c000000000011002000b0372000167c0200e2
:10262c000000000090c0b300d46a0200000000005b
:10263c0090002000567a020000000000926902000f
:10264c000000000011002000b0372000167c0200b2
:10265c000000000090c0b300d46a0200000000002b
:10266c00c0002000567a02000000000092690200af
:10267c000000000011002000b0372000167c020082
:10268c000000000090c0b300d46a020000000000fb
:10269c00b0002000567a020000000000926902008f
:1026ac000000000011002000b0372000167c020052
:1026bc000000000090c0b300d46a020000000000cb
:1026cc0021e3a900004020009cff0700001020001f
:1026dc009aff07000020200098ff0700000420004c
:1026ec0096ff07000008200094ff07003091280097
:1026fc00d265040000000000881f78005100200003
:10270c0050922000167c020000000000c1bf2a007d
:10271c000000eb00d86902000000000040690200d4
:10272c000000000061002000a0922000167c020036
:10273c0000000000e1bf2a000000eb00d869020095
:10274c0000000000406902000000000030912800e9
:10275c00d265020000000000c1002000707820004b
:10276c006e7c0200000000007cff0700c202ab0080
:10277c008000320011012000a0622000167c0200b3
:10278c0000000000c0c2b300d46a020000000000c8
:10279c0000c2b300d46a020000000000cb62ab00a0
:1027ac006f00320041012000705d2000167c020099
:1027bc0000000000c0c2b300d46a02000000000098
:1027cc0000c2b300d46a020000000000889c210003
:1027dc009840780070c060005c003200210220003c
:1027ec00307920006e7c02000000000098407800d8
:1027fc0068c060002a003a00b1012000307d200042
:10280c00167c020000000000c0c2b300d46a0200b3
:10281c000000000000c2b300d46a020000000000f7
:10282c00b1012000b01a2100167c0200000000004b
:10283c00709b21001040780094680200000000009a
:10284c0030912800d2650200000000001844780086
:10285c0063406400e14f50002a0032006101200007
:10286c00a05720006e7c0200000000000003200036
:10287c0021cf80000088b9006002b000018d2100da
:10288c006100780000000100c10020007078200079
:10289c006e7c0200000000004f047800000006006f
:1028ac00c1012000e07e2000167c02000000000028
:1028bc00c0c2b300d46a02000000000000c2b30022
:1028cc00d46a020000000000b1012000b01a2100ff
:1028dc00167c020000000000709b21001040780064
:1028ec00946802000000000030912800d2650200bc
:1028fc00000000001844780063406400e14f500071
:10290c00d6ff3a0051012000005920006e7c0200d5
:10291c00000000000003200021cf80000088b900d7
:10292c006002b000018d2100610078000000010000
:10293c00c1002000707820006e7c020000000000b6
:10294c004f04780000000600d5ff3700e10120009d
:10295c00507b20006e7c020000000000a3ff3700bb
:10296c0051012000205c2000167c020000000000b9
:10297c0090ff370021012000b0632000167c02007c
:10298c00000000007fff370010c480000000e8004a
:10299c00f007b20010c4880002802100e2417800e8
:1029ac0001c2b30081cf510006003a000000e800dc
:1029bc00f007b200e240780083cf5000fbff3200fa
:1029cc0010c4880066fb07000000e900e30f50000c
:1029dc0005003e0010cf88002101200090832000cc
:1029ec006e7c040000000000408821000048eb00d1
:1029fc0021022000708120006e7c0200000000008b
:102a0c008001eb004200200011002000100020008b
:102a1c0035fc0700219e21008008e90021012000df
:102a2c00908320006e7c040000000000eeff370055
:102a3c00889fbe008a1f780010c480000000e80048
:102a4c00f007b20010c488000880210068417800ab
:102a5c0001c2b300814f510006003a000000e800ab
:102a6c00f007b200e840780082cf5000fbff320044
:102a7c0010c488003afb07000040e900e94f500001
:102a8c001d003e00099e2100804c78000045eb00a3
:102a9c002a00320041012000309020006e7c0200a0
:102aac000000000011012000a01921006e7c020022
:102abc00000000000c6a0200000000000004e000ae
:102acc00fcff320090c0b300994f10003e00320062
:102adc00ec6902000000000008c2b300c66a0200e4
:102aec0000000000884f5000fcff3a004f057800b2
:102afc004f04be0000000600408821000048eb0097
:102b0c00d1082000608720006e7c020000000000cd
:102b1c008001eb00a200200011002000900020009a
:102b2c00f1fb07000040e900099e2100804c780071
:102b3c000045eb00e94f5000d6ff3a0010c480006e
:102b4c006841780001c2b300814f510006003a0081
:102b5c000000e800f007b200e840780082cf500097
:102b6c00fbff320010c48800fdfa07000045780016
:102b7c000004e000c7ff3a0041882100804878003b
:102b8c00d09e2800d2650200000000008001eb00fe
:102b9c00f2ff27008000eb0020022000d2fb070090
:102bac000045780041012000309020006e7c02002e
:102bbc000000000011012000a01921006e7c020011
:102bcc0000000000bbff37000a407800e66a0200f4
:102bdc0000000000ec6902000000000008c2b30015
:102bec00beff3700f8874700889fbe008a9fbe0053
:102bfc008c9fbe008e1f78000000eb0010c4880074
:102c0c0000c48800409e21000008eb004d88210084
:102c1c00804eeb008001eb005a882100020220005c
:102c2c007818b9008000e9008a8040000000eb00b1
:102c3c008068eb000000e800820f5000fcff3a00b7
:102c4c008301e800e38f5100f5ff3a000000eb0030
:102c5c0070c688000006eb008cb79f00acb79f00d5
:102c6c000b8d210009802100889c210071075400e4
:102c7c000003200021cf80000088b9008002b00042
:102c8c0000804500b26502000000000050a0280042
:102c9c00b2650200000000000000eb00c0b79f000e
:102cac0070c680000000e0001b0032000000e9004c
:102cbc0070c688007800b9006a4078000004e00013
:102ccc001300320002c480008000eb00dcb79f00d0
:102cdc000106780080747900d46a020000000000bc
:102cec000c06e80002c480000201e800f207b20002
:102cfc0002c4880070c680007800b900000046004d
:102d0c006a4078000004e000f2ff3a005fb69700da
:102d1c000000eb0070c68800146a0200000000007e
:102d2c000004e00028003a009840780064c060007d
:102d3c00f9ff320020cf8000020320000280b9008e
:102d4c007a0040006b007800000001000004e000f5
:102d5c00f1ff320020cf8000030320000380b90074
:102d6c008002b000048d210004004000b265020016
:102d7c000000000050a02800b26502000000000016
:102d8c0011c4800000c48000808f5000e2ff32002c
:102d9c0069c07800e1b79f00d46a0200000000000f
:102dac00efb09700f107b2008100e80000c480008a
:102dbc00808f5000f6ff3a00146a020000000000f9
:102dcc000004e000d8ff3200ec6a020000000000b2
:102ddc000004e00003003200f26a02000000000070
:102dec00afff3700c66a0200000000008040780088
:102dfc000181fb008001eb00f5072000850f5100dd
:102e0c00e08f59003b00360002c480000200e8004d
:102e1c00f007b20013c48000830f5000f50032009d
:102e2c00ffcf5000f3003600e0c7b30080cf500056
:102e3c00f0003e00820f56006c083200b0a0280053
:102e4c00e1b79f0082bf9f00b26502000000000046
:102e5c000fb997000c005100f007b2009468020003
:102e6c0000000000a0a12800b265020000000000d4
:102e7c0002c480008c01e900f307b200efb09700a8
:102e8c00828f51000e0032000c027800014678004f
:102e9c0002804400e94279001540980069407900ad
:102eac000004e00069023a000201e900f207b200f6
:102ebc00828f5100f6ff3a008c40780004067800af
:102ecc0001407800e1b79f00d46a020000000000c6
:102edc00efb0970081747e000c06e800fc07b2008e
:102eec0000c480000000e800f007b20000c48800b5
:102efc006bff37000260010013023700010237003c
:102f0c00ef013700c0ff3700c001370090003700d9
:102f1c00b5013700bcff370082013700baff37001c
:102f2c00b8003700b8ff3700b7ff3700b5003700df
:102f3c000d023700b4ff370096003700b2ff3700a0
:102f4c00b1ff3700b0ff3700afff3700aeff3700df
:102f5c00adff3700acff3700abff3700aaff3700df
:102f6c00a9ff370064003700a7ff3700a6ff370022
:102f7c00a5ff3700a4ff3700a3ff3700a2ff3700df
:102f8c00a1ff3700a0ff37009fff37009eff3700df
:102f9c009dff37009cff37009bff37009aff3700df
:102fac0099ff370098ff370097ff370096ff3700df
:102fbc0095ff370094ff370093ff370092ff3700df
:102fcc0091ff370090ff37008fff37008eff3700df
:102fdc008dff37008cff37008bff37008aff3700df
:102fec0089ff370088ff370087ff370086ff3700df
:102ffc0085ff370084ff370083ff370082ff3700df
:10300c0081ff370080ff37007fff37007eff3700de
:10301c007dff37007cff37007bff37007aff3700de
:10302c0079ff370078ff370077ff370076ff3700de
:10303c0075ff370074ff370073ff370072ff3700de
:10304c0071ff370070ff37006fff37006eff3700de
:10305c006dff37006cff37006bff37006aff3700de
:10306c0069ff370068ff370067ff370066ff3700de
:10307c0065ff370064ff370063ff370062ff3700de
:10308c0061ff370060ff37005fff37005eff3700de
:10309c005dff37005cff37005bff37005aff3700de
:1030ac0059ff370058ff370057ff370056ff3700de
:1030bc0055ff370054ff370053ff370052ff3700de
:1030cc0051ff370050ff37004fff37004eff3700de
:1030dc004dff37004cff37004bff37004aff3700de
:1030ec0049ff370048ff370047ff370046ff3700de
:1030fc0045ff370045013700c66a0200000000009a
:10310c00b1c5b300814f5000e5fe3a00c66a02001b
:10311c000000000011c4b300814f50001d003200ac
:10312c0060013e00f0c05000814f50007001320031
:10313c00e3c04000814f5000d9fe3a00c66a02003d
:10314c0000000000e1c7b300814f5000d4fe3a00ec
:10315c0001c48000810f560026003200b0a0280068
:10316c00e1b79f00b265020000000000efb09700cd
:10317c000c805000f007b2009468020000000000c0
:10318c00a0a12800b2650200000000000cc4800061
:10319c00c3fe370016c480008600e900f107b200b8
:1031ac0000c48000808f5000120032000002eb003f
:1031bc00cfb39700d0b79f0069c178000204e0003c
:1031cc00fb063a000101e900f207b200058021007c
:1031dc00e54179000304e000030032000402e8003a
:1031ec00870f52002c063e0082007800808f500022
:1031fc00f1ff3a0070c0b300d46a02000000000076
:10320c00a7fe37000cc480000040eb0080747e00e9
:10321c000c06e800fc07b2000cc4880030912800b2
:10322c00d26502000000000005c4800095b79f0025
:10323c0010c48000d0b79f00804eeb000041eb0023
:10324c00c2df9f00fcaf9f00694178000281fb0048
:10325c008001eb00e1072000810f5100e08f590045
:10326c001e00360011c0b300814e78000000e8004b
:10327c00f007b20010c488000001eb001d04e00050
:10328c0096003a0001c48000808f5000020032008a
:10329c000200e000ecff32007fae97001fb19700f8
:1032ac0012c4880002c488000003200021cf8000d3
:1032bc000088b9008002b00000804500b2650200b1
:1032cc000000000050a02800b265020000000000c1
:1032dc000000eb00c0b79f0071fe370002600100d8
:1032ec00e2ff3700dfff3700deff3700ddff37007e
:1032fc00dcff3700dbff3700daff3700d9ff370080
:10330c00d8ff3700d7ff3700d8ff3700d5ff37007d
:10331c00d4ff3700d5ff3700d2ff3700d1ff37007d
:10332c00d0ff3700cfff3700ceff3700cdff37007f
:10333c00ccff3700cbff3700caff3700c9ff37007f
:10334c00c8ff3700c7ff3700c6ff3700c5ff37007f
:10335c00c4ff3700c3ff3700c2ff3700c1ff37007f
:10336c00c2ff370058013700d8023700c6023700b9
:10337c003e03370025033700ab023700b9ff370097
:10338c008b023700b7ff3700b6ff3700b5ff3700a9
:10339c00b6ff3700740237005f0237002602370091
:1033ac00b7013700b6013700b5013700b40137005b
:1033bc00b3013700b2013700b1013700b00137005b
:1033cc00af013700ae013700a6ff3700a5ff37006d
:1033dc002b02370087013700a2ff37007b01370033
:1033ec005b0137003f0437009eff37002d04370088
:1033fc00220437009bff37009aff370099ff3700f4
:10340c0098ff370097ff370096ff370095ff37007e
:10341c000a04370093ff370092ff370091ff370003
:10342c003d0437008fff37008eff3700f60337005f
:10343c008cff37008bff37008aff3700c80337003b
:10344c0088ff370087ff370086ff3700b703370048
:10345c00a403370095033700780337006503370062
:10346c0080ff3700560337004c0337003d0337000d
:10347c00270337007bff3700210537001305370082
:10348c0003053700f504370076ff370075ff37006a
:10349c002e0537002405370072ff37004e04370025
:1034ac00390437006fff3700870437006dff370092
:1034bc006cff37006bff37007a0437005d04370070
:1034cc0068ff370067ff370066ff37004b04370093
:1034dc00bd04370000033700ec0037005101200019
:1034ec00106c2000167c02000000000010c480004c
:1034fc00dfb29700808f5200370631000540500034
:10350c009468020000000000804eeb00309128000f
:10351c00d26502000000000010c4800012002000e0
:10352c0058ff370010c48000800f560031ff320066
:10353c0000c48000800f56005c0632000c06e900c7
:10354c00fc07b20070a02800b26502000000000069
:10355c0000c480000001eb00800f56001300320005
:10356c008c017800dcb79f000306e80069407e0000
:10357c0080f479000004e00001003a0000c2b300be
:10358c0082bf9f00d46a0200000000000fb99700b0
:10359c000201e8008c017800f307b20000c480003f
:1035ac00808f5100f0ff3a005fb697000000e900f1
:1035bc00f007b20000c48800b0a0280082bf9f00b2
:1035cc00b2650200000000000fb9970002407800bd
:1035dc009468020000000000e0a02800b265020020
:1035ec0000000000aefd370000c48000800f5600c4
:1035fc0000ff32000c06e800fc07b20000a1280016
:10360c00b265020000000000a5fd370000c4800078
:10361c00800f5600f7fe32008c0178000001eb00a1
:10362c00dcb79f000306e80069407e0080f4790057
:10363c000004e00001003a0000c2b30082bf9f000a
:10364c00d46a0200000000000fb997000201e800e4
:10365c008c017800f307b20000c48000808f510009
:10366c00f0ff3a005fb697008301e900f307b20060
:10367c0003c48800b0a0280082bf9f00b26502007e
:10368c00000000000fb99700024078009468020017
:10369c0000000000e0a02800b2650200000000005d
:1036ac007ffd370031c4b300814f5000ceff320094
:1036bc002d0039008140e800814f500078fd3a0020
:1036cc008fb09700e48f5000e7053c0010c48000d9
:1036dc00800f5600c7fe32000c06e900fc07b20052
:1036ec0070a02800b2650200000000006cfd3700dd
:1036fc00c66a020000000000e1c7b300814f500011
:10370c0067fd3a0011c48000810f5600b9fe3200eb
:10371c00b0a02800e1b79f00b265020000000000d5
:10372c00efb0970001005600f007b2009468020059
:10373c0000000000e0a02800b265020000000000bc
:10374c001cc4800056fd37008fb197008301e80040
:10375c0083b79f00f48f510051fd3a00887302002b
:10376c00000000004efd370017c480008700e90000
:10377c00f107b20000c48000808f500013003200ab
:10378c000002eb004fb197000203e900d0b79f0095
:10379c0069c178000204e0008a053a000101e900e1
:1037ac00f207b20005802100e54179000304e00036
:1037bc00030032000402e800840f5300730432004b
:1037cc0082007800808f5000f1ff3a00cfb0970054
:1037dc00e18f500087fe3a0040a12800b26502003c
:1037ec00000000000003200021cf80000088b900f9
:1037fc008002b00000804500b265020000000000ad
:10380c0050a02800b2650200000000000cc480002b
:10381c0010c48000800f5600070032000041eb00fe
:10382c0082747e000c06e900fc07b200800f560083
:10383c00faff3a000cc488008041eb0083747e00d0
:10384c000002eb00c4b79f0015fd370082bf9f003c
:10385c00e3b79f00f4b79f00d46a02000000000099
:10386c00c0a12800b2650200000000007fb29700e2
:10387c00efb197000fb997000201e900f207b2000f
:10388c00828f510082fd3a008bfd370020cf8000e3
:10389c000000e00079053a0011c0b3000140780047
:1038ac00726f02000000000010c480000000e800ed
:1038bc00f007b20010c488000001eb001d04e0000a
:1038cc0070fe320005ff370039f80700000678005b
:1038dc00a1002000706b2000167c0200000000008c
:1038ec000c00e0000e00320020cf8000040320000a
:1038fc000480b900780040006b00780000000100e3
:10390c000080fb00626502000000000000c2b300f2
:10391c00d46a0200000000000c06e900f2ff3a0035
:10392c0001012000a06920006e7c02000000000054
:10393c0010c480000000e800f007b20010c488003a
:10394c000001eb001d04e0004efe3200e3fe3700e8
:10395c0017f80700000678000c00e000f4ff3200b6
:10396c006101200040612000167c02000000000074
:10397c000e5402000000000062650200000000000e
:10398c0030912800d2650200000000000c06e9000e
:10399c00e7ff32006101200040612000167c02002c
:1039ac00000000000e5402000000000062650200de
:1039bc000000000030912800d265020000000000d9
:1039cc000c06e900e6ff3a00d9ff3700767c0200ce
:1039dc000000000010c480000000e800f007b200f6
:1039ec0010c488000001eb001d04e00025fe32002d
:1039fc00bafe37000000e800f007b20010c48800df
:103a0c006941780001c2b300814f510006003a00b1
:103a1c000000e800f007b200e940780082cf5000c7
:103a2c00fbff320010c488004df707000006780039
:103a3c000c007800086902000000000040a4280077
:103a4c00b2650200000000000c407800946802008f
:103a5c000000000040a42800b26502000000000035
:103a6c000c4078000666020000000000309128002f
:103a7c00d26502000000000010c48000adff3700ca
:103a8c007100200010662000167c0200000000006f
:103a9c0033f70700c0b79f0010c480000000e90096
:103aac00f007b20010c48800c1f707000006e80058
:103abc00d2f707000000e00004003200004f78004d
:103acc00e80f5000020534001854a0000c06e90061
:103adc00300032004fb09700e87a0200000000007e
:103aec00184078000058a300c804320005c1b30088
:103afc009ecf120007003200b0c3b300d46a02009c
:103b0c00000000001e4078009468020000000000d5
:103b1c00184078000038a30029003a0020cf80001c
:103b2c00020320000280b90068004000eb0078001e
:103b3c004fb0970001000100b0b79f0000c2b30066
:103b4c00d46a02000000000003c4b30018c0610076
:103b5c00deff32006100200080662000167c02002f
:103b6c0000000000849c2100144278006840620030
:103b7c0026003a003fb09700e87a020000000000ef
:103b8c0000c2b300d46a0200000000000c06e90079
:103b9c00d0ff3a0030912800d265020000000000ee
:103bac0010c480000000e800f007b20010c48800c8
:103bbc000001eb001d04e000b2fd320047fe3700af
:103bcc004fb09700f07b020000000000c0b79f00d0
:103bdc0020cf8000020320000280b9006800400062
:103bec00eb0078004fb0970001000100b0b79f00c8
:103bfc0000c2b300d46a02000000000003c4b3008a
:103c0c0018c06100b1ff3200d2ff37003fb09700ff
:103c1c00f07b020000000000b0b79f003fb097009f
:103c2c00e87a02000000000000c2b300d46a02006f
:103c3c0000000000d5ff370081002000e066200066
:103c4c006e7c0200000000000003200021cf8000e9
:103c5c000088b9006c0040006b0078000000010087
:103c6c0010c480000000e800f007b20010c4880007
:103c7c000001eb001d04e00082fd320017fe37004e
:103c8c0013c0b300834e78008000e800f107b20047
:103c9c00e9c078000104e00074fd3200120020003d
:103cac00e5c3b30085cf5000130032000201e800d9
:103cbc0080004100f107b200e9c078000104e00087
:103ccc00f7ff3a0041882100834e7800fa0f51002b
:103cdc00b503340012c0b300824878000000e8003d
:103cec00f007b20010c488000001eb001d04e000d6
:103cfc0064fd3200f9fd37008041eb000201e80061
:103d0c0080004100f107b200e9c078000104e00036
:103d1c00e3ff3a00ebff3700c1002000d064200025
:103d2c00167c0200000000000003200021cf800060
:103d3c000088b900740040006b007800000001009e
:103d4c00626502000000000010c480000000e80062
:103d5c00f007b20010c488000001eb001d04e00065
:103d6c0048fd3200ddfd3700e1002000e067200057
:103d7c006e7c0200000000000003200021cf8000b8
:103d8c000088b900700040006b0078000000010052
:103d9c0010c480000000e800f007b20010c48800d6
:103dac000001eb001d04e00036fd3200cbfd3700b6
:103dbc000000e800f007b20010c4880068f60700a5
:103dcc0011c48000e9c1780002c2b30082cf510057
:103ddc0006003a008100e800f107b20069c17800e2
:103dec00834f5100fbff320011c48800f107b20071
:103dfc0069c1780091c2b300814f51007004320048
:103e0c0010c0b300804e780010c480000000e800a1
:103e1c00f007b20010c488000001eb001d04e000a4
:103e2c0018fd3200adfd3700e1f607000006780002
:103e3c006100200090652000167c0200000000004c
:103e4c000c007800e8660200000000002100200051
:103e5c00f06520006e7c0200000000000c00780071
:103e6c009e7b02000000000010c480000000e800ef
:103e7c00f007b20010c488000001eb001d04e00044
:103e8c0000fd320095fd37005100200050602000ed
:103e9c006e7c0200000000000c6a020000000000b2
:103eac000004e000fcff32000000fe0010c48000a3
:103ebc000000e800f007b20010c488000001eb001d
:103ecc001d04e000effc320084fd370013c0b3008a
:103edc00834e78008000e800f107b200e9c078005a
:103eec000104e000e1fc32000081e80024c2b300d0
:103efc0084cf50003d00320082007800f107b20000
:103f0c00e9c078000201e8000104e000f7ff3a0084
:103f1c00834e78000304e000d4fc3a0071002000ca
:103f2c0010662000167c02000000000020c2b300c6
:103f3c00d46a02000000000011c480008100e80077
:103f4c00f107b2000080210060c0780025c2b300e8
:103f5c00854f5000160032000c03200011c488005d
:103f6c00d46a02000000000010c480006940780090
:103f7c000000fb0018417800e840610044033a005f
:103f8c0022cf80000c91b90068014100eb00790050
:103f9c000100010011c480008100e800f107b200ab
:103fac0069c0780023c2b300834f5000ebff3a0086
:103fbc0011c4880020c2b300d46a020000000000c3
:103fcc0030912800d26502000000000010c480006f
:103fdc000000e800f007b20010c488000001eb00fc
:103fec001d04e000a7fc32003cfd37008041eb00d3
:103ffc0082007800f107b200e9c078000201e80005
:10400c000104e000b9ff3a00c1ff370068f6070071
:10401c00000678006100200090652000167c0200ec
:10402c00000000000c007800e866020000000000b0
:10403c002100200030ee20006e7c02000000000009
:10404c000c007800cc7b02000000000010c4800043
:10405c000000e800f007b20010c488000001eb007b
:10406c001d04e00087fc32001cfd3700007d0200bf
:10407c00000000000004e0002dfe3200a100200032
:10408c00a06020006e7c02000000000040062000b2
:10409c00cc7b020000000000147a0200000000003b
:1040ac000c6a0200000000000004e000fcff32007b
:1040bc0081bf2a000140010010c480000000e8000c
:1040cc00f007b20010c488000001eb001d04e000f2
:1040dc006cfc320001fd37000003200021cf800072
:1040ec000088b900660040006b00780000000100f9
:1040fc0010c480000000e800f007b20010c4880073
:10410c000001eb001d04e0005efc3200f3fc370004
:10411c00f1002000c0362000167c020000000000d8
:10412c00647a02000000000011002000b03720006b
:10413c00167c02000000000030912800d2650200bd
:10414c000000000010c480000000e800f007b2007e
:10415c0010c488000001eb001d04e00049fc320093
:10416c00defc3700c0cfb300184c600061012000aa
:10417c00a05720006e7c02000000000010c48000dc
:10418c000000e800f007b20010c488000001eb004a
:10419c001d04e0003bfc3200d0fc370024fa070081
:1041ac0010c480000000e800f007b20010c48800c2
:1041bc000001eb001d04e00032fc3200c7fc3700ac
:1041cc00fbf50700000678000c00e000d8fd32007b
:1041dc00ec530200000000000c06e900d4fd320094
:1041ec00ec530200000000000c06e900f8ff3a0056
:1041fc00cffd3700e1002000c06820006e7c02007b
:10420c00000000000003200021cf80000088b900ce
:10421c00720040006b0078000000010010c48000a8
:10422c000000e800f007b20010c488000001eb00a9
:10423c001d04e00013fc3200a8fc3700dcf507007d
:10424c0000067800d1002000a06a2000167c020035
:10425c00000000000c007800e87a0200000000006a
:10426c000c00e0004bfe320020cf80000303200046
:10427c000380b900760040006b007800000001005c
:10428c000c06e90043fe320020cf8000030320001f
:10429c000380b900760040006b007800000001003c
:1042ac000c06e900f0ff3a003afe3700000320004c
:1042bc0021cf80000088b900640040006b007800ba
:1042cc000000010010c480000000e800f007b200fc
:1042dc0010c488000001eb001d04e000e9fb320073
:1042ec007efc370081002000606720006e7c02009d
:1042fc00000000000003200021cf80000088b900de
:10430c006e0040006b0078000000010010c48000bb
:10431c000000e800f007b20010c488000001eb00b8
:10432c001d04e000d7fb32006cfc370000032000ba
:10433c0021cf80000088b9006b00780000000100dc
:10434c0010c480000000e800f007b20010c4880020
:10435c000001eb001d04e000cafb32005ffc3700db
:10436c0020cf80000000e000b3023200c002a900a0
:10437c00c202a80021e3a80020002000cc7b020090
:10438c0000000000a0002000567a0200000000008f
:10439c00011b2000810f5000060036009000200009
:1043ac00567a020000000000712b2000810f500093
:1043bc006c023e00c002a900c202a900a0a5280000
:1043cc00d26502000000000021012000b063200033
:1043dc00167c02000000000030912800d26502001b
:1043ec000000000021e3a90010c480000000e800d8
:1043fc00f007b20010c488000001eb001d04e000bf
:10440c00a0fb320035fc370020cf80000000e0001c
:10441c0089023200385402000000000010c48000f1
:10442c000000e800f007b20010c488000001eb00a7
:10443c001d04e00093fb320028fc37001834a00068
:10444c00c1012000e07e2000167c0200000000006c
:10445c0030912800d26502000000000010c48000da
:10446c000000e800f007b20010c488000001eb0067
:10447c001d04e00083fb320018fc37007c7a02003c
:10448c000000000010c480000000e800f007b2003b
:10449c0010c488000001eb001d04e00079fb320021
:1044ac000efc3700184078000000a0000014a1009a
:1044bc00004c780051012000005920006e7c020055
:1044cc000000000010c480000000e800f007b200fb
:1044dc0010c488000001eb001d04e00069fb3200f1
:1044ec00fefb370032f50700000678000c00e000f8
:1044fc000ffd3200ca530200000000000c06e90058
:10450c000bfd3200ca530200000000000c06e9004b
:10451c00f8ff3a0006fd370020cf80000000e000d5
:10452c00450232001842780070406200f8013200f7
:10453c00c962a800cb62a90041012000705d200077
:10454c00167c02000000000030912800d2650200a9
:10455c000000000021e3a800b0002000567a020001
:10456c0000000000f1042000810f50009dff3e0070
:10457c0010a22800d26502000000000021e3a9006f
:10458c0010c4800099ff370020cf80000000e000ad
:10459c0029023200cb62a900c962a9005101200096
:1045ac00205c2000167c02000000000030912800e6
:1045bc00d26502000000000010c480000000e8007a
:1045cc00f007b20010c488000001eb001d04e000ed
:1045dc002cfb3200c1fb3700ebf8070010c4800045
:1045ec000000e800f007b20010c488000001eb00e6
:1045fc001d04e00023fb3200b8fb37000003200051
:10460c0021cf80000088b9000080e8006b007800a2
:10461c000000010010c480000000e800f007b200a8
:10462c0010c488000001eb001d04e00015fb3200f3
:10463c00aafb370020cf80000000e000fe01320012
:10464c00010320000180b9002002b0006b0078004b
:10465c000000010090912800d265020000000000cb
:10466c00c002a900c202a90021012000b0632000f1
:10467c00167c02000000000030912800d265020078
:10468c000000000010c480000000e800f007b20039
:10469c0010c488000001eb001d04e000f9fa3200a0
:1046ac008efb3700adf7070010c480000000e80057
:1046bc00f007b20010c488000001eb001d04e000fc
:1046cc00f0fa320085fb3700610020008066200084
:1046dc00167c020000000000dbf4070080ef9f0056
:1046ec00b3f4070000067800c4f407000000e000f3
:1046fc0004003200004f7800e80f50001202340022
:10470c001854a0008fea97000504e0000500320061
:10471c0010cf8000c0df9f000580fb00219e210090
:10472c008008e9000c00e0001c00320020cf800063
:10473c00020320000280b9006a0040006b00780080
:10474c000000010098417800e8c061005f013a0068
:10475c00e87a02000000000004c2b30018406200b6
:10476c006101320000c1b3009e4f10000600320000
:10477c00b0c3b300d46a0200000000001e407800f1
:10478c00946802000000000000c2b300d46a02006a
:10479c00000000000c06e900e4ff3a008fe89700e7
:1047ac000104e000fbfc32004fd997000280fb00b3
:1047bc0010cf880030912800d26502000000000064
:1047cc0010c48000f7fc37000000e800f007b200ce
:1047dc0010c488006941780001c2b300814f5100b8
:1047ec0006003a000000e800f007b200e94078004b
:1047fc0082cf5000fbff320010c48800d8f30700b2
:10480c000080fb00f07b0200000000000006780036
:10481c000c007800086902000000000040a4280089
:10482c00b2650200000000000c40780094680200a1
:10483c000000000040a42800b26502000000000047
:10484c000c40780006660200000000003091280041
:10485c00d26502000000000087fc370063f60700f9
:10486c0020cf80000000e00031fc3200a2f70700ee
:10487c0010c480000000e800f007b20010c48800eb
:10488c000001eb001d04e0007efa320013fb370040
:10489c003ff507000000e00025fc3a0012c4800040
:1048ac00d2b79f000200780003c4800093b79f002a
:1048bc000000e800f007b20010c488000001eb0013
:1048cc001d04e0006ffa320004fb370020cf80009b
:1048dc000000e000580132007e4d02000000000094
:1048ec0010c480000000e800f007b20010c488007b
:1048fc000001eb001d04e00062fa3200f7fa370009
:10490c00665002000000000010c480000000e800a7
:10491c00f007b20010c488000001eb001d04e00099
:10492c0058fa3200edfa3700a0f5070010c48000e9
:10493c000000e800f007b20010c488000001eb0092
:10494c001d04e0004ffa3200e4fa37001834a100dd
:10495c00b1012000307d2000167c02000000000018
:10496c0030912800d26502000000000010c48000c5
:10497c000000e800f007b20010c488000001eb0052
:10498c001d04e0003ffa3200d4fa3700dfb2970082
:10499c00c6b79f00808f53000b0032000040eb0025
:1049ac0080f47a008502e900f507b200858f530088
:1049bc00faff3a0007c48800008021008041eb0018
:1049cc0003f07b0007007800800f510007003200d5
:1049dc00e94179000304e0003f0132000201e900e3
:1049ec00f207b200800f5100f9ff3a0040a12800f5
:1049fc00e1b79f00b2650200000000000003200038
:104a0c0022cf80000091b9008002200002004000fb
:104a1c0000804500b26502000000000050a0280094
:104a2c00b265020000000000efb097002fb29700b3
:104a3c00810f52003e0132002fb6970069407e0074
:104a4c00e1b79f00d46a02000000000000c480009f
:104a5c006cf07c000000e800f007b20000c4880095
:104a6c000c06e800fc07b200efb09700810f56006f
:104a7c00f2ff3a00000678000040eb0080747e00e4
:104a8c00810f560086f83a00cfb09700e18f5000a6
:104a9c00d8f93a0050fb3700dfb29700cfb197003e
:104aac008301e800c3b79f00800f53000a00320057
:104abc000042eb0084f47a008502e900f507b200ad
:104acc00850f5300faff3a0006c4880000802100cd
:104adc0004707b0006007800800f51000700320044
:104aec00e94179000304e000190132000201e900f8
:104afc00f207b200800f5100f9ff3a0040a12800e4
:104b0c00e1b79f00b2650200000000000003200026
:104b1c0022cf80000091b9008002200002004000ea
:104b2c0000804500b26502000000000050a0280083
:104b3c00b265020000000000efb09700afb2970022
:104b4c00818f5200180132002fb6970069407e0009
:104b5c00e1b79f00d46a02000000000000c480008e
:104b6c006cf07c000000e800f007b20000c4880084
:104b7c000c06e800fc07b200efb09700810f56005e
:104b8c00f2ff3a00000678008041eb0083747e004f
:104b9c00810f560042f83a0070c0b300d46a02008c
:104bac00000000003ef837000304e000aff93a00c3
:104bbc000000e800f007b20010c48800e1b79f00c5
:104bcc00e7f207000006780010c4800000017800ae
:104bdc00f207b20003802100e3417900d2c3b30095
:104bec00efb0970082cf5100160132000c00e000ac
:104bfc000b013a00518821001c0020000c40780069
:104c0c00e1b79f009468020000000000a0a72800f4
:104c1c00b2650200000000006fb09700b2650200a0
:104c2c000000000050a02800d26502000000000027
:104c3c000c06e800efb09700f8804000e40f560037
:104c4c003bfb32000c407800e1b79f0094680200f7
:104c5c0000000000a0a72800b265020000000000c0
:104c6c006fb09700b26502000000000050a0280051
:104c7c00d2650200000000000c06e800efb09700bf
:104c8c00f8804000e40f5600dcff3a0028fb3700a8
:104c9c00f07b02000000000022cf80000c91b900d4
:104cac0068014100eb0079000100010011c4800093
:104cbc008100e800f107b20069c0780023c2b3009c
:104ccc00834f5000a5fc3a00b9fc3700f07b020082
:104cdc0000000000e87a02000000000004c2b300eb
:104cec00184062009ffe3a0085c0b3009ecf1200b0
:104cfc00a5fe3200b0c3b300d46a0200000000006d
:104d0c001e40780094680200000000009efe3700f0
:104d1c0021022000f0e920006e7c0200000000005f
:104d2c00c962a800cb62a90041012000705d20007f
:104d3c00167c02000000000030912800d2650200b1
:104d4c000000000021e3a800b0002000567a020009
:104d5c0000000000f1042000810f5000a1fd3e0076
:104d6c0003fe370011012000a0622000167c020017
:104d7c000000000030912800d26502000000000005
:104d8c000003200021cf80000088b9000002b00091
:104d9c006b0078000000010080a42800d26502009e
:104dac000000000021e3a90010c480008ffd370033
:104dbc008100e900f107b200808f5000fef83a0044
:104dcc000cf937008100e900f107b200808f500028
:104ddc006ffa3a007dfa370001c8b3000140400079
:104dec00afe89700014050009468020000000000fa
:104dfc00804eeb0030912800d265020000000000cc
:104e0c0010c48000120020001ef9370084c0b300cb
:104e1c009e4f12003ffb3200b0c3b300d46a0200b5
:104e2c00000000001e4078009468020000000000a2
:104e3c001840780037fb3700d1012000505a200071
:104e4c006e7c02000000000010c480000000e8002e
:104e5c00f007b20010c488000001eb001d04e00054
:104e6c0008f932009df93700b27d02000000000005
:104e7c000001eb0082b79f0089f73700a1012000e9
:104e8c00b05e20006e7c02000000000010c48000a8
:104e9c000000e800f007b20010c488000001eb002d
:104eac001d04e000f7f832008cf937000c06e9001d
:104ebc00fc07b2000cc488000040eb0080747e003c
:104ecc00f0902800b26502000000000074f7370073
:104edc001854a100fdfa37000201e800f207b200f5
:104eec00a2b79f0040a12800e1b79f00b265020065
:104efc00000000000003200022cf80000091b900c8
:104f0c00800220000200400000804500b2650200d3
:104f1c000000000050a02800b26502000000000054
:104f2c00efb097002fb29700810f5200c2fe3a00eb
:104f3c000cc480000040eb0080747e00810f560092
:104f4c0057f73a00d0fe37001854a100edfd37009a
:104f5c000201e800f207b200a2b79f0040a12800ae
:104f6c00e1b79f00b26502000000000000032000c2
:104f7c0022cf80000091b900800220000200400086
:104f8c0000804500b26502000000000050a028001f
:104f9c00b265020000000000efb09700afb29700be
:104fac00818f5200e8fe3a000cc480008041eb0077
:104fbc0083747e00810f560039f73a00f6fe3700f5
:104fcc000103200022cf80000191b900fc004100b8
:104fdc00eb8078000100010030912800d2650200be
:104fec000000000010c4800052fa37000140780025
:104ffc00e1b79f00d46a0200000000000cc48000de
:10500c00efb0970081747e000c06e800fc07b2003c
:10501c000cc488000042eb0084747e0020f737003b
:10502c000c01e900e20f51002afb3e0030912800f0
:10503c00d2650200000000007cc6880010c480000d
:10504c003cfa37000c06e900e20f560021fb3e004b
:10505c000000e800f007b20010c488007860b900c6
:10506c008000e9008a804000010178000000eb001c
:10507c000069eb000000e800f80f5000fcff3a005c
:10508c0010c4800069417800e3c3b300834f510022
:10509c0076f83200826878000000e800f007b20071
:1050ac00f8ff37005752490054452000424954003c
:1050bc003a2020002a6e650078742000636c6f0023
:1050cc00636b2000285e2900207769006c6c20003f
:1050dc0075736500207468006973200076616c003c
:1050ec0075654e006f2064006576690063652c0061
:1050fc002074720079202800414c4100524d290047
:10510c00205345004152430048206d0061637200fa
:10511c006f2066006972730074414400445245006c
:10512c00535320004d414300524f200020302e009d
:10513c004d616300726f20006d656e00754d6100ee
:10514c0063726f002020200020203100574952004c
:10515c004520610064647200657373000d0a2000c1
:10516c0020202a003157490052452000524f4d0053
:10517c0020434f004d4d41004e4420004d41430013
:10518c00524f73003a0d0a00203531002e52450063
:10519c0041442000524f4d0020283000783333001a
:1051ac0029202a00666f7200207369006e676c00fc
:1051bc006520640065766900636520006275730084
:1051cc000d0a200038352e004d4154004348200074
:1051dc00524f4d00202830007835350029202a0008
:1051ec00666f6c006c6f770065642000627920003c
:1051fc003634620069742000616464007265730067
:10520c00730d0a0020323000342e53004b495000ed
:10521c0020524f004d2028003078430043292000b5
:10522c002a666f006c6c6f007765640020627900f1
:10523c0020636f006d6d61006e640d000a203200fa
:10524c0033362e00414c4100524d20005345410055
:10525c00524348002028300078454300290d0a00ad
:10526c0020323400302e5300454152004348200078
:10527c00524f4d00202830007846300029414c0018
:10528c0041524d0020534500415243004820280014
:10529c0030784500432953004541520043482000d3
:1052ac002830780046302900446576006963650033
:1052bc002049440073206100726520006176610012
:1052cc00696c6100626c650020627900204d4100c0
:1052dc0043524f002c2073006565200028302900b4
:1052ec002e52450041442000524f4d0020283000e2
:1052fc0078333300293a20004d41540043482000b4
:10530c00524f4d00202830007835350029534b0082
:10531c0049502000524f4d00202830007843430064
:10532c0029556e006b6e6f00776e20006d61630007
:10533c00726f2c002074720079203f00206f720075
:10534c0020283000292066006f72200068656c00f0
:10535c0070425500532052004553450054205700cd
:10536c0061726e00696e67003a202a0053686f0004
:10537c00727420006f7220006e6f200070756c00cc
:10538c006c2d750070202a004e6f2000646576002d
:10539c00696365002064650074656300746564006e
:1053ac0020445300313853003230200048696700e4
:1053bc006820500072657300204469006720540017
:1053cc00686572006d445300313842003230200061
:1053dc0050726f00672052006573200044696700ab
:1053ec002054680065726d0044533100383232002d
:1053fc00204563006f6e20004469670020546800ec
:10540c0065726d0044533200343034002045630023
:10541c006f6e7200616d200074696d006520430031
:10542c0068697000445332003433310020314b0032
:10543c002045450050524f004d556e006b6e6f006d
:10544c00776e2000646576006963650050574d00e7
:10545c0020646900736162006c656400314b480024
:10546c007a2d34002c303000304b48007a2050001c
:10547c00574d46007265710075656e0063792000aa
:10548c00696e20004b487a002050720065736300ef
:10549c00616c65003a505200323a440075747900e0
:1054ac0020637900636c650020696e002025200064
:1054bc0050574d00206163007469760065455200b9
:1054cc00524f52003a205000574d20006163740037
:1054dc00697665002c20670020746f0020646900d9
:1054ec00736162006c65410055582000467265007e
:1054fc00717565006e6379003a20410055582000a3
:10550c00494e500055542f0048492d005a41550022
:10551c00582048004947480041555800204c4f003e
:10552c0057564f004c544d004554450052204d00e9
:10553c004f444500564f4c00544147004520500005
:10554c00524f4200453a200056457200726f72006d
:10555c0028292000406c69006e653a0020407000dc
:10556c00676d730070616300653a200062797400a6
:10557c0065732e00546f6f00206c6f006e672100f6
:10558c0053796e007461780020657200726f72003e
:10559c004e6f200045455000524f4d004572610042
:1055ac0073696e0067646f006e6553006176690005
:1055bc006e672000746f2000736c6f0074204900bc
:1055cc006e7661006c69640020736c006f744c0023
:1055dc006f616400696e6700206672006f6d200059
:1055ec00736c6f007420450052524f00523a2000e9
:1055fc00636f6d006d616e00642068006173200044
:10560c006e6f200065666600656374002068650037
:10561c0072654100434b4e0041434b0049324300fd
:10562c002053540041525400204249005449320046
:10563c0043205300544f500020424900544932003b
:10564c0043206d006f6465003a0d0a0020312e0076
:10565c0020536f0066747700617265000d0a20009c
:10566c00322e20004861720064776100726553002d
:10567c00657420007370650065643a000d0a2000a3
:10568c00312e20007e354b00487a0d000a20320066
:10569c002e207e0035304b00487a0d000a20330056
:1056ac002e207e00313030004b487a000d0a20004d
:1056bc00342e20007e343000304b48007a574100a5
:1056cc00524e49004e473a00204841005244570080
:1056dc00415245002049320043206900732062008a
:1056ec00726f6b00656e20006f6e2000746869002d
:1056fc0073205000494321002028520045562000b9
:10570c004133290053657400207370006565640093
:10571c003a0d0a0020312e0020313000304b480069
:10572c007a0d0a0020322e0020343000304b480015
:10573c007a0d0a0020332e0020314d00487a4900a2
:10574c0032432000286d6f006420730070642900c0
:10575c003d28200020302e004d616300726f200028
:10576c006d656e00750d0a0020312e0037626900e0
:10577c0074206100646472006573730020736500ab
:10578c0061726300680d0a0020322e00493243001a
:10579c0020736e0069666600657253006561720065
:1057ac00636869006e672000493243002061640021
:1057bc0064726500737320007370610063652e0062
:1057cc0020466f00756e6400206465007669630086
:1057dc006573200061743a00536e6900666665005b
:1057ec00722842004153490043295200656164000c
:1057fc0079612f00412f400020636f006e7472009e
:10580c006f6c73002041550058207000696e610068
:10581c002f412f00402063006f6e7400726f6c007c
:10582c007320430053207000696e43006f6d6d0050
:10583c00616e6400206e6f007420750073656400e7
:10584c0020696e0020746800697320006d6f64001d
:10585c00655075006c6c2d007570200072657300be
:10586c00697374006f727300204f460046507500c8
:10587c006c6c2d0075702000726573006973740078
:10588c006f727300204f4e0053656c00662d7400d0
:10589c006573740020696e00204869005a206d0001
:1058ac006f646500206f6e006c79520045534500a3
:1058bc0054424f004f544c004f414400455241005c
:1058cc0055582000494e500055542f0048492d0082
:1058dc005a2c200052454100443a2000504f5700aa
:1058ec004552200053555000504c49004553200060
:1058fc004f4e50004f57450052205300555050000a
:10590c004c49450053204f00464644004154410049
:10591c0020535400415445003a204400454c41006a
:10592c005920750073575200495445003a205200d3
:10593c00454144003a2043004c4f43004b2c20007f
:10594c0031434c004f434b002c2030004441540059
:10595c0041204f005554500055542c002031440028
:10596c0041544100204f550054505500542c2000f8
:10597c0030202a0070696e0020697300206e6f0061
:10598c0077204800695a43004c4f43004b20540089
:10599c0049434b00533a20005245410044204200f9
:1059ac0049543a00205379006e74610078206500e8
:1059bc0072726f0072206100742063006861720063
:1059cc0020782e00206578006974280077697400af
:1059dc00686f75007420630068616e00676529004c
:1059ec006e6f20006d6f64006520630068616e004f
:1059fc00676523003a204e006f2073006f667400b9
:105a0c0077617200652072006573650074206f0009
:105a1c006e207600342c20007573650020746800ad
:105a2c0065207200657365007420620075747400e3
:105a3c006f6e2e004e6f6e00657869007374650092
:105a4c006e74200070726f00746f63006f6c2100b5
:105a5c00782e200065786900740d0a00496e760076
:105a6c00616c690064206300686f690063652c00d9
:105a7c002074720079206100676169006e444500f2
:105a8c00564944003a68740074703a002f2f640031
:105a9c00616e670065726f0075737000726f7400d1
:105aac006f747900706573002e636f006d2a2d0082
:105abc002d2d2d002d2d2d002d2d2d002a4f70005c
:105acc00656e200064726100696e20006f75740051
:105adc007075740073202800483d4800692d5a00e9
:105aec002c204c003d474e0044294e006f726d0037
:105afc00616c20006f757400707574007320280041
:105b0c00483d33002e3376002c204c003d474e0090
:105b1c0044294d0053422000736574003a204d0017
:105b2c004f53540020736900672062006974200091
:105b3c006669720073744c005342200073657400e4
:105b4c003a204c00454153005420730069672000f3
:105b5c0062697400206669007273740020426f00e1
:105b6c006f746c006f6164006572200076203100e8
:105b7c002e20480045580d000a2032002e204400eb
:105b8c0045430d000a2033002e204200494e0d00e3
:105b9c000a2034002e2052004157440069737000d3
:105bac006c61790020666f00726d61007420730067
:105bbc00657456006f6c740061676500206d6f0032
:105bcc006e6974006f7273003a203500563a2000eb
:105bdc00207c2000332e3300563a2000207c2000fd
:105bec00565055004c4c5500503a200053657400eb
:105bfc0020736500726961006c2070006f72740014
:105c0c0020737000656564003a2028006270730090
:105c1c00290d0a0020312e0020333000300d0a00ef
:105c2c0020322e002031320030300d000a2033009b
:105c3c002e203200343030000d0a2000342e20008b
:105c4c0034383000300d0a0020352e002039360053
:105c5c0030300d000a2036002e2031003932300051
:105c6c00300d0a0020372e0020333800343030003d
:105c7c000d0a2000382e20003537360030300d004c
:105c8c000a2039002e2031003135320030300d0021
:105c9c000a3130002e2042005247200072617700fa
:105cac00207661006c75650041646a007573740040
:105cbc0020796f0075722000746572006d696e003a
:105ccc00616c410072652000796f7500207375005e
:105cdc0072653f002043460047313a00204346009e
:105cec0047323a00285c2d002f5f5c002d292800dc
:105cfc005c5f2f002d295300656c650063742000d8
:105d0c006f757400707574002074790070653a00ba
:105d1c000d0a2000312e20004f7065006e206400ab
:105d2c00726169006e202800483d4800692d5a00b8
:105d3c002c204c003d474e0044290d000a20320017
:105d4c002e204e006f726d00616c200028483d00c3
:105d5c00332e3300562c20004c3d47004e44290076
:105d6c0052325700202873007064200068697a0052
:105d7c00293d2800202030002e4d610063726f00f9
:105d8c00206d65006e750d000a2031002e49530000
:105d9c004f37380031362d003320410054520d005e
:105dac000a2032002e4953004f37380031362d006f
:105dbc00332070006172730065206f006e6c790087
:105dcc0049534f002037380031362d003320410025
:105ddc00545220002852450053455400206f6e0049
:105dec0020435300290d0a0052455300455420000e
:105dfc0048494700482c2000434c4f00434b20009f
:105e0c00544943004b2c200052455300455420006c
:105e1c004c4f570049534f002037380031362d0076
:105e2c003320720065706c00792028007573650052
:105e3c007320630075727200656e7400204c530001
:105e4c004220730065747400696e6700293a200063
:105e5c0050726f00746f63006f6c3a0020736500b2
:105e6c00726961006c332000776972006532200022
:105e7c00776972006552460055756e006b6e6f0047
:105e8c00776e5200656164002074790070653a0089
:105e9c0020746f0020656e00647661007269610089
:105eac00626c6500206c65006e677400684461006c
:105ebc0074612000756e690074733a00206e6f0077
:105ecc0020696e0064696300617469006f6e440040
:105edc006174610020756e00697420006c656e0041
:105eec00677468002028620069747300293a2000e6
:105efc0043532000454e4100424c4500444353005f
:105f0c0020444900534142004c4544005233570051
:105f1c00202873007064200063736c002068690093
:105f2c007a293d00282029000d0a4400697363007a
:105f3c006f6e6e006563740020616e0079206400e2
:105f4c0065766900636573000d0a43006f6e6e0021
:105f5c00656374002028560070752000746f200053
:105f6c002b355600292061006e6420002841440026
:105f7c00432074006f202b00332e3300562943002e
:105f8c0074726c00415558004d4f440045204c0034
:105f9c0045445000554c4c0055502000485055007d
:105fac004c4c550050204c00565245004741440083
:105fbc00432061006e64200073757000706c790072
:105fcc0035565600505533002e335600414443008d
:105fdc004275730020686900676842007573200081
:105fec0048692d005a203000427573002048690022
:105ffc002d5a2000314d4f0044452000616e640045
:10600c0020565200454720004c4544007320730035
:10601c00686f75006c642000626520006f6e210053
:10602c00466f75006e64200020657200726f7200fe
:10603c00732e4d004f534900434c4b004d495300b8
:10604c004f435300204f4b0020464100494c530016
:10605c00657420007370650065643a000d0a2000b9
:10606c00312e200033304b00487a0d000a203200cc
:10607c002e20310032354b00487a0d000a203300b7
:10608c002e20320035304b00487a0d000a203400a7
:10609c002e2031004d487a00436c6f00636b20005a
:1060ac00706f6c006172690074793a000d0a2000ff
:1060bc00312e200049646c0065206c006f77200045
:1060cc002a646500666175006c740d000a2032004c
:1060dc002e204900646c65002068690067684f00d9
:1060ec007574700075742000636c6f00636b200016
:1060fc0065646700653a0d000a2031002e204900c6
:10610c00646c650020746f00206163007469760014
:10611c00650d0a0020322e00204163007469760060
:10612c00652074006f206900646c6500202a64008f
:10613c0065666100756c7400496e700075742000a2
:10614c0073616d00706c6500207068006173650090
:10615c003a0d0a0020312e00204d690064646c0059
:10616c0065202a006465660061756c00740d0a0078
:10617c0020322e0020456e00645350004920280028
:10618c007370640020636b00702073006b652000db
:10619c00736d7000206373006c206800697a2900ad
:1061ac003d28200020302e004d616300726f2000ce
:1061bc006d656e00750d0a0020312e00536e69005e
:1061cc0066662000435320006c6f77000d0a200098
:1061dc00322e53006e696600662061006c6c2000e4
:1061ec007472610066666900632d7000202d660074
:1061fc00202a42007974650073206400726f70006d
:10620c00706564002a464100494c4500442c20002e
:10621c004e4f200044415400414461007461200001
:10622c0062697400732061006e64200070617200fa
:10623c00697479003a0d0a0020312e0020382c00a8
:10624c00204e4f004e4520002a64650066617500a3
:10625c006c7420000d0a2000322e2000382c2000f7
:10626c00455645004e200d000a2033002e203800e4
:10627c002c204f00444420000d0a2000342e200016
:10628c00392c20004e4f4e00455374006f70200087
:10629c0062697400733a0d000a2031002e2031001f
:1062ac00202a640065666100756c74000d0a20007c
:1062bc00322e20003252650063656900766520003d
:1062cc00706f6c006172690074793a000d0a2000dd
:1062dc00312e200049646c0065203100202a6400b6
:1062ec0065666100756c74000d0a2000322e20006a
:1062fc0049646c0065203000554152005420280040
:10630c007370640020627200672064006270200069
:10631c007362200072787000206869007a293d0051
:10632c0028202000302e4d00616372006f206d001c
:10633c00656e75000d0a2000312e540072616e00de
:10634c007370610072656e00742062007269640083
:10635c0067650d000a2032002e4c6900766520001e
:10636c006d6f6e0069746f00720d0a0020332e0081
:10637c0042726900646765002077690074682000c8
:10638c00666c6f00772063006f6e7400726f6c0028
:10639c000a0d2000342e410075746f0020426100fc
:1063ac00756420004465740065637400696f6e0049
:1063bc0055415200542062007269640067655200b6
:1063cc0065736500742074006f2065007869740033
:1063dc00526177002055410052542000696e7000c4
:1063ec007574550041525400204c4900564520000c
:1063fc0044495300504c4100592c20007d2054003e
:10640c004f205300544f50004c4956004520440037
:10641c00495350004c415900205354004f505000e8
:10642c004544570041524e00494e47003a207000f7
:10643c00696e7300206e6f0074206f0070656e00c3
:10644c002064720061696e0020284800695a290096
:10645c0020524500564944003a0d0a00496e760018
:10646c00616c690064206300686f690063652c00cf
:10647c002074720079206100676169006e6d730091
:10648c00525320004c4f57002c2043004f4d4d00d1
:10649c00414e4400204d4f004445520053204800cb
:1064ac00494748002c20440041544100204d4f00e6
:1064bc00444541006464720065737300206f66008c
:1064cc00205043004638350037343f00546869008b
:1064dc0073206d006f646500207265007175690032
:1064ec007265730020616e0020616400617074003d
:1064fc0065724c004344200074797000653a0d00bd
:10650c000a2031002e204800443434003738300043
:10651c002028750073696e006720500043463800d0
:10652c003537340020494f002065780070616e00cb
:10653c0064657200294c4300442028007479700073
:10654c002061640064722900203d20002820200076
:10655c00302e4d00616372006f206d00656e75000a
:10656c000d0a2000312e4c0043442000526573006c
:10657c0065740d000a2032002e496e0069742000eb
:10658c004c4344000d0a2000332e43006c6561001f
:10659c0072204c0043440d000a2034002e43750039
:1065ac0072736f00722070006f73690074696f00f2
:1065bc006e206500783a280034292000300d0a003e
:1065cc0020362e00577269007465200074657300c4
:1065dc0074206e00756d6200657273002065780022
:1065ec003a28360029203800300d0a0020372e00ba
:1065fc005772690074652000746573007420630021
:10660c0068617200616374006572730020657800c4
:10661c003a283700292038003044690073706c0028
:10662c00617920006c696e0065733a000d0a2000d8
:10663c00312e200031200d000a2032002e204d007a
:10664c00756c740069706c0065494e0049544300c8
:10665c004c4541005243550052534f0052205300b9
:10666c0045544e006f204100434b2c0020636800c2
:10667c0065636b0020616400617074006572430097
:10668c004c4b09004d4f53004909430053094d0031
:10669c0049534f0050696e00737461007465730048
:1066ac003a474e00440933002e33560009352e006c
:1066bc003056090041444300095650005509410029
:1066cc005558090050095000095009004909490062
:1066dc00092d09004f574400092d09002d2d0900e3
:1066ec0054784400092d09005278440053434c005f
:1066fc000953440041092d00092d5000474309005e
:10670c0050474400092d09002d312e00284252001b
:10671c00290932002e28520044290900332e280062
:10672c004f52290009342e002859570029093500e9
:10673c002e2847004e290900362e2800424c2900ed
:10674c0009372e0028505500290938002e284700fb
:10675c0052290900392e28005754290009302e00df
:10676c0028426c006b2947004e440900474e4400f8
:10677c0009414400430935002e30560009332e00e0
:10678c00335609005650550009415500580965000b
:10679c007865630075746500203a200020617500ef
:1067ac00746f7200616e670065202b004d487a0093
:1067bc00292b6b00487a2900526177002076610002
:1067cc006c75650020666f007220420052472000f5
:1067dc00284d490044493d003132370029574100ca
:1067ec00524e49004e473a0020506f0073736900b7
:1067fc00626c65002062750066666500726f7600db
:10680c00657266006c6f7700416e7900206b6500d5
:10681c00792074006f2065007869740053706100f2
:10682c0063652000746f2000636f6e0074696e00e6
:10683c0075654e00756d6200657220006f662000f4
:10684c006269740073207200656164002f777200b6
:10685c00697465003a204300533a0d000a20310058
:10686c002e204300530d0a0020322e00202f43000f
:10687c0053202a006465660061756c0074506f00cb
:10688c0073697400696f6e0020696e002064650086
:10689c006772650065735300657276006f20610046
:1068ac00637469007665570061697400696e6700ee
:1068bc002061630074697600697479002e2e2e00b5
:1068cc002a2a2000456172006c7920004578690005
:1068dc0074212a002a42610075643e0031366d0035
:1068ec003a20420050204300616e6e006f7420000d
:1068fc006d6561007375720065203e0020313600b5
:10690c0030303000303030002c2044006f6e650089
:10691c002e0a0d0043616c0063756c006174650098
:10692c00643a2000090a0d0045737400696d61001a
:10693c00746564003a202000092062007073200006
:10694c0047656e00657261006c0909000909090050
:10695c0050726f00746f63006f6c2000696e74006e
:10696c0065726100637469006f6e20002d2d2d001f
:10697c002d2d2d002d2d2d002d2d2d002d2d2d00ef
:10698c002d2d2d002d2d2d002d2d2d002d2d2d00df
:10699c002d2d2d002d2d2d002d2d2d002d2d2d00cf
:1069ac002d2d2d002d2d2d002d2d2d002d2d2d00bf
:1069bc002d2d2d002d2d2d002d2d2d002d2d2d00af
:1069cc002d2d2d002d2d2d002d2d2d002d2d2d009f
:1069dc00203f09005468690073206800656c7000e2
:1069ec000909090028302900094c6900737420003a
:1069fc006375720072656e0074206d0061637200c5
:106a0c006f7320003d582f007c580900436f6e00b7
:106a1c007665720074732000582f720065766500dd
:106a2c0072736500205809000928780029094d0067
:106a3c00616372006f207800207e090053656c0042
:106a4c00667465007374090009095b0009537400ce
:106a5c006172740020230900526573006574200074
:106a6c0074686500204250002020200009090900ac
:106a7c005d095300746f7000202409004a756d0085
:106a8c00702074006f2062006f6f74006c6f610077
:106a9c006465720009097b0009537400617274000b
:106aac0020776900746820007265610064202600fc
:106abc002f25090044656c00617920003120750098
:106acc00732f6d0073090900097d090053746f0061
:106adc00702061002f412f00400941005558500093
:106aec00494e2000286c6f00772f4800492f520028
:106afc004541440029090900226162006322090012
:106b0c0053656e0064207300747269006e67200018
:106b1c006209530065742000626175006472610043
:106b2c00746509000909310032332000632f4300da
:106b3c00094155005820610073736900676e6d0040
:106b4c00656e74002028610075782f00435329006e
:106b5c000909300078313200332064002f440900d9
:106b6c004d6561007375720065204100444320003f
:106b7c00286f6e0063652f00434f4e00542e290082
:106b8c000930620031313000095365006e64200019
:106b9c0076616c007565200066094d0065617300b7
:106bac00757265002066720065717500656e630014
:106bbc0079090900720952006561640020672f0091
:106bcc0053094700656e65007261740065205000c2
:106bdc00574d2f0053657200766f0900092f09007d
:106bec00434c4b002068690020680900436f6d001e
:106bfc006d616e006468690073746f0072790900ce
:106c0c0009095c0009434c004b206c006f206900a3
:106c1c0009566500727369006f6e69006e666f00cd
:106c2c002f7374006174750073696e00666f0900d0
:106c3c00095e0900434c4b0020746900636b200013
:106c4c006c2f4c0009426900746f7200646572000d
:106c5c0020286d0073622f004c5342002909090053
:106c6c002d09440041542000686920006d0943003f
:106c7c0068616e00676520006d6f6400650909002e
:106c8c00095f090044415400206c6f00206f09001b
:106c9c0053657400206f7500747075007420740057
:106cac0079706500090909002e094400415420003f
:106cbc0072656100642070002f50090050756c00e3
:106ccc006c7570002072650073697300746f7200cc
:106cdc00732028006f6666002f4f4e002909210093
:106cec000942690074207200656164002073090018
:106cfc00536372006970740020656e0067696e00e2
:106d0c0065090900093a0900526570006561740053
:106d1c0020652e00672e2000723a3100302076005c
:106d2c00095368006f772000766f6c0074732f0026
:106d3c00737461007465730009092e0009426900bf
:106d4c0074732000746f200072656100642f7700eb
:106d5c0072697400652065002e672e002030780063
:106d6c0035352e00322077002f570900505355002f
:106d7c0020286f0066662f004f4e290009093c0041
:106d8c00783e2f003c783d00203e2f003c303e00ea
:106d9c000955730065726d00616372006f20780095
:106dac002f617300736967006e2078002f6c690087
:106dbc0073742000616c6c00809c21001064a00036
:106dcc0020a22100104078006840600008003200ca
:106ddc00cac2a900f0c2b300d46a020000000000cd
:106dec00a100200090ab20006e7c0400000000008d
:106dfc00cac2a800a100200090ab20006e7c040049
:106e0c0000000000faff3700809c21001064a100f4
:106e1c0020a2210010407800684060000800320079
:106e2c00cac2a900f0c2b300d46a0200000000007c
:106e3c00a100200090ab20006e7c0400000000003c
:106e4c00cac2a800a100200090ab20006e7c0400f8
:106e5c0000000000faff370020a22100104078004b
:106e6c006840600008003200cac2a800f0c2b3003b
:106e7c00d46a020000000000b100200030ac2000f9
:106e8c006e7c040000000000cac2a900b100200002
:106e9c0030ac20006e7c040000000000faff3700cc
:106eac00f00f2000401288000140200022048000d6
:106ebc0002806000fdff3200401280008540a90076
:106ecc000080fb00000006000080fb0040128800e0
:106edc00014020002204800002806000fdff32008f
:106eec00421280008540a900809c210003c4b3009d
:106efc0090c061000000eb00010032000280fb003a
:106f0c0000000600881f78000102200000ca200043
:106f1c00167c020000000000609b21001040e8007d
:106f2c00946802000000000000c2b300d46a0200a2
:106f3c000000000028a221009840780061c0600089
:106f4c00946802000000000000c2b300d46a020082
:106f5c00000000001800d10061406000946802003d
:106f6c000000000000c2b300d46a02000000000060
:106f7c00180078004200de00614060009468020056
:106f8c000000000000c2b300d46a02000000000040
:106f9c00180078004300de00614060009468020035
:106fac000000000000c2b300d46a02000000000020
:106fbc00809c21001080fb004400de0061406000da
:106fcc00946802000000000000c2b300d46a020002
:106fdc00000000003100200020ae2000167c0200d2
:106fec00000000004f04780000000600889fbe00df
:106ffc008a9fbe008c1f7800600d0200000000000c
:10700c00b60b02000000000080047800600d020046
:10701c0000000000b60b0200000000000006780023
:10702c00600d020000000000b60b02000000000022
:10703c0080057800600d020000000000b60b020015
:10704c000000000000057800600d02000000000048
:10705c00b60b02000000000000047800600d020076
:10706c0000000000b60b0200000000008900e900df
:10707c00e38f50007b003e00619b21008948e900b2
:10708c008c00e900e18f50007a0036008004eb00a0
:10709c008b00e900e18f50007f0036008004eb008c
:1070ac008a00e900e18f5000850036008004eb0077
:1070bc008800e900e18f50008c0036008004eb0062
:1070cc008000e900889c2100e18f5000930036007d
:1070dc00408821000048eb007103200000bc200018
:1070ec006e7c0200000000008001eb0042002000da
:1070fc0011002000100020007a0d0200000000009a
:10710c00619b21008048e9005103200070bf2000e2
:10711c006e7c0200000000008001eb0022002000c9
:10712c0011002000100020007a0d02000000000069
:10713c0029a221000040e9006140600099407800dc
:10714c000104a10080cc700031042000c0c22000da
:10715c006e7c0200000000008001eb002200200089
:10716c0011002000200020007a0d02000000000019
:10717c000040e90061406000004040009940780008
:10718c000114a10080cc700011032000f0c6200077
:10719c006e7c0200000000008001eb002200200049
:1071ac0011002000100020007a0d020000000000e9
:1071bc000040e900614060002a0020000a00dd0068
:1071cc00994078000124a10080cc7000d1012000ee
:1071dc00601c21006e7c0200000000008001eb00ae
:1071ec000a017800110020000a0078007a0d0200d4
:1071fc00000000000040e900614060003100200008
:10720c000100dd00994078000134a10080cc7000b1
:10721c00f1042000e09320006e7c020000000000ce
:10722c008001eb000a017800110020001000200002
:10723c007a0d020000000000614060004100200057
:10724c000100dd00984078000144a10000cc7000e2
:10725c001864a1004f0678004f05be004f04be0015
:10726c00000006008004eb008c00e900e18f500068
:10727c0086ff3e0021a221000c46e9006146660013
:10728c00114178000204a1008c4871008b00e900c8
:10729c00e18f500081ff3e0021a221008b45e900c7
:1072ac00e1c565008bc54500114178000214a100b1
:1072bc008b4871008a00e900e18f50007bff3e0093
:1072cc0021a221000a45e900614565002200200049
:1072dc000255dd00114178000224a1008a4871009a
:1072ec008800e900e18f500074ff3e0021a22100cc
:1072fc000844e90061446400320020000244dd00cf
:10730c00114178000234a100884871008000e90026
:10731c00889c2100e18f50006dff3e0061406000b1
:10732c00410020000100dd00984078000144a100dc
:10733c0000cc70000900e00065ff3200f1fe070090
:10734c001864a1004f0678004f05be004f04be0024
:10735c0000000600c3ff370041e2a9004035800061
:10736c00f001b30040358800f00f2e00c826b6009f
:10737c0000fe2f00c826b600cf22a900cf02a9001c
:10738c00cec2a90000000600010120004006210029
:10739c006e7c04000000000041e2a900819c2100e9
:1073ac0091407800f0c0600031003a00cf22a90073
:1073bc00cf02a900cec2a90001fe2f0043358000e8
:1073cc00038160007200b30042358800f30f2e0079
:1073dc00423680008281610002702000030171003e
:1073ec004236880043368000838060000130a00064
:1073fc0041368800cac2a800c8c2a900c902a900a7
:10740c00c8e2a800c922a9000080fb001012880065
:10741c0042a2a80010d18000610160004611dd007d
:10742c00111280000160a10081007100111288000e
:10743c00c700dd000110b200121280000280a10012
:10744c0002817000121288004700dd000020b2009b
:10745c00111280000190a1008100700011128800af
:10746c004422ef004022ef0041e2a8000000060099
:10747c00cf22a800cf02a800cec2a80001fe2f0088
:10748c0043358000038160007200b30042358800f0
:10749c00f30f2e00423680008281610002702000c2
:1074ac0003017100423688004336800083806000ff
:1074bc000130a00041368800cac2a800c8c2a90089
:1074cc00c902a900c8e2a800c922a9000080fb00db
:1074dc001012880042a2a80010d180006101600047
:1074ec004611dd00111280000160a10081007100c5
:1074fc0011128800c700dd000110b20012128000ca
:10750c000280a10002817000121288004700dd0089
:10751c000020b200111280000190a10081007000c7
:10752c00111288004422ef004022ef0041e2a80033
:10753c0000000600ceff3700609b21001080fb008e
:10754c0051b628006140780093ff070010d18000ed
:10755c004300dd000004b200f1fb2f005216800046
:10756c0082806000810070005116880000000600c7
:10757c0041e2a90040358000f001b300403588009d
:10758c00f00f2e00c826b60000fe2f00c826b6004d
:10759c00cf22a900cf02a900cec2a900000006008c
:1075ac000080fb0040128800014020002204800073
:1075bc0002806000fdff3200401280008540a9006f
:1075cc0000000600c8c2a800c902a800c8e2a800b2
:1075dc00c922a80000fe2f005235800082006000f6
:1075ec006100b30051358800743580008400600060
:1075fc006100b3007135880045358000850060005e
:10760c009100b30041358800f20f2e004635800002
:10761c008601610001802000838170004335880061
:10762c00ac06b6007000b300603588006035800091
:10763c00000161000281700062358800609b2100ae
:10764c001080fb0051b62800614278000482fb00d8
:10765c001412880010d18000610160004611dd0019
:10766c00f3fb2f00151280008580610081007100f2
:10767c00111288004700dd000010b200f1ef2f005e
:10768c001612800086826000850270001512880038
:10769c004422ef004022ef001413880014138000e2
:1076ac00848161008301710013138800151380001d
:1076bc008580600081007000111388006422ef0047
:1076cc006022ef004822ef006822ef004322a9005d
:1076dc006322a9004362a80042a2a9006362a80029
:1076ec0062a2a90040c2a90060c2a9004402a8007d
:1076fc006402a80000000600889fbe008a9fbe009e
:10770c008c9fbe008e1f78000044780001467800e4
:10771c00ab9e21000efe2f000a2020001a6a0200e8
:10772c000000000041e2a90040358000f001b300e8
:10773c0040358800f00f2e00c826b600806c200063
:10774c0010086700cf22a900cf02a900cec2a90061
:10775c009cff07000804e00031003a0042e2a80058
:10776c0062e2a80041e2a80061e2a80019c0b300df
:10777c0040a2ab0015003a0060a2ab0013003a0027
:10778c004d128000e1cf5400890032000c04e0005f
:10779c004c0032000d80fb00a66a020000000000c5
:1077ac004913800080c2b3007e6a02000000000012
:1077bc000980fb00a66a02000000000090c2b30022
:1077cc007e6a0200000000008044eb0040c2ab0067
:1077dc0048003a0060c2ab0046003a001b0065004e
:1077ec0046003a00286a020000000000146a0200f9
:1077fc0000000000e14f50000d0032000904e000d1
:10780c00daff3a00cac2ab00d9ff3200d0c5b300d0
:10781c007e6a02000000000019c0b300d4ff3700dc
:10782c00e14f5400cfff360019c0b300d0ff370032
:10783c00c66a0200000000000c04e00037003a00a9
:10784c0041e2a9004362a90061e2a9006362a900b8
:10785c0050358000f001b300503588007035800041
:10786c00f001b3007035880040358000f001b300a2
:10787c00403588004035800001f021000080700008
:10788c004035880060358000f001b3006035880019
:10789c00603580000080700060358800609b21009e
:1078ac001080fb0051b6280061407800bafe07003a
:1078bc004f0778004f06be004f05be004f04be00b8
:1078cc0000000600c0c5b3007e6a02000000000084
:1078dc000d4078007e6a020000000000401380001a
:1078ec007e6a0200000000008044eb0040c2ab0046
:1078fc00b8ff32001b006500310032004022ef005f
:10790c006022ef000c04e0003000320060b428006c
:10791c00d26502000000000080ff370070b528001f
:10792c00d26502000000000041e2a9004362a900f8
:10793c0061e2a9006362a90050358000f001b30038
:10794c005035880070358000f001b3007035880028
:10795c0040358000f001b300403588004035800090
:10796c0001f02100008070004035880060358000f7
:10797c00f001b30060358800603580000080700035
:10798c0060358800609b21001080fb0051b62800f8
:10799c006140780080fe07004f0778004f06be005c
:1079ac004f05be004f04be0000000600c5ff3700a7
:1079bc00b0c5b3007e6a02000000000073ff370000
:1079cc00526a020000000000ccff3700c222a9005e
:1079dc0041e2a9004362a90061e2a9006362a90027
:1079ec0050358000f001b3005035880070358000b0
:1079fc00f001b3007035880040358000f001b30011
:107a0c00403588004035800001f021000080700076
:107a1c004035880060358000f001b3006035880087
:107a2c00603580000080700060358800609b21000c
:107a3c001080fb0051b628006140780056fe07000c
:107a4c004f0778004f06be004f05be004f04be0026
:107a5c00000006009bff37008000eb00ef0f50008a
:107a6c00e08f58000500360041022000e01d200088
:107a7c006e7c0200000000000000060000600100a7
:107a8c000f003700120037001c003700faff3700d8
:107a9c00f5ff3700f4ff3700f3ff3700f2ff370034
:107aac00f1ff3700f0ff37001f00370039003700b7
:107abc00530037006c003700850037009e003700fc
:107acc004103200000cc20006e7c0400000000006c
:107adc0071002000705620006e7c02000000000037
:107aec00f1002000b01821006e7c020000000000a4
:107afc0011c0b3000040eb00fffe37007100200006
:107b0c00705620006e7c020000000000f100200086
:107b1c00b01821006e7c02000000000011c0b30000
:107b2c0001407800f4fe370020a221001004a100cf
:107b3c0011d180000101d10061416100c208de0059
:107b4c00e1c060008041eb00e1816100c619dd00fd
:107b5c00101280000060a1000080710010128800db
:107b6c00610161004811dd00101280000080a1004d
:107b7c000000710010128800e1806000c908dd006f
:107b8c00101280000090a10000807000101288007c
:107b9c00dcfc370020a221001004a00011d18000d1
:107bac000101d10061416100c208de00e1c060004a
:107bbc0013c0b300e1816100c619dd001012800012
:107bcc000060a1000080710010128800610161004a
:107bdc004811dd00101280000080a100000071002f
:107bec0010128800e1806000c908dd0010128000ce
:107bfc000090a1000080700010128800c1fc3700ba
:107c0c0020a221001014a10011d18000e1c160005c
:107c1c00c208de00e1c060000041eb00e1816100c0
:107c2c00c619dd00101280000060a10000807100f8
:107c3c0010128800610161004811dd0010128000f3
:107c4c000080a1000000710010128800e18060002b
:107c5c00c908dd00101280000090a10000807000a7
:107c6c0010128800a7fc370020a221001014a000dd
:107c7c0011d18000e1c16000c208de00e1c06000eb
:107c8c0012c0b300e1816100c619dd001012800042
:107c9c000060a10000807100101288006101610079
:107cac004811dd00101280000080a100000071005e
:107cbc0010128800e1806000c908dd0010128000fd
:107ccc000090a10000807000101288008dfc37001d
:107cdc0020a221001024a10012d18000e1416100fa
:107cec000201d100614161008040eb00e181610043
:107cfc00c619dd00101280000060a1000080710028
:107d0c0010128800610161004811dd001012800022
:107d1c000080a1000000710010128800e18060005a
:107d2c00c908dd00101280000090a10000807000d6
:107d3c001012880073fc370020a221001024a00030
:107d4c0012d18000e14161000201d100614161006a
:107d5c0011c0b300e1816100c619dd001012800072
:107d6c000060a100008071001012880061016100a8
:107d7c004811dd00101280000080a100000071008d
:107d8c0010128800e1806000c908dd00101280002c
:107d9c000090a100008070001012880059fc370080
:107dac0041e2a9004362a90061e2a9006362a90053
:107dbc0050358000f001b3005035880070358000dc
:107dcc00f001b3007035880040358000f001b3003d
:107ddc00403588004035800001f0210000807000a3
:107dec004035880060358000f001b30060358800b4
:107dfc00603580000080700060358800000006004f
:107e0c0080b52800b265040000000000f28747002e
:107e1c00889fbe008a9fbe008c9fbe008e1f78007c
:107e2c006e9b210010c0b300004f78002ba22100e4
:107e3c001b4078000000a1000010a0000020a10051
:107e4c00804d7800f20647001d44a00080c1b300ad
:107e5c0051fd070080b52800b2650200000000004b
:107e6c0059a221004aa221000906780008402000ee
:107e7c00c66a020000000000804c78008081fb0084
:107e8c004419de00024d7800e44f5100110032001d
:107e9c00e44f510033003e000204e0005c0032006d
:107eac00e14f5100110032000040eb00d46a020097
:107ebc0000000000c66a020000000000804c780040
:107ecc008081fb004419de00024d7800e44f510024
:107edc00efff3a00388102000000000010c0b30030
:107eec00d46a020000000000e1ff37006f40600020
:107efc00004ee80002407800d46a02000000000046
:107f0c0033a221008049eb001c04e000d8ff3200b2
:107f1c00c66a0200000000000080fb0040128800ce
:107f2c002404800004006400fdff32004012800035
:107f3c008540a900d46a02000000000035a221008f
:107f4c001540e800804a7800994f1000c8ff3600b1
:107f5c00c66a0200000000000080fb00401288008e
:107f6c00efff3700e64f51001e003200e84f510082
:107f7c00cdff3a001b4078000000a1000010a100ca
:107f8c000020a100804d78001d44a1000328a3000f
:107f9c00030032000004a00021a2210080487800d8
:107fac000318a300010032001b14a0000308a30057
:107fbc00010032001b24a0000338a30001003a008a
:107fcc001d44a0001e80fb00d3b528006340780040
:107fdc00f1fc070010c0b300d46a020000000000de
:107fec00a3ff370067406000004e7800004f780018
:107ffc000080fb00d6b5280066407800e6fc070040
:10800c0010c0b300d46a02000000000098ff3700d3
:10801c00e54f500075003e00e44f50001c01390044
:10802c00c66a020000000000c800dd0081bf9f008e
:10803c00c66a0200000000000081fb008fb89700a8
:10804c0001017100e2b79f00c66a02000000000047
:10805c008040780081bf9f00c66a020000000000cb
:10806c006fb197008fb8970003002100830f510068
:10807c008dff3e00c808dd000080fb000100700091
:10808c00b0b79f00830f500087ff3e000200e00056
:10809c00120032008000eb00e39d2100a2b79f008c
:1080ac0093b79f009fb297001582400081bf9f003d
:1080bc00f4b79f00c66a0200000000007fb2970070
:1080cc00004a78008fb897008100e8002fb3970022
:1080dc00810f5300f3ff3e000601780040c0b3004f
:1080ec00994f10002c0132000200e0000c0032000d
:1080fc00f3ce80008000eb003380fb004012880040
:10810c002404800004006400fdff32004012800053
:10811c008540a9008100e800828f5000f6ff3a00ec
:10812c00100020009e7b020000000000bfb29700f0
:10813c000500e0000e0032008000eb00e39d210002
:10814c00f40f2000138140004412880026048000a4
:10815c0006006400fdff3200401280008540a9003b
:10816c00004978008100e800858f5000f5ff3a0047
:10817c0040c0b300994f10000501320010c0b3008d
:10818c00d46a020000000000bfb097000100e000bc
:10819c0037ff32008000eb00f0ce800060c078002a
:1081ac0081bf9f00d46a0200000000008fb89700c6
:1081bc008100e800bfb19700818f51002cff360081
:1081cc00f0ce800060c0780081bf9f00d46a0200ae
:1081dc00000000008fb897008100e800bfb1970045
:1081ec00818f5100ecff3e0021ff3700ed4f500016
:1081fc00d4003200ee4f5000cb003200e64f50005e
:10820c0029ff3a0010c0b300d46a0200000000003d
:10821c00c66a02000000000080407800014e780021
:10822c00e1cf5000ce0032006aff3900e2cf50009f
:10823c001dff3a006022b8008000eb0081bf9f0058
:10824c00f4b79f00c5b79f00c66a0200000000008b
:10825c00804c78007fb29700cfb297004829dd00a0
:10826c00c821de00830171004821dd000082fb0083
:10827c008002eb0002027200838272008fb89700ba
:10828c008100e800e48f5000ecff3a006011b80068
:10829c008000eb0081bf9f00e2b79f00d3b79f0027
:1082ac00f4b79f00c5b79f00c66a0200000000002b
:1082bc00804c78006fb19700dfb19700481bdd0050
:1082cc00c813de00870373004813dd000081fb0038
:1082dc008001eb0006017100878171008fb8970057
:1082ec008100e8007fb29700cfb29700e48f500076
:1082fc00e8ff3a00e10f4200e08f5a00eafe3e0030
:10830c00e10f4100e08f5900e7fe3e000200420001
:10831c0083804a00e10f4000e08f5800e2fe3e00ef
:10832c0010c0b300e2b79f00d3b79f00f4b79f0013
:10833c00c5b79f00d46a0200000000007fb297000e
:10834c006fb19700dfb19700e00f5100e08f59003b
:10835c00c7fe32000502200045128800260480006a
:10836c0006006400fdff3200401280008540a90029
:10837c00c822de0045128800210480000100640040
:10838c00fdff3200401280008540a9008480fb0074
:10839c00411288002604800006006400fdff3200b4
:1083ac00401280008540a9004822ef00260480007e
:1083bc0006006400fdff3200401280008540a900d9
:1083cc0081bf9f00e2b79f00d3b79f00f4b79f0017
:1083dc00c5b79f00d46a0200000000006fb197007f
:1083ec00dfb197008fb897007fb29700cfb297009c
:1083fc00e10f5100e08f59009dfe320080022000f9
:10840c00401288002604800006006400fdff320044
:10841c00401280008540a900451288002504800088
:10842c0005006400fdff3200401280008540a90069
:10843c00411288002604800006006400fdff320013
:10844c00401280008540a9004822ef0021048000e2
:10845c0001006400fdff3200401280008540a9003d
:10846c00e2b79f00d3b79f00f4b79f00d46a020015
:10847c00000000006fb19700dfb19700620151005e
:10848c00e08159007fb297000402e800aeff37008c
:10849c00e14f5000200032000e003900e24f500036
:1084ac0007003200e34f50007ffe3a00ccc2a80018
:1084bc0010c0b300d46a0200000000006cfe37004c
:1084cc00ccc2a90010c0b300d46a020000000000a6
:1084dc0067fe370041e2a90040358000f001b3008f
:1084ec0040358800f00f2e00c826b60000fe2f0085
:1084fc00c826b600cf22a900cf02a900cec2a9007f
:10850c004f0778004f06be004f05be004f04be005b
:10851c002f01b1000000060080b52800b2650200f2
:10852c000000000052fe370010c0b300d46a0200f5
:10853c00000000008040eb00014078006efc07005a
:10854c004bfe370010c0b300d46a020000000000dc
:10855c008040eb0010c0b30067fc070044fe3700fe
:10856c000140780081bf9f00d46a02000000000027
:10857c000040eb00d46a0200000000008fb89700a6
:10858c0001407800d46a02000000000038fe370079
:10859c00cac2a800f9fe3700cac2a900d2fe370031
:1085ac00881f780048800200000000000004e000f2
:1085bc00260032003262ab001d003a003242ab00a2
:1085cc0011003a0040800200000000000004780016
:1085dc003222ab0003003a00080078004f04780008
:1085ec0000000600f1002000a0cf2000167c020045
:1085fc00000000003222a900080078004f04780027
:10860c0000000600f7ff37003100200070cf20007b
:10861c00167c0200000000004080020000000000f8
:10862c00000478003222ab00ebff3200edff370084
:10863c003100200040cf2000167c0200000000001a
:10864c003242ab00dfff3200efff3700f1002000b9
:10865c0090d02000167c0200000000000000eb000f
:10866c004f04780000000600deff3700388002005f
:10867c000000000000000500881f780001022000a7
:10868c00f0db2000167c020000000000689b21003b
:10869c0018407800946802000000000000c2b3008b
:1086ac00d46a02000000000018407800e94f500026
:1086bc002f0032000080fb000000400081ad28003c
:1086cc0061007800e86602000000000000c2b30000
:1086dc00d46a02000000000010d0800063406000eb
:1086ec00946802000000000000c2b300d46a0200cb
:1086fc000000000010d080004200de0061406000ed
:10870c00946802000000000000c2b300d46a0200aa
:10871c000000000010d080004300de0061406000cb
:10872c00946802000000000000c2b300d46a02008a
:10873c0000000000809c21001080fb004400de0043
:10874c0061406000946802000000000000c2b300a9
:10875c00d46a0200000000003100200020ae20008e
:10876c00167c0200000000004f0478000000060098
:10877c00c0118000e86602000000000000c2b300d7
:10878c00d46a02000000000010d08000634060003a
:10879c00946802000000000000c2b300d46a02001a
:1087ac000000000010d080004200de00614060003c
:1087bc00946802000000000000c2b300d46a0200fa
:1087cc000000000010d080004300de00614060001b
:1087dc00946802000000000000c2b300d46a0200da
:1087ec0000000000809c21001080fb004400de0093
:1087fc0061406000946802000000000000c2b300f9
:10880c00d46a0200000000003100200020ae2000dd
:10881c00167c0200000000004f04780000000600e7
:10882c00d3ff37000200fa00889fbe008a9fbe006b
:10883c008c1f7800600d020000000000b60b0200d7
:10884c000000000000057800ea0f55000f0132000f
:10885c00600d020000000000b60b020000000000da
:10886c0080047800600d020000000000b60b0200ce
:10887c000000000000067800600d020000000000ff
:10888c00b60b02000000000080057800600d0200ad
:10889c0000000000b60b0200000000008a00e90096
:1088ac00e98f50009c0036000001eb000005eb0046
:1088bc00689b21008900e900e38f500069003e00ad
:1088cc0021a021008944e900e3c46400c3cfb300b4
:1088dc0091c1610089c871008c00e900e18f5000e2
:1088ec00640036000005eb008b00e900e18f5000be
:1088fc006b0036000005eb008000e900899c21002c
:10890c00e18f500072003600408821000048eb00d7
:10891c00d1082000608720006e7c0200000000005f
:10892c008001eb00a20020001100200010002000ac
:10893c007a0d0200000000000040e900004c7800b5
:10894c00e94f5000830032004105200080d1200007
:10895c00167c0200000000008001eb0042002000a9
:10896c0011002000100020007a0d02000000000011
:10897c0028a021000040e90063406000c1cfb30093
:10898c0098c0600000cc700011022000c0d62000fe
:10899c00167c0200000000008001eb002200200089
:1089ac0011002000100020007a0d020000000000d1
:1089bc000040e900614060002a0020000a00dd0050
:1089cc00984078000124a10000cc70002103200005
:1089dc00d0d82000167c0200000000008001eb00c3
:1089ec000a01780011002000100020007a0d02000e
:1089fc00000000000040e9006140600031002000f0
:108a0c000100dd00984078000134a10000cc70001a
:108a1c00f1042000e09320006e7c020000000000b6
:108a2c008001eb000a0178001100200010002000ea
:108a3c007a0d02000000000061406000410020003f
:108a4c000100dd00994078000144a10080cc700049
:108a5c004f0678004f05be004f04be000080fa00a0
:108a6c00000006000005eb008c00e900e18f5000cf
:108a7c009cff3e0021a021000c46e90061466600e7
:108a8c00230020000366dd00914178000324a1003f
:108a9c008cc871008b00e900e18f500095ff3e00ff
:108aac0021a021008b45e900e1c5650033002000c1
:108abc00835ddd00914178000334a1008bc8710007
:108acc008000e900899c2100e18f50008eff3e0060
:108adc0061406000410020000100dd0099407800f9
:108aec000144a10080cc70000a00e00086ff320037
:108afc0090c0b300984f10000b003200defe070050
:108b0c004f0678004f05be004f04be000080fa00ef
:108b1c0000000600d3ff37000001eb00689b21002a
:108b2c000a4ce90063ff3700cf91de000090200073
:108b3c00d103200086060200000000000001be00e8
:108b4c0061015100e0815900c2118800cafe070082
:108b5c00ebff3700c1012000f01421006e7c0200f5
:108b6c00000000008001eb00f2ff27001100200044
:108b7c00200220007a0d020000000000c0118800c5
:108b8c004105200080d12000167c0200000000006e
:108b9c008001eb004200200011002000100020009a
:108bac007a0d02000000000028a021000040e9001e
:108bbc0063406000c1cfb30098c0600000cc70006f
:108bcc0011022000c0d62000167c0200000000001c
:108bdc008001eb002200200011002000100020007a
:108bec007a0d0200000000000040e90061406000c6
:108bfc002a0020000a00dd00984078000124a10022
:108c0c0000cc700021032000d0d82000167c02007c
:108c1c00000000008001eb000a0178001100200028
:108c2c00100020007a0d0200000000000040e90056
:108c3c0061406000310020000100dd0098407800a8
:108c4c000134a10000cc7000f1042000e09320005e
:108c5c006e7c0200000000008001eb000a0178002d
:108c6c0011002000100020007a0d0200000000000e
:108c7c0061406000410020000100dd009940780057
:108c8c000144a10080cc700071ff3700600d020020
:108c9c0000000000b60b020000000000000178008c
:108cac00a2bf9f00600d020000000000b60b020086
:108cbc000000000080047800600d0200000000003d
:108ccc00b60b02000000000000067800600d0200e8
:108cdc0000000000b60b02000000000080057800c8
:108cec00600d020000000000b60b02000000000046
:108cfc002fb99700689b21000a4ce900edfe370064
:108d0c00609b210010407800e94f50002800320091
:108d1c0013d08000421ade004319de00614161006d
:108d2c00819c21009180fb00c408de00e1c0600042
:108d3c000080fb000000400085ad28006500780035
:108d4c0061426200e3c16100be7f020000000000ce
:108d5c0020a021001040780063406000e34f5000d9
:108d6c000a0032001a80020000000000c0118000ce
:108d7c002802e30001003e00000006000102200072
:108d8c00b01621006e7c04000000000091c0b300fe
:108d9c00709b2100014878001a800200000000003e
:108dac00c01180002802e300f3ff3600f3ff370008
:108dbc00c011800013d08000421ade004319de007f
:108dcc0061416100819c21009180fb00c408de00a0
:108ddc00e1c0600061426200e3c16100be7f02003d
:108dec000000000020a021001040780063406000cb
:108dfc00e34f5000dbff3a00e4ff3700248004000f
:108e0c00000000003222a90020a021001044a00084
:108e1c00809c21001024a000c1012000f0e620005d
:108e2c006e7c04000000000020a021001044a10072
:108e3c00809c21001024a10041012000b0e82000fa
:108e4c006e7c040000000000889fbe008004eb00d4
:108e5c0028a0210048800200000000000004e0006f
:108e6c001c0032009840780070c06000370032005f
:108e7c00e0a72800d265020000000000610020007d
:108e8c0080662000167c0200000000003262ab00fd
:108e9c0027003a003242ab001a003a004080020030
:108eac0000000000e87a0200000000003222ab0053
:108ebc000b003a00e0a72800d26502000000000079
:108ecc001900200048800200000000000004e000af
:108edc00e4ff3a00090078004f04be0000000600d1
:108eec00f1002000a0cf2000167c02000000000042
:108efc003222a900e0a72800d26502000000000081
:108f0c00efff37003100200070cf2000167c0200ec
:108f1c00000000004080020000000000e87a02001f
:108f2c00000000003222ab00e2ff3200ecff370001
:108f3c003100200040cf2000167c02000000000011
:108f4c003242ab00d5ff3200eeff3700408002000a
:108f5c000000000019002000daff3700b1002000eb
:108f6c00b00a21006e7c0400000000001e21ef00fe
:108f7c001021ef0080002000800888000821ef00fd
:108f8c000621ef001621ef001421ef00f0088800f5
:108f9c000000060011e1a9001fe1a9003034800097
:108fac00f001b300303488001e21ef001021ef00d7
:108fbc000621ef000821ef00000006000003be00b0
:108fcc0080a9280080017800110020005302be0007
:108fdc00860f5200878f5a0006003e008100e80081
:108fec00ef8f5000f9ff3a006011b8000200be008c
:108ffc00000006008100e900c208dd00010040000d
:10900c001001be000200520083805a008100d10082
:10901c000080d3000000410081804900800f530084
:10902c00818f5b00f1ff36000401be000200be0020
:10903c0000000600efff3700881f78008a9fbe00f3
:10904c0000047800cae2a900c8e2a8000800e00009
:10905c0071003200cae2ab00050032002202ab0004
:10906c0003003a0000000000cae2ab00fbff3a002c
:10907c00110020006033b800830020002202ab00f6
:10908c006c003a001e21ef001021ef0083088800cd
:10909c000821ef000621ef001621ef001421ef004c
:1090ac00f3088800cae2ab00feff32001fe1a80003
:1090bc0011e1a800cae2ab00feff3a0011e1a900e1
:1090cc001fe1a90030348000f001b3003034880077
:1090dc001e21ef001021ef004b0880000005eb0073
:1090ec00300880000a024000e0824d00e18f500001
:1090fc0008003200e00f5300e08f5b000f003200dd
:10910c00840f5300858f5b000c003e00f88f5000dd
:10911c000d003e008100e8001e21ef001021ef0041
:10912c00830888000821ef000621ef001621ef00cc
:10913c001421ef00f3088800daff37000403be00a7
:10914c00f88f5000f3ff360011e1a9001fe1a900d0
:10915c0030348000f001b300303488001e21ef0061
:10916c001021ef000621ef000821ef000601be00e0
:10917c0000402200410f2000860602000000000083
:10918c0080017800010178000305780082057800e1
:10919c000800e0001c003a00009f24002100200081
:1091ac00800f5500818f5d0036003e00f1002000dd
:1091bc0020252100167c0200000000000a00be00e1
:1091cc004a66020000000000410020000027210038
:1091dc006e7c020000000000f1002000102621002f
:1091ec00167c0200000000000a00be0073ff07009e
:1091fc004a66020000000000410020000027210008
:10920c006e7c0200000000000a00be004f05be008c
:10921c004f047800000006003101200020202100be
:10922c006e7c020000000000cae2ab008bff3a002b
:10923c008fff37003011800011e1a9001fe1a90058
:10924c0030348000f001b300303488001e21ef0070
:10925c001021ef000621ef000821ef00e1002000b3
:10926c00502121006e7c0200000000006055b80007
:10927c000a00be004f05be004f0478000000060037
:10928c00e5ff3700f1022000302221006e7c020045
:10929c00000000000a00be004f05be004f0478001d
:1092ac0000000600dcff3700881f780000047800ff
:1092bc00e20f54004500320008003e000800e000b8
:1092cc0011003a00a1062000f0dd2000167c0200ff
:1092dc00000000004f04780000000600e30f54006b
:1092ec0069003200e40f54005700320041022000a4
:1092fc00e01d20006e7c0200000000004f0478008e
:10930c0000000600f5ff3700e10f5400f7ff3a00ac
:10931c00b100200090e420006e7c020000000000f0
:10932c00d100200040e520006e7c0200000000000f
:10933c00007d0200000000000004e000e5ff3200a8
:10934c003222a9003202ab00040032002322ab000f
:10935c0002003a003602f8002402f900146a0200f6
:10936c0000000000e14f5000300032003222ab0010
:10937c0002003a002222ab00030032003222a90084
:10938c002222a900c222a900e30f5400edff3a00eb
:10939c00101680004400dd000010b2005116800051
:1093ac000180a100810070005116880051168000c8
:1093bc00c308de00e8806000101680000030a100b9
:1093cc000080700010168800deff3700e1002000de
:1093dc0010e620006e7c020000000000f10020006e
:1093ec00b01821006e7c0200000000003222a9009f
:1093fc003202ab00040032002322ab0002003a0020
:10940c003602f8002402f900146a02000000000081
:10941c00e14f5000f6ff3a00c66a0200000000005f
:10942c004f04780000000600acff37003322ab007d
:10943c00ceff3a00c66a0200000000000080fb006c
:10944c00a0118800c9ff3700248002000000000032
:10945c000000eb00f8fe07001a800200000000007c
:10946c00c01180002802e3009aff360001022000a0
:10947c00b01621006e7c0200000000004f04780042
:10948c000000060095ff3700c062a900c082a8004a
:10949c00c8c2a800c902a9009dff3700f0a7280088
:1094ac00b265040000000000889fbe008a9fbe00c9
:1094bc008c9fbe008e1f780029a021009940780057
:1094cc000100a1008c9c21001c44a0004041230001
:1094dc0020d0880002ceb30082cc60000042eb00aa
:1094ec00844178000441780011c0b300be7f0200b3
:1094fc00000000001a80020000000000f0a7280005
:10950c00b2650200000000008ba021007da02100ac
:10951c000b0778006aa021004880020000000000c0
:10952c000004e000070032009940780070c0600031
:10953c00230032004080020000000000d46a0200c8
:10954c00000000003222ab00010032003222a900e0
:10955c00146a02000000000000447800e14f54003f
:10956c00edff3a00c66a020000000000804d780052
:10957c000081fb00c411de00834e7800e4cf510063
:10958c009500320011003e000304e00050003a0048
:10959c00e24f50009c00320043003e000004e0000b
:1095ac0093003a0024800200000000004f0778006e
:1095bc004f06be004f05be004f04be000000060063
:1095cc004080020000000000deff3700e6cf5100b3
:1095dc00620032003a003900e8c05100e1cf50007f
:1095ec0037003e00194078000000a1000010a100d7
:1095fc000020a1000030a100804c78001c44a10088
:10960c000238a300030032000014a00021a02100a6
:10961c00804878000228a3000600320010d0800099
:10962c00634060000004a000c1cfb30099c060008b
:10963c0080cc70000218a300010032001924a00095
:10964c000208a300010032001934a0000248a30054
:10965c0001003a001c44a00024800200000000001d
:10966c0013d08000421ade004319de006141610014
:10967c009c80fb00c408de00e1c060006142620017
:10968c00e3c1610020d08000be7f0200000000001a
:10969c001a8002000000000010c0b300d46a02005f
:1096ac00000000009cff3700e74f500078003200ac
:1096bc00ef4f500061003200e34f50005a0032006f
:1096cc000040eb00d46a02000000000092ff37005b
:1096dc00e1cf5100faff3a006f406000004fe80004
:1096ec0003407800d46a020000000000004deb003b
:1096fc001e04e00088ff3200c66a02000000000071
:10970c000080fb00388002000000000010c0b30095
:10971c00d46a0200000000001a40e800004d7800f6
:10972c009b4f10007cff3600c66a02000000000050
:10973c000080fb00388002000000000010c0b30065
:10974c00d46a0200000000001a40e800004d7800c6
:10975c009b4f1000e8ff3e006fff37006f4060002a
:10976c00004f7800ea4f500002003600a0c0b30052
:10977c00004f78001b80fb000000400041a828002f
:10978c006100780020d088002480020000000000d6
:10979c0013d08000421ade004319de0061416100e3
:1097ac009c80fb00c408de00e1c0600061426200e6
:1097bc00e3c1610020d08000be7f020000000000e9
:1097cc001a8002000000000010c0b300d46a02002e
:1097dc000000000050ff370038810200000000003c
:1097ec0008407800d46a0200000000004aff3700ed
:1097fc00e14f5000b2ff3a00f0a72800b26502001a
:10980c000000000044ff370008407800d46a0200d2
:10981c00000000003222ab00010032003222a9000d
:10982c001944a0003cff37001944a10008407800ff
:10983c00d46a02000000000037ff370008407800af
:10984c00d46a0200000000003222a9003202ab00f0
:10985c00040032002322ab0002003a003602f8006a
:10986c002402f900146a020000000000e14f5000cd
:10987c00f6ff3a003322ab00f4ff3a00c66a02004e
:10988c00000000000080fb00a0118800efff3700f3
:10989c0008407800d46a0200000000002480020016
:1098ac0000000000c66a0200000000004800dd0055
:1098bc0020d0880008407800d46a02000000000024
:1098cc00c66a0200000000008080fb0020d08000ef
:1098dc000100700020d0880013d08000421ade00f6
:1098ec004319de00614161009c80fb00c408de006e
:1098fc00e1c0600061426200e3c16100be7f020012
:10990c00000000001a8002000000000008407800ef
:10991c00d46a020000000000fffe37001021ef00a7
:10992c001e21ef009c21ef0082cc80000200e000a1
:10993c0039003200e30f510019003e0010a1a800bd
:10994c001081a800e0032000110009000280d8005b
:10995c000000e9006008880091cc80000180b9000b
:10996c0043062000110009000380d8008000fd0090
:10997c0000fe2f00ca06b6006001b3005036880006
:10998c00d10c8800c10c880060002000e00c88001d
:10999c0011e1a80020002000a0cc880000000600e7
:1099ac00fe0f510020003600400f2000800f5100a8
:1099bc0036003e0010a1a9001081a800007d2000f7
:1099cc00110009000280d8000000e900600888003e
:1099dc0091cc80000180b9004306200011000900e1
:1099ec000380d8008000fd0000fe2f00ca06b600e0
:1099fc006001b30050368800d10c8800c10c88007f
:109a0c0060002000e00c880011e1a800200020007c
:109a1c00a0cc88000000060000fe2f00ca26b6006d
:109a2c00a2cc88000000060010a1a8001081a9009b
:109a3c00a00f2000110009000280d8000000e900ee
:109a4c006008880091cc80000180b900430620009a
:109a5c00110009000380d8008000fd0000fe2f00db
:109a6c00ca06b6006001b30050368800d10c8800dd
:109a7c00c10c880060002000e00c880011e1a800f7
:109a8c0020002000a0cc88000000060010a1a90036
:109a9c001081a90000e82300110009000280d80001
:109aac000000e9006008880091cc80000180b900ba
:109abc0043062000110009000380d8008000fd003f
:109acc0000fe2f00ca06b6006001b30050368800b5
:109adc00d10c8800c10c880060002000e00c8800cc
:109aec0011e1a80020002000a0cc88000000060096
:109afc00889fbe008a9fbe008c9fbe001021ef0085
:109b0c001e21ef009c21ef00a0cc8000e20f500042
:109b1c009000320010c480000000e800f007b20092
:109b2c0010c48800600d020000000000b60b02009b
:109b3c000000000000047800600d0200000000002e
:109b4c00b60b020000000000cf80de001005020002
:109b5c000000000000057800810478008a06780077
:109b6c00090678008800e9001b002000e0f92000bd
:109b7c00808f50006e003e006011b8000a00780023
:109b8c008900780094040200000000000000e0004e
:109b9c004e00340002002000832c24008a0278003e
:109bac000902780005007800840078009004020017
:109bbc00000000000000e00044003d00e18f550073
:109bcc0041003a002b002000e30f540052003e00ed
:109bdc0010a1a8001081a800e003200011000900ca
:109bec000880d8000004e900e28f55000f00320015
:109bfc0001012000902f2000167c020000000000c4
:109c0c008001eb00320620008000eb0020032000d6
:109c1c007a0d020000000000cf80de00100502006b
:109c2c00000000008006780001067800080078002b
:109c3c008000eb0074050200000000000005be006f
:109c4c0002002000832c24000c02be0005007800ca
:109c5c00840078000c040200000000000001be002b
:109c6c000a00be001e06020000000000da0402001a
:109c7c000000000001fe2f00523680008280600040
:109c8c006101b30051368800d00c8800c00c8800ec
:109c9c0060002000e00c88006808880011e1a80032
:109cac00a1002000903020006e7c0200000000001b
:109cbc0020002000a0cc88004f06be004f05be003f
:109ccc004f04be00000006001b002000408821004d
:109cdc000048eb0011012000a02c20006e7c02003b
:109cec000000000011012000b02d2000167c0200a5
:109cfc00000000008001eb0002fa2000110020009f
:109d0c00200320007a0d02000000000000047800ff
:109d1c00e30f5400aeff3600fe0f540033003e003c
:109d2c0010a1a8001081a900a00f2000abff3700e4
:109d3c008005eb006011b8000a00780089007800fb
:109d4c0094040200000000000000e000dfff34007b
:109d5c0090ff370000fe2f00ca26b600c10020007d
:109d6c00e02b20006e7c0200000000000000eb00e5
:109d7c00a0cc880010c480000000e800f007b200fe
:109d8c0001802100e14078000104e000caff3200ac
:109d9c0010c48800600d020000000000b60b020029
:109dac000000000000047800600d020000000000bc
:109dbc00b60b020000000000cf80de001005020090
:109dcc000000000000057800810478008a06780005
:109ddc00090678008800e9001b002000e0f920004b
:109dec00808f500064ff3600d1ff3700400f2000f9
:109dfc00800f540004003e0010a1a9001081a8009f
:109e0c00007d200075ff370010a1a9001081a9006a
:109e1c0000e8230071ff37000ea1ef000ca1ef004a
:109e2c000821ef000621ef001621ef001421ef00ae
:109e3c0080002000f0088800400f2000e008880017
:109e4c0000402200d00888008780a9001fe1a800ec
:109e5c0011e1a800010021003204800002806000a2
:109e6c00fdff320011e1a9001fe1a90032088000ba
:109e7c00a2cd8800410880000000eb0000014100e9
:109e8c00e081480082cd880093cd88000200be009e
:109e9c00000006001e21ef001021ef00c942a800af
:109eac0000fe2f008606b600a000b30030348800f8
:109ebc00a003200080088800d7ff0700f20f2000c5
:109ecc00820f5000e08f58000b0036004809dd006f
:109edc00c801de00830171004801dd0030348000d0
:109eec00f001b300303488001e21ef001021ef0088
:109efc000200be0000000600a000200080088800c0
:109f0c00c5ff07000001be0030348000f001b30033
:109f1c00303488001e21ef001021ef000200be003b
:109f2c0000000600f4ff3700889fbe008a9fbe0029
:109f3c000001780084a0a9008420a900f10f2e0054
:109f4c00703480008080600000a020000100700050
:109f5c007034880000fe2f008e06b600a000b300ff
:109f6c00703488000821ef000621ef0080002000eb
:109f7c008008880011e1a80030002000300a880019
:109f8c0030082000100a88004261ab000600320045
:109f9c00000a8000110a8000e8806000fcff3a0093
:109fac0050cd880061cd88004661ab0003003200c3
:109fbc00200a80004661ab00fdff3a004261ab0015
:109fcc00feff3200080a80008004eb0038cd8800c8
:109fdc0049cd88002a0a80008005eb00facc880065
:109fec000bcd88006000b800b0cc8800c1cc8800d4
:109ffc000000eb0070cd88006000b8008001eb0021
:10a00c000200e000250032004261ab00feff32008e
:10a01c00060a80008003eb00240a80008002eb001b
:10a02c000804530089845b000a0552008b855a0092
:10a03c00c055dd000a0020000804450089844d004d
:10a04c000000440081804c008301e800830f510024
:10a05c00050036000604be000405be004261ab00dc
:10a06c00e9ff3200eaff370056cd880067cd880043
:10a07c0036cd880047cd880014cd880025cd8800ca
:10a08c00d8cc8800e9cc8800b0cc8800c1cc880042
:10a09c00f4cc880005cd880072cd88004221ef00f9
:10a0ac004221ef0011e1a9008001eb0086060200bd
:10a0bc00000000004f05be004f04be00000006006b
:10a0cc00889fbe008a9fbe00a0cc8000e20f50008b
:10a0dc00cb003200f100200020332000167c02005f
:10a0ec00000000001e21ef001021ef00c942a80063
:10a0fc0000fe2f008606b600a000b30030348800a6
:10a10c00a00320008008880043ff07000004be0065
:10a11c006055b800f2ff2300820f5000e08f58000a
:10a12c0012003600c84cdd004840de008904700087
:10a13c004844dd000800be00546702000000000027
:10a14c00c0b12800d265020000000000303480004d
:10a15c00f001b300303488001e21ef001021ef0015
:10a16c004f05be004f04be0000000600b1002000e9
:10a17c00a0132100167c020000000000a0002000ab
:10a18c008008880024ff07000004be006055b8005a
:10a19c00f2f92000820f5000e08f5800e5ff3e00de
:10a1ac00e00f5400e08f5c00e00f5d00e08f5d007d
:10a1bc005b003200b1002000a0132100167c0200cd
:10a1cc00000000000800780057ff07006011b8007d
:10a1dc0004a82100650020006033b8000400e100f1
:10a1ec000588e1000690e1000798e1008c003e0034
:10a1fc00b4e12e00150020006033b8000400e1002b
:10a20c000588e1000690e1000798e1004d003e0052
:10a21c0004c42900050020006033b8000400e100ec
:10a22c000588e1000690e1000798e1001b013e0063
:10a23c0094162300050020006033b8000400e100f0
:10a24c000588e1000690e1000798e100a3003600c4
:10a25c0016050200000000000001be0000c22b0029
:10a26c00e1eb24000c040200000000009804020042
:10a27c00000000000004be000205be0044062000e1
:10a28c00050020006033b8000800be000a01780009
:10a29c00de0702000000000054670200000000000e
:10a2ac00e0c2b300d46a02000000000044062000a3
:10a2bc00050020006033b8000800be000a01be0093
:10a2cc00ec070200000000000004be000205be0006
:10a2dc0090002000010020006011b8000040e10057
:10a2ec0001c8e10002d0e10003d8e100e40036002f
:10a2fc00084078009468020000000000c0b12800fb
:10a30c00d26502000000000030348000f001b30080
:10a31c00303488001e21ef001021ef0090ff370031
:10a32c0000b22800d265020000000000303480002a
:10a33c00f001b300303488001e21ef001021ef0033
:10a34c0087ff370016050200000000000001be0068
:10a35c00902f2000512125000c0402000000000069
:10a36c0098040200000000000004be000205be00bc
:10a37c0004712200050020006033b8000800be0004
:10a38c000a017800de07020000000000546702009a
:10a39c0000000000e0c2b300d46a0200000000001c
:10a3ac0004712200050020006033b8000800be00d4
:10a3bc000a01be00ec070200000000000004be0011
:10a3cc000205be00703e2000010020006011b800a4
:10a3dc000040e10001c8e10002d0e10003d8e10037
:10a3ec008a00360008007800e866020000000000d1
:10a3fc00c0b12800d265020000000000c2ff370087
:10a40c00f1012000303120006e7c020000000000c1
:10a41c004f05be004f04be000000060053ff37007e
:10a42c0016050200000000000001be00703b240075
:10a43c00a13b25000c04020000000000980402005f
:10a44c00000000000004be000205be00046a2800e3
:10a45c00150020006033b8000800be000a01780027
:10a46c00de0702000000000054670200000000003c
:10a47c00e0c2b300d46a020000000000046a2800a5
:10a48c00150020006033b8000800be000a01be00b1
:10a49c00ec070200000000000004be000205be0034
:10a4ac00f0702200010020006011b8000040e100b3
:10a4bc0001c8e10002d0e10003d8e1002b00360016
:10a4cc000800be004a66020000000000c0b128006f
:10a4dc00d2650200000000008bff37001605020059
:10a4ec00000000000001be000068290081d124009a
:10a4fc000c040200000000009804020000000000a0
:10a50c000004be000205be00a400200005002000cf
:10a51c006033b8000800be000a017800de070200b4
:10a52c00000000005467020000000000e0c2b3000d
:10a53c00d46a020000000000a400200005002000e6
:10a54c006033b8000800be000a01be00ec07020030
:10a55c00000000009468020000000000c0b1280058
:10a56c00d26502000000000067ff370000c3b30093
:10a57c00d46a020000000000703e200001002000a0
:10a58c006011b8000040e10001c8e10002d0e10018
:10a59c0003d8e100caff3e0000c3b300d46a020036
:10a5ac000000000030062000010020006011b800ff
:10a5bc000040e10001c8e10002d0e10003d8e10055
:10a5cc00bfff3e0000c3b300d46a020000000000cd
:10a5dc0090002000010020006011b8000040e10054
:10a5ec0001c8e10002d0e10003d8e100b4ff3e0055
:10a5fc0000c3b300d46a0200000000000800be00d3
:10a60c004a66020000000000b0ff370000c3b30030
:10a61c00d46a020000000000300620000100200077
:10a62c006011b8000040e10001c8e10002d0e10077
:10a63c0003d8e1006bff3e0000c3b300d46a0200f4
:10a64c000000000090002000010020006011b80004
:10a65c000040e10001c8e10002d0e10003d8e100b4
:10a66c0060ff3e0000c3b300d46a0200000000008b
:10a67c0008007800e8660200000000005cff37006c
:10a68c0000c3b300d46a0200000000000840780048
:10a69c00946802000000000018ff37001605020045
:10a6ac00000000000001be0080b22600e10625007b
:10a6bc000c040200000000009804020000000000de
:10a6cc000004be000205be00843e200005002000f0
:10a6dc006033b8000800be000a017800de070200f3
:10a6ec00000000005467020000000000e0c2b3004c
:10a6fc00d46a020000000000843e20000500200007
:10a70c006033b8000800be000a01be00ec0702006e
:10a71c00000000000004be000205be003006200050
:10a72c00010020006011b8000040e10001c8e10008
:10a73c0002d0e10003d8e100bfff3600080078002a
:10a74c00e86602000000000029ff3700809c210011
:10a75c00104078006340600005003200c8c2a800b9
:10a76c00e100200010342000167c040000000000e2
:10a77c00c942a800e100200010342000167c04001f
:10a78c0000000000faff3700809c21001040780088
:10a79c006340600006003200c8c2a900cac2a8000b
:10a7ac0081002000f03420006e7c040000000000ca
:10a7bc00c942a900cb42a80081002000f03420003f
:10a7cc006e7c040000000000f9ff3700809c210023
:10a7dc00104078006340600006003200c8c2a90037
:10a7ec00cac2a90071002000703520006e7c0400e4
:10a7fc0000000000c942a900cb42a9007100200052
:10a80c00703520006e7c040000000000f9ff37005a
:10a81c00809c2100104078006340600008003200ea
:10a82c00c8c2a80000000000000000005016800004
:10a83c004600de00614060000080fb000000060066
:10a84c00c942a80000000000000000005016800063
:10a85c004a00de00614060000080fb000000060042
:10a86c00f7ff3700889fbe008a9fbe008c1f7800c0
:10a87c001021ef001e21ef009c21ef00a0cc8000e6
:10a88c00e20f50006600320010c480000000e800a7
:10a89c00f007b20010c48800600d02000000000038
:10a8ac00b60b0200000000004a8821001a04e000e8
:10a8bc000c003a00cf80de00100502000000000002
:10a8cc000004be0002002000433324000800be0038
:10a8dc0094040200000000000046eb000000e000c1
:10a8ec0010003400004deb0031012000301e21001f
:10a8fc006e7c0200000000008001eb00420b200087
:10a90c008000eb00a00520007a0d02000000000082
:10a91c00cf80de0010050200000000000004be0025
:10a92c001cc0b3000bfe2f002a4e200010a1a80063
:10a93c001081a80002002c00a35524008802780086
:10a94c000902780005007800840078000c040200ed
:10a95c000000000002002400c34924001e0602006f
:10a96c000000000002002000832724005203020094
:10a97c0000000000da0402000000000052368000e3
:10a98c00828065006101b30051368800d00c8800cc
:10a99c00c00c880060002000e00c88006a08880069
:10a9ac0011e1a800c1002000601f21006e7c020094
:10a9bc000000000020002000a0cc8800e14f5600d1
:10a9cc0013003a0013002000420b20008000eb0023
:10a9dc000080eb007a0d020000000000cf80de004a
:10a9ec0010050200000000000004be006011b80059
:10a9fc000800be0090040200000000000000e0000f
:10aa0c00caff3d0050b42800d265020000000000cf
:10aa1c004f0678004f05be004f04be000000060034
:10aa2c0010c480008000e800f107b2000280210011
:10aa3c00e2c078000104e00094ff3a0000fe2f0011
:10aa4c00ca26b600c1002000e02b20006e7c02005c
:10aa5c00000000000000eb00a0cc88004f0678003e
:10aa6c004f05be004f04be0000000600ecff37008f
:10aa7c0000ba2800b265040000000000889fbe00e8
:10aa8c008044780068c0b30061c06400a676020000
:10aa9c00000000008984fb008904d1000844e9000f
:10aaac00f9ff3a004277020000000000d46a02006d
:10aabc00000000004277020000000000d46a02008f
:10aacc00000000004f04be0000000600889fbe007e
:10aadc008a9fbe008c1f7800004478008144780067
:10aaec00024678000bc8b3008b4564006ac0b30003
:10aafc0061406400a6760200000000000884fb00a0
:10ab0c000804d1000a45e900f9ff3a000b04e00003
:10ab1c00040032004f0678004f05be004f04be0003
:10ab2c00000006000980fb00c47602000000000053
:10ab3c000c80fb00c4760200000000004f06780079
:10ab4c004f05be004f04be0000000600f5ff3700a5
:10ab5c00889fbe0048c0b3008084fb000908a30096
:10ab6c000900320010c0b300a676020000000000fd
:10ab7c000844e900090032000900d1008084fb0080
:10ab8c000908a300f7ff3a000040eb00a67602008c
:10ab9c00000000000844e900f7ff3a004277020089
:10abac00000000004277020000000000d46a02009e
:10abbc00000000004f04be0000000600889fbe008d
:10abcc008a9fbe008c1f78000144780002467800f2
:10abdc000085fb00c655de008044eb000a08a3008c
:10abec000b00320010c0b300a6760200000000007b
:10abfc008944e800e4cf54000b003200e3cf54004a
:10ac0c00130032000a05d1000a08a300f5ff3a0030
:10ac1c000040eb00a6760200000000008944e8002a
:10ac2c00e4cf5400f5ff3a000880fb00c476020024
:10ac3c00000000000c80fb00c47602000000000045
:10ac4c004f0678004f05be004f04be000000060002
:10ac5c000b04e000ebff320010c0b3009276020050
:10ac6c00000000000b80fb00cc7b02000000000009
:10ac7c000040eb0092760200000000000880fb0010
:10ac8c00c4760200000000000c80fb00c4760200b9
:10ac9c00000000004f0678004f05be004f04be00b8
:10acac0000000600eaff37000040eb00a676020029
:10acbc00000000000040eb00a6760200000000003f
:10accc000040eb00a6760200000000000040eb0004
:10acdc00a6760200000000000000eb00c476020023
:10acec00000000000000eb00c47602000000000031
:10acfc000000eb00c476040000000000889fbe003a
:10ad0c0000047800814478000040eb00a676020035
:10ad1c00000000000040eb00a676020000000000de
:10ad2c000040eb00a6760200000000000040eb00a3
:10ad3c00a6760200000000001880fb00c47602001a
:10ad4c0000000000184090000080fb00c476020058
:10ad5c0000000000284090000080fb00c476020038
:10ad6c0000000000efc4640003003200ceff0700b7
:10ad7c008944e900fdff3a004f04be0000000600c4
:10ad8c00889fbe008a1f78000004be000245780030
:10ad9c000040eb00a6760200000000000040eb0033
:10adac00a6760200000000000040eb00a676020030
:10adbc00000000000040eb00a6760200000000003e
:10adcc0008007800f07b020000000000c47602004e
:10addc00000000004849dd004840de000000710022
:10adec00c848de00f07b020000000000c4760200c0
:10adfc000000000009007800f07b02000000000059
:10ae0c00c4760200000000006f45650005003200aa
:10ae1c000044eb00a4ff07000844e800884f5500ed
:10ae2c00fcff3e004f0578004f04be0000000600fa
:10ae3c00881f780010c0b300a67602000000000046
:10ae4c000040eb00a6760200000000000040eb0082
:10ae5c00a6760200000000000040eb00a67602007f
:10ae6c00000000000000eb00c476020000000000af
:10ae7c0042770200000000000004780042770200d4
:10ae8c0000000000d46a02000000000008407800b6
:10ae9c00d46a02000000000083ff070082ff070055
:10aeac004f04780000000600e8874700889fbe002a
:10aebc008a9fbe008c9fbe008e1f78008a9c21004a
:10aecc001a4078000040a0000034a100004d78002a
:10aedc00f206550018c0b300884e780081c0b3004c
:10aeec0071005500014878008b9d210020c0b300f3
:10aefc00804d780080c0eb004a7502000000000015
:10af0c00c922a900c902a900c8e2a800084078001b
:10af1c00887602000000000000ba2800b26502002a
:10af2c0000000000c99d2100b89d21000906780091
:10af3c006ea22100c66a020000000000804c78005e
:10af4c008081fb004419de00024c7800e34f510075
:10af5c0015003200e34f510032003e00e14f51002a
:10af6c00f8003200810036006f4060000040e800bd
:10af7c00004e7800e27502000000000010c0b30023
:10af8c00d46a020000000000c66a02000000000043
:10af9c00804c78008081fb004419de00024c780064
:10afac00e34f5100ebff3a006f406000004ee800a9
:10afbc0010c0b300d46a020000000000c66a020090
:10afcc0000000000b19d210080487800a29d210066
:10afdc00f2b79f000049eb001c04e0000d003200aa
:10afec000004e000550035000040eb00a67602009e
:10affc00000000001840780000404000004c780031
:10b00c00ffb197009340e8008149780099cf100078
:10b01c00f3ff3e0010c0b300d46a02000000000031
:10b02c00c4ff3700e64f51003d0032000a003e00dd
:10b03c00e44f5100040032000040eb00d46a0200df
:10b04c0000000000bbff3700388102000000000048
:10b05c0010c0b300f0ff3700e84f51000e00320073
:10b06c00ea4f5100f4ff3a0041cab300814f50003f
:10b07c00ac01320001013e00e4c05000814f500091
:10b08c00edff3a00c66a020000000000004f780095
:10b09c0010c0b300e0ff37001a4078000040a10058
:10b0ac00004d78000338a30003003a000044a000d0
:10b0bc00819c21008048780020c0b300804d78002e
:10b0cc000328a3000300320030c0b300829d21008e
:10b0dc00004978001a4078000030a100004d78003b
:10b0ec000318a300030032000034a000839c21004d
:10b0fc00804978009d4078001b4078004a7502001a
:10b10c000000000010c0b3008876020000000000b0
:10b11c0010c0b300d46a02000000000085ff3700a5
:10b12c00e3406000014e7800814e78001b407800af
:10b13c004a75020000000000f2ff370010c0b30097
:10b14c00a676020000000000184078000040400085
:10b15c00004c7800ffb197009340e80081497800db
:10b16c0099cf10009eff3e00aaff37000080fb0025
:10b17c008000eb00ed0f5000e08f5800aeff3e005a
:10b18c0000600100620037005d0037005600370098
:10b19c004f00370047003700daff37002d0037002b
:10b1ac002700370021003700190037001100370045
:10b1bc0009003700010037005b0037000040eb004e
:10b1cc009c7602000000000010c0b300d46a02009c
:10b1dc000000000057ff370010c0b3009276020049
:10b1ec000000000010c0b300d46a02000000000090
:10b1fc0050ff37000040eb00927602000000000088
:10b20c0010c0b300d46a02000000000049ff3700f0
:10b21c0010c0b300e27502000000000010c0b300c3
:10b22c00d46a02000000000042ff37001c770200c5
:10b23c0000000000d46a0200000000003dff37004f
:10b24c002077020000000000d46a02000000000019
:10b25c0038ff370020c0b3009b4f1000360232007d
:10b26c00f00f2000847702000000000080007800be
:10b27c0001407800a39d2100f3b79f00814978001d
:10b28c001a417800e840610063ff32000080fb0047
:10b29c00f07b020000000000800078000140780084
:10b2ac00ffb1970081497800d46a020000000000c9
:10b2bc0020ff37000040eb00887602000000000001
:10b2cc0010c0b300d46a02000000000019ff370060
:10b2dc00087602000000000010c0b300d46a02001f
:10b2ec000000000013ff370024760200000000006d
:10b2fc0010c0b300d46a0200000000000dff37003c
:10b30c0000ba2800b26502000000000009ff3700f7
:10b31c004f0778004f06be004f05be004f04be001d
:10b32c008f00b1000000060010c0b3009c76020034
:10b33c000000000010c0b300d46a0200000000003e
:10b34c00fcfe37006f406000004ee80002407800c1
:10b35c00d46a020000000000a09d2100f0b79f00fd
:10b36c000048eb001c04e000f2fe3200919d21002d
:10b37c00e1b79f00c66a0200000000006fb19700a1
:10b38c00004978009a417800e8c061001b003a003f
:10b39c0023c0b3009bcf1100220032000080fb00c1
:10b3ac008477020000000000804078006fb19700a5
:10b3bc00004978009a41780068c0610025003a0085
:10b3cc0001407800d46a020000000000ffb1970031
:10b3dc001340e80080497800994f1000d5fe3600e4
:10b3ec00c66a0200000000006fb1970000497800a7
:10b3fc009a417800e8c06100e5ff32000080fb0054
:10b40c00f07b020000000000800078000140780012
:10b41c00929d21000149780023c0b3009bcf1100fd
:10b42c00deff3a000080fb00c47602000000000042
:10b43c0010c0b300d46a020000000000ffb19700f6
:10b44c001340e80080497800994f1000e4ff3e005b
:10b45c00b8fe37000180fb00f07b0200000000000a
:10b46c0080407800929d21000049780001407800ce
:10b47c00d46a020000000000d4ff370051cab300a8
:10b48c00814f50006800320081c0e800814f5000ad
:10b49c00e9fe3a00c66a0200000000000080fb00d2
:10b4ac00a0ce8800c66a0200000000008080fb006d
:10b4bc0091ce88001e407800e24f50007f01320090
:10b4cc00e14f500002003200e34f5000dafe3a0028
:10b4dc00a0ce8000000040008080400081804000b1
:10b4ec00b1ce88000000eb0080ce88000100e000a7
:10b4fc00100032008000eb00e09d2100e0b79f00bf
:10b50c006fb197009280400081bf9f00c66a020015
:10b51c00000000008fb897008048780081ce800032
:10b52c008100e80081ce8800b0ce8000810f5000f1
:10b53c00f3ff3e0090ce80000000e00021003a00b6
:10b54c000000eb0080ce8800b3ce80000001eb0041
:10b55c00830f510009003100f0ce8000e0407900eb
:10b56c00e1cf50001f003200e2cf50000800320043
:10b57c0082ce8000830f5100f7ff390090ce8000ff
:10b58c000000e0006bfe3a0010c0b300a2fe3700d2
:10b59c009e407800e3cf500057013200e1cf5000bd
:10b5ac005d013200e2cf5000f1ff3a0020fe0700af
:10b5bc0082ce80000201e80082ce8800b3ce8000eb
:10b5cc00e3ff370010c0b300d46a02000000000093
:10b5dc000000eb0080ce8800b3ce80000001eb00b1
:10b5ec00dbff37009e407800e3cf5000290132008a
:10b5fc00e1cf500036013200e2cf5000dcff3a00c0
:10b60c0082004000c14090000201e80002004000ae
:10b61c00bafd070082ce80006501410082ce880011
:10b62c00b3ce8000caff37001e407800e14f5000b7
:10b63c00d5003200e24f50003efe3a00c66a0200ce
:10b64c00000000000080fb00b0ce88008000eb0002
:10b65c0081ce880037fe320022c0b30060b92000d2
:10b66c00a10b2000c6fd0700f1fd070022c0b300ae
:10b67c0060bb2d00a10b2000c1fd070022c0b30050
:10b68c00603d2d00a10b2000bdfd0700e8fd07006b
:10b69c0022c0b30060bb2000a10b2000b8fd070046
:10b6ac00e3fd070080ce80000000e80080ce88001b
:10b6bc00b1ce8000808f50001efe360022c0b30039
:10b6cc0060b92000a10b2000adfd0700d8fd0700dc
:10b6dc0022c0b30060bb2d00a10b2000a8fd070009
:10b6ec0022c0b300603d2d00a10b2000a4fd07007b
:10b6fc00cffd070022c0b30060bb2000a10b2000cf
:10b70c009ffd0700cafd070080ce80000000e80006
:10b71c0080ce8800b1ce8000808f5000ceff3e00de
:10b72c0004fe37001e407800e14f50005e003200ee
:10b73c00e24f500040fe3a00c66a020000000000d2
:10b74c000080fb004200dd00b0ce88008000eb00e2
:10b75c0081ce880008013200e39d2100e3b79f00f1
:10b76c006fb097009080400081bf9f00c66a0200b6
:10b77c00000000008fb897008048780081ce8000d0
:10b78c008100e80081ce8800b0ce8000810f50008f
:10b79c00f3ff3e008000eb0081ce88000000e0004b
:10b7ac003d003200a19d2100f1b79f000040eb004d
:10b7bc00a6760200000000000040eb00a676020016
:10b7cc00000000000040eb00a67602000000000024
:10b7dc000040eb00a67602000000000080ce800046
:10b7ec00f1ce8000614078000080fb00c47602003e
:10b7fc000000000080ce8000f1ce80000080400070
:10b80c00104090000080fb00c47602000000000095
:10b81c0080ce8000f1ce800000804000204090005f
:10b82c000080fb00c47602000000000081ce800086
:10b83c0063804000efb19700130140009241780003
:10b84c006fc961007fb197000049eb00f2ce800018
:10b85c00624078000004e0000a00320012fd07008c
:10b86c00ffb197001340e8008049780081ce80003a
:10b87c00f2ce80000101410032419000804f510016
:10b88c00f6ff3e00e480400081ce8800b0ce800000
:10b89c00810f5000c5ff3e0010c0b300d46a0200f7
:10b8ac0000000000a3fd3700c66a02000000000083
:10b8bc000080fb006300b90000017800b0ce880066
:10b8cc000000eb0080ce88000200e000a5003200f2
:10b8dc008000eb00e09d2100e0b79f006fb1970066
:10b8ec009280400081bf9f00c66a020000000000e9
:10b8fc008fb897008048780081ce80008100e800e6
:10b90c0081ce8800b0ce8000810f5000f3ff3e0046
:10b91c008000eb0081ce88000000e000deff3200ea
:10b92c000000eb00f3ce80008080410021419000ac
:10b93c009140900063407800a0fc070080ce80000e
:10b94c006300400080ce8800b1ce8000808f500014
:10b95c00d1ff3600f3ce8000808041002141900061
:10b96c00914090006340780094fc070080ce8000ea
:10b97c006300400080ce8800b1ce8000808f5000e4
:10b98c00e8ff3e00c4ff3700c66a0200000000005a
:10b99c000080fb00b0ce8800c66a020000000000e8
:10b9ac00004c78008000eb0081ce8800b1ce800086
:10b9bc000100e0005ffd3200a19d2100f1b79f0066
:10b9cc00929d2100e2b79f00efb19700804978006b
:10b9dc00ffb097008048eb000008a3001f00320066
:10b9ec0010c0b300a6760200000000006fb19700f3
:10b9fc009280fb008100d100014078000149780061
:10ba0c00ffb197009340e80081497800e3cf5000e4
:10ba1c00f1ff36004277020000000000427702007e
:10ba2c0000000000d46a02000000000080ce8000fc
:10ba3c000000e80080ce8800b1ce8000808f5000de
:10ba4c003cfd360018407800efb197008049780033
:10ba5c00ffb097008048eb00dfff37000040eb00a1
:10ba6c00a6760200000000006fb197009280fb00e8
:10ba7c008100d1000140780001497800ffb19700a6
:10ba8c009340e80081497800e3cf5000d2ff3600a4
:10ba9c00e0ff37000200400030419000a0409000d1
:10baac001040900009fc070082ce80006401410028
:10babc0082ce8800b3ce8000a5fe3700a2ce8000d7
:10bacc006511b90082804000b1ce880085fe370038
:10badc000200400030419000a040900010409000c7
:10baec0036fc070082ce80006401410082ce8800c3
:10bafc00b3ce800096fe370002004000104090004c
:10bb0c00defb070082ce80000281e80082ce880036
:10bb1c00b3ce80008efe3700020040001040900033
:10bb2c000bfc070082ce80000281e80082ce8800e8
:10bb3c00b3ce800086fe3700427702000000000082
:10bb4c008000780001407800a29d2100f2b79f0090
:10bb5c00014978001a417800e84061002efd32005e
:10bb6c00cafd370082ce880010c0b300d46a020030
:10bb7c0000000000effc37000000eb0080ce8800d6
:10bb8c0010c0b300d46a020000000000e9fc3700ca
:10bb9c00881f7800e8a12100984078000118a300c4
:10bbac000f0032000108a3001a00320000c2b300db
:10bbbc00d46a020000000000310020003041200057
:10bbcc00167c02000000000000c2b300d46a020020
:10bbdc0000000000984078000110a100014c780092
:10bbec000000eb000108a300030032001814a000b1
:10bbfc004f047800000006004277020000000000ad
:10bc0c000080fb001814a0004f0478000000060010
:10bc1c00f9ff37000040eb00a676020000000000a0
:10bc2c0000c2b300d46a0200000000003100200002
:10bc3c0030412000167c02000000000000c2b3005e
:10bc4c00d46a020000000000984078000110a100a6
:10bc5c00014c7800e2ff3700889fbe00800478001a
:10bc6c00e8a12100184078000018a30021003a0038
:10bc7c000008a3000c00320000c2b300d46a02001a
:10bc8c00000000000900e00012003200410020001a
:10bc9c0060412000167c0200000000000010200013
:10bcac004f04be000000060009007800c4760200b4
:10bcbc000000000020770200000000008084fb00e0
:10bccc0000c2b300d46a0200000000000900e000ca
:10bcdc00eeff3a003100200030412000167c0200bb
:10bcec0000000000003020004f04be0000000600e1
:10bcfc00edff370000c2b300d46a02000000000060
:10bd0c003100200030412000167c020000000000b1
:10bd1c0000c2b300d46a0200000000009840780012
:10bd2c0061c0600006003200184078000010a100cd
:10bd3c00004c78000008a300cfff3a00daff370070
:10bd4c00a676020000000000184078000010a10048
:10bd5c00004c7800f7ff3700881f7800e8a121001d
:10bd6c00184078000018a3001e003a000008a30039
:10bd7c0006003200d1002000a04120006e7c0200a1
:10bd8c00000000004f04780000000600247602003a
:10bd9c00000000000000e000f6ff320091002000df
:10bdac00c0202000167c0200000000005101200081
:10bdbc0050212000167c02000000000040b8280032
:10bdcc00d265020000000000d1002000a04120003c
:10bddc006e7c0200000000004f047800000006009a
:10bdec00eaff37004100200060412000167c020071
:10bdfc000000000040b82800d265020000000000de
:10be0c009840780061c0600006003200184078004d
:10be1c000010a100004c78000008a300d5ff3a00e8
:10be2c00daff370010c0b300a67602000000000055
:10be3c00184078000010a100004c7800f6ff370085
:10be4c00881f7800e8a12100184078000018a30092
:10be5c0011003a000008a30006003200c1002000c7
:10be6c00704220006e7c0200000000004f0478003d
:10be7c00000006000876020000000000c10020004f
:10be8c00704220006e7c0200000000004f0478001d
:10be9c0000000600f7ff3700410020006041200041
:10beac00167c02000000000040b82800d265020099
:10bebc00000000009840780061c06000060032006d
:10becc00184078000010a100004c78000008a30076
:10bedc00e2ff3a00e7ff370010c0b300a67602007d
:10beec0000000000184078000010a100004c780001
:10befc00f6ff370001012000404f2000167c0200a5
:10bf0c00000000000040eb009468020000000000fc
:10bf1c0000c2b300d46a020000000000609b210044
:10bf2c0010407800946802000000000000c2b300ca
:10bf3c00d46a02000000000050b82800d26504004a
:10bf4c0000000000881f7800e8a121001804a1005f
:10bf5c00600d020000000000b60b020000000000a3
:10bf6c008000e900e38f50000c003e00619b210033
:10bf7c008048e90041cf800030002300808f5000c2
:10bf8c001a003600dbff07001814a100809c21006a
:10bf9c001044a0004f0478000000060040882100e7
:10bfac000048eb001804a100b103200080452000dc
:10bfbc006e7c0200000000008001eb0042002000bb
:10bfcc0011002000100020007a0d0200000000007b
:10bfdc00619b21008048e900809c21001044a00056
:10bfec004f04780000000600ecff370051032000de
:10bffc0030492000167c020000000000bdff070045
:10c00c001814a100e1ff3700e0a1210010407800d6
:10c01c00614060000100320000000600c922a80047
:10c02c00c902a800cb02a900cb22a900609b210069
:10c03c009040780020c0b3004a7504000000000056
:10c04c00e1a12100114078000010a1008048780087
:10c05c000008a3000100320007e2a900000006005e
:10c06c00b1002000600b21006e7c04000000000079
:10c07c00889fbe008a9fbe008c9fbe008e1f7800da
:10c08c00004678001a6a020000000000c922a800cd
:10c09c00c902a800cb02a900cb22a90062a0a8006b
:10c0ac0062c0a8008660a9005a1680004955de00bf
:10c0bc00581680004844de00614464006145650008
:10c0cc000047eb008e4678008e4578008660ab000a
:10c0dc0011003a00286a020000000000146a0200f5
:10c0ec00000000000004e000f8ff3200c66a020005
:10c0fc000000000062a0a90062c0a9000c04e000ce
:10c10c0032003a004f0778004f06be004f05be00c4
:10c11c004f04be00000006008660a900591680007e
:10c12c00c94cde00e1c46400501680004800de00fb
:10c13c00614060000b04e0000e0032000804e000d7
:10c14c0011003a000004e0000d003200e7cf560069
:10c15c002c003e000e4747000904e00001003200ad
:10c16c000e04a0008d46e8000945780018c0b30005
:10c17c00d6ff37000804e00003003a0000447800c2
:10c18c0009457800d1ff37000004e0000c003200b4
:10c19c000a04e00016003a0018c0b3000904e000dd
:10c1ac00caff3200d0c5b3007e6a02000000000056
:10c1bc008046eb008d45780008457800c3ff3700ba
:10c1cc00094578000044eb00c0ff370040b8280058
:10c1dc00d2650200000000004f0778004f06be0039
:10c1ec004f05be004f04be0000000600caff37001a
:10c1fc000904e000110032001ac0b3000a447800b0
:10c20c00b2ff37000c04e000140032000e80fb007b
:10c21c00a66a0200000000000904e00016003200cb
:10c22c00d0c2b3007e6a0200000000008046eb0022
:10c23c0018c0b30008457800a4ff3700b0c5b300a0
:10c24c007e6a0200000000008046eb001bc0b300b9
:10c25c000b4478000d4578009cff3700c0c5b30037
:10c26c007e6a0200000000000e4078007e6a020028
:10c27c0000000000e8ff3700b0c2b3007e6a020085
:10c28c00000000008046eb0018c0b3000d4578009c
:10c29c008eff3700889fbe008a9fbe000004780086
:10c2ac00e10f54001200320009003900e20f540073
:10c2bc003000320041022000e01d20006e7c0200a4
:10c2cc00000000004f05be004f04be000000060039
:10c2dc005103200040502000167c0200000000009a
:10c2ec004f05be004f04be0000000600f8ff3700eb
:10c2fc008040eb0000302000b87502000000000008
:10c30c00e1022000905320006e7c0200000000002f
:10c31c00cb02ab005e003200cb22ab005c003200e3
:10c32c008004eb00eaa121000b1020009a40780059
:10c33c0061c06000430032000800e00026003200bb
:10c34c009a40780061c060001d0032008904e8004a
:10c35c008b8f5400f5ff3a0040b82800d2650200dc
:10c36c00000000004f05be004f04be000000060098
:10c37c00d7ff3700e0a12100104078006140600039
:10c38c000100320007e2a900710020007056200065
:10c39c006e7c020000000000f1002000b0182100ab
:10c3ac006e7c02000000000010c0b30030ff0700dc
:10c3bc004f05be004f04be0000000600c4ff37004e
:10c3cc0008760200000000008904e8008b8f5400fe
:10c3dc00d6ff3a00e0ff370009007800e87a020047
:10c3ec000000000080c2b300d46a0200000000000c
:10c3fc000980d100e87a0200000000000908a300bf
:10c40c00320032009a40780061c0600017003200a0
:10c41c00a0b82800b26502000000000050b8280047
:10c42c00b26502000000000000c2b300d46a020032
:10c43c00000000009a40780061c06000c3ff3a0021
:10c44c00dfff3700247602000000000009007800ae
:10c45c00c4760200000000002077020000000000fb
:10c46c000084fb00b6ff3a00dbff37004277020086
:10c47c000000000010c0b300a6760200000000000f
:10c48c00a0b82800b265020000000000e3ff3700ee
:10c49c0091002000c0202000167c0200000000004b
:10c4ac005101200050212000167c020000000000e9
:10c4bc0040b82800d2650200000000004f05be0005
:10c4cc004f04be000000060081ff370070b8280042
:10c4dc00b26502000000000050b82800b2650200ee
:10c4ec000000000000c2b300d46a0200000000008b
:10c4fc00d0ff3700d0b82800b2650400000000005f
:10c50c00ea874700889fbe008a9fbe008c9fbe00b2
:10c51c008e1f7800c922a800c902a800cb02a9006e
:10c52c00cb22a900c8c2a9008d9c21001d40780017
:10c53c000040a0000034a100804e780080c0eb00c9
:10c54c0020c0b3004a75020000000000d0b82800db
:10c55c00b26502000000000019a221000aa221000d
:10c56c00890578000e002100ec9d2100f8a1210026
:10c57c00c66a020000000000804c78000081fb00bd
:10c58c004411de00024d7800e14f510012003200e0
:10c59c00e14f5100a60031000080fb008000eb0051
:10c5ac00ef0f5000e08f58002e0036000040eb00db
:10c5bc00d46a020000000000c66a020000000000fd
:10c5cc00804c78000081fb004411de00024d7800a5
:10c5dc00e14f5100eeff3a006f406000804de800e3
:10c5ec0002407800d46a020000000000004ceb000e
:10c5fc001b04e000deff3200c66a020000000000ef
:10c60c000080fb00c47602000000000020770200ce
:10c61c0000000000d46a0200000000001840e8008e
:10c62c00004c7800994f1000d1ff3600c66a02000a
:10c63c00000000000080fb00c47602000000000037
:10c64c002077020000000000d46a02000000000005
:10c65c001840e800004c7800994f1000e6ff3e00af
:10c66c00c3ff3700006001006b0037006600370025
:10c67c00130037000c0037001e003700cbff3700cb
:10c68c0015003700590037003b00370024003700f5
:10c69c00c6ff3700c5ff3700c4ff3700c3ff3700a4
:10c6ac00c2ff3700180037000876020000000000b7
:10c6bc0010c0b300d46a020000000000acff3700c9
:10c6cc00247602000000000010c0b300d46a0200ff
:10c6dc0000000000a6ff37000040eb00a676020029
:10c6ec000000000010c0b300d46a0200000000007b
:10c6fc009fff37004277020000000000d46a02005e
:10c70c00000000009aff37000040eb0058fe0700c5
:10c71c0010c0b300d46a02000000000094ff370080
:10c72c0010c0b300d46a0200000000002202ab006b
:10c73c00feff32003111800001407800814c7800fe
:10c74c00e2cf5000d3003200a3003600f0cf5000ef
:10c75c00ca00320001c2b300814f5000b000320059
:10c76c00e34f5000b600320010c0b300d46a020090
:10c77c00000000007eff3700c66a020000000000c7
:10c78c00c800dd0081bf9f00c66a020000000000e7
:10c79c000080fb008fb8970001007000e0b79f008d
:10c7ac00c66a020000000000a0ef9f00c66a0200eb
:10c7bc0000000000efb097008e8f500007003e0085
:10c7cc002fe99700c810dd000080fb00010070000d
:10c7dc00d0b79f008e0f5000280036000040eb00b1
:10c7ec00d46a02000000000061ff370010c0b300e3
:10c7fc00a67602000000000010c0b300d46a02004c
:10c80c00000000005aff3700d0b82800b2650200c3
:10c81c000000000056ff37004f0778004f06be009f
:10c82c004f05be004f04be00af00b1000000060073
:10c83c00e44f51000b003200e64f5100e7ff3a0085
:10c84c00e3406000814d780020c0b3004a750200bf
:10c85c000000000010c0b300d46a02000000000009
:10c86c0043ff3700388102000000000010c0b30005
:10c87c00d46a0200000000003dff37008000eb008e
:10c88c006fb097000000e000880032001c8140006f
:10c89c0081bf9f00f2b79f00c66a02000000000033
:10c8ac007fb19700004978008fb897008100e800ad
:10c8bc006fb19700810f5100f4ff3e002476020007
:10c8cc00000000008000eb00f0ce800060c078001b
:10c8dc000080fb0081bf9f00c476020000000000b6
:10c8ec0020770200000000008fb89700e14f500045
:10c8fc00baff32008100e8006fb09700810f500042
:10c90c00f1ff3e00dfb097008100e900e1b79f0026
:10c91c005fb197000200e00063ff32008000eb0083
:10c92c001c81400081bf9f00f2b79f00427702003c
:10c93c00000000007fb19700004978008fb8970085
:10c94c006fb09700808f5000420031000040eb0028
:10c95c00a6760200000000008fb897008100e80066
:10c96c005fb19700810f5100edff3e000876020089
:10c97c000000000010c0b300d46a020000000000e8
:10c98c008000eb00f0ce800060c0780081bf9f007b
:10c99c00d46a0200000000008fb897008100e80004
:10c9ac005fb09700810f5000f1fe3600f0ce800092
:10c9bc0060c0780081bf9f00d46a020000000000b4
:10c9cc008fb897008100e8005fb09700810f50008e
:10c9dc00ecff3e00e6fe37000104e00006003a00e2
:10c9ec00ec5302000000000010c0b300d46a020037
:10c9fc0000000000defe3700e1cf50005aff3a0085
:10ca0c0081bf9f00ca530200000000008fb897003e
:10ca1c0001407800d46a020000000000d4fe370008
:10ca2c001d4078000000a0000014a100804e78008a
:10ca3c0010c0b300d46a020000000000ccfe370026
:10ca4c000e54020000000000d46a02000000000036
:10ca5c00c7fe370010c0b30081bf9f00a67602004e
:10ca6c00000000008fb897008100e8005fb19700cc
:10ca7c00810f5100aaff3e00bcff3700c0cfb300ae
:10ca8c009d4e600010c0b300d46a0200000000008c
:10ca9c00b7fe3700ac5302000000000010c0b3001a
:10caac00d46a020000000000b1fe370024760200b8
:10cabc000000000093ff37000000e0000900320086
:10cacc0000102000a19e2100110060000d003a0012
:10cadc002322ab00feff3a00100320002011880037
:10caec000000060000102000a19e21001100600033
:10cafc0004003a002322ab00feff3a0000032000a2
:10cb0c0020118800000006000100e000090032003e
:10cb1c0054cf80000410b2000001eb00b04178004b
:10cb2c000400e000040032000201e800828f500093
:10cb3c00faff3e00000006002322ab00feff3a0085
:10cb4c008301fb00231188000201e800828f500052
:10cb5c00f2ff3e00f7ff370002102000a19e2100db
:10cb6c0011016100b04078000104e00009003200be
:10cb7c000200e000fbff3a002322ab00feff3a006c
:10cb8c008100fb0021118800b04078000104e00016
:10cb9c00f7ff3a000000060052cf80000210b200ee
:10cbac00b04078000104e000090032000200e0000f
:10cbbc00fbff3a002322ab00feff3a008100fb0092
:10cbcc0021118800b04078000104e000f7ff3a0022
:10cbdc000200e00001003200000006002322ab003e
:10cbec00feff3a00d0002000201188002322ab0069
:10cbfc00feff3a00a0002000201188000000060073
:10cc0c00881f780000447800c0ae2800d2ff0700cf
:10cc1c0003102000a09e21009081610080c0b30011
:10cc2c0001c8b300050320001403200008c16000f4
:10cc3c00080032000300e0000f0032000040e90061
:10cc4c000b0032008180fb008100d10008c1600024
:10cc5c00f8ff3a000300e000f8ff3a002322ab0093
:10cc6c00feff3a00251188000040e900f5ff3a006c
:10cc7c004f047800000006002322ab00feff3a00b0
:10cc8c0024118800edff3700889fbe008a9fbe00ec
:10cc9c008c9fbe008e1f78000006be005ecf800009
:10ccac000e10b2008ac0b3008045eb0008102e00b5
:10ccbc00595f20000801be000c00be008606020071
:10cccc00000000000001be000b04e00015003a005b
:10ccdc00e00f5100e08f590012003a000a45e900bc
:10ccec001c003200a2002000030020000800be003f
:10ccfc008606020000000000800178000101780027
:10cd0c0003047800820478000801be000c00be0009
:10cd1c0086060200000000000001be000b04e000cb
:10cd2c00ebff32000e00e000170032000898b9004b
:10cd3c0002cab900000042000811b800830140008b
:10cd4c000206560083865e001bc0b3000a45e9004c
:10cd5c00e4ff3a000e00e00006003a002322ab008c
:10cd6c00feff3a0001c3b300014046000000fb0087
:10cd7c00201188004f0778004f06be004f05be00fb
:10cd8c004f04be00000006002322ab00feff3a0059
:10cd9c0001c3b300014041000000fb0020118800da
:10cdac000898b90002cab900000042000811b80086
:10cdbc00830140000206560083865e001bc0b30050
:10cdcc00e2ff3700889fbe008a9fbe0000057800f6
:10cddc0055cf80000510b2004bc0b3000042eb00f1
:10cdec0002712200a6002000110009000285d80063
:10cdfc00800178000404e0000c003a000300e0001d
:10ce0c000a003a008b45e9000f00320011000900be
:10ce1c000681d80000017800110009000285d800b5
:10ce2c00800178000404e000f4ff32000500e0000b
:10ce3c0010003200029cb9000805550014c0b30064
:10ce4c008b45e900f1ff3a000500e00006003a00ce
:10ce5c002322ab00feff3a0001c3b30001404500a2
:10ce6c000000fb00201188004f05be004f04be00df
:10ce7c00000006002322ab00feff3a0000c3b30003
:10ce8c0000c241000402fb0024118800029cb9007e
:10ce9c000805550014c0b300e9ff3700889fbe0099
:10ceac008a9fbe008c9fbe000004be00f0232400ad
:10cebc00f1002000800f5400818f5c004e003e007a
:10cecc008005eb00703e2000800f5400e08f5c006a
:10cedc0017003e0030062000800f5400e08f5c00ed
:10ceec000d003e000b00e0000b003200e90f540077
:10cefc00e08f5c007800360000102000a19e21001d
:10cf0c001100600004003a002322ab00feff3a003f
:10cf1c00000320002011880008007800a9ff0700fa
:10cf2c004f06be004f05be004f04be0000000600b9
:10cf3c00aa9e2100823e2000030020000800be00b3
:10cf4c0086060200000000000006be00300620002d
:10cf5c00800f5600e08f5e0008003e000b00e000e2
:10cf6c0006003200e90f5600e08f5e0063003600c9
:10cf7c00001020001a0060004d0032000c007800f8
:10cf8c0090ff0700001020001a0060000b00320018
:10cf9c00823e2000030020000800be00a60602000e
:10cfac000000000080017800010178000304780083
:10cfbc00820478001b002000c6ff37002322ab0040
:10cfcc00feff3a00c002200020118800823e2000a3
:10cfdc00030020000800be00a606020000000000ae
:10cfec008001780001017800030478008204780045
:10cffc001b002000b7ff370002242400f3002000a0
:10d00c000800be0086060200000000006dff07004d
:10d01c00aa9e2100001020001a00600011003200ae
:10d02c0002242400f30020000800be00a606020023
:10d03c0000000000800178000101780003047800f2
:10d04c00820478001b002000703e2000800f5400ea
:10d05c00e08f5c00b7ff3e00f0ae2800befe07007c
:10d06c009cff37002322ab00feff3a00c0022000d9
:10d07c002011880002242400f30020000800be00c8
:10d08c00a606020000000000800178000101780073
:10d09c0003047800820478001b002000703e2000fe
:10d0ac00800f5400e08f5c00a2ff3e00eaff3700c7
:10d0bc002322ab00feff3a00000320002011880061
:10d0cc000c0078003fff0700001020001a006000e1
:10d0dc00afff3a00b9ff370040af28009efe0700b3
:10d0ec000800780037ff07004f06be004f05be0052
:10d0fc004f04be00000006008dff370040af280033
:10d10c0095fe07000c0078002eff07000010200091
:10d11c001a0060009eff3a00a8ff3700889fbe00ef
:10d12c008a9fbe008045780054cf80000410b20066
:10d13c002ac0b3008042eb0042c6b300a600200018
:10d14c008b81fb000281fb00110009008281d80059
:10d15c00800178000504e0000e003a000304e000b2
:10d16c000c003a000a45e9001100320011000900d8
:10d17c000681d800000178008b81fb000281fb0046
:10d18c00110009008281d800800178000504e000bc
:10d19c00f2ff32000400e000100032000394b900ea
:10d1ac0088c5550015c0b3000a45e900efff3a00e9
:10d1bc000400e00006003a002322ab00feff3a0018
:10d1cc0001c3b30001c045000000fb002011880022
:10d1dc004f05be004f04be00000006002322ab002a
:10d1ec00feff3a0000c3b30080c241008502fb0081
:10d1fc00251188000394b90088c5550015c0b300eb
:10d20c00e9ff3700881f7800000478002100200017
:10d21c00a0b028003cfe0700c440de00ef80600098
:10d22c00c0b02800e0c1780001102000a29e2100af
:10d23c0092806000020032004f047800000006006b
:10d24c002322ab00feff3a008301fb002311880070
:10d25c006f04640060407c002322ab00feff3a00a8
:10d26c000000fb00201188004f047800000006002d
:10d27c00f3ff3700881f780000047800210020009d
:10d28c00a0b0280020fe0700cc40de00c0b0280073
:10d29c00e0c1780001102000a29e21009280600065
:10d2ac00020032004f047800000006002322ab007d
:10d2bc00feff3a008301fb0023118800c840de000a
:10d2cc00ef806000e0c078002322ab00feff3a0044
:10d2dc008100fb0021118800c440de00ef8060005b
:10d2ec00e0c078002322ab00feff3a008100fb0077
:10d2fc00211188006f04640060407c002322ab0085
:10d30c00feff3a000000fb00201188004f0478005b
:10d31c0000000600e5ff3700889fbe000001780082
:10d32c007d14b900d2022000110009000284d8003b
:10d33c000004780042062000110009000284d80085
:10d34c0076ff070001102000a09e21009081600054
:10d35c000f00320042062000110009000284d800a0
:10d36c008000fd00e94f500006003e000300e00085
:10d37c0004003a002322ab00feff3a000103200018
:10d38c002111880065ff07004f04be000000060055
:10d39c002322ab00feff3a00e0022000201188009f
:10d3ac00ecff3700220320001241780032e0b70076
:10d3bc001180ba009100ba00230320008249780042
:10d3cc004800dd000080700000000600009e210077
:10d3dc0010407800e94f5000050032000080fb003f
:10d3ec000000400081af2800e10078004111880066
:10d3fc002022ef002062a8002222ef0021e2a800e8
:10d40c002342a8008560a9000000060010118000ce
:10d41c004800de0061406000000006001011800032
:10d42c0061406000000006000000eb00c0d08800e6
:10d43c0010002000b0d08800a09e21001090a10008
:10d44c00000006002322ab000d003a00c0d0800083
:10d45c000000e80001002100810f5000090032009b
:10d46c00b1d08000810f500005003200c0d0880080
:10d47c00f1ce8000614078000080fb002011880014
:10d48c00000006000000eb00b1d08000810f5000be
:10d49c00f6ff3a00faff3700c4d08000b3d080000a
:10d4ac00f5ce800004007800020021008000e80026
:10d4bc000000eb00828f5000010032000100780068
:10d4cc00830f5000080032002322ab00f8ff3a0013
:10d4dc0000027800e54078008180fb002111880073
:10d4ec008000e800f2ff3700c4d08800000006007e
:10d4fc00b1d08000c2d08000828f50000b0032006f
:10d50c00f2ce800000f178008100e800b1d08800f4
:10d51c0000002100808f5000010032000000060046
:10d52c000000eb00b0d0880000000600c222a90069
:10d53c0050cf80000090a00050cf88000000060063
:10d54c00889fbe008004780000c3b300e8ff07008a
:10d55c0080c7b300e6ff07004448de006f006000a0
:10d56c00c8b0280068407800e1ff0700ef84640031
:10d57c0068c07c00deff07004f04be000000060000
:10d58c002202ab00feff32003011800000000600ca
:10d59c002302ab00feff3200000006000110200049
:10d5ac00a29e21009280600004003a002322ab006e
:10d5bc00feff3a000000fb0020118800000006006e
:10d5cc000080fb0040118800000006002202d500fc
:10d5dc0061406000000006002222a9000000060045
:10d5ec009580ab000c003a00a0cf8000b1cf80003a
:10d5fc00808f5000080032002322ab00feff3a005f
:10d60c008580a9009580a80091cf800061407800aa
:10d61c000080fb002011880000000600809fbe00e7
:10d62c00821f78003211800080cf800061cf800093
:10d63c008270780080cf80000000e80080cf8800e6
:10d64c0071cf8000810f5000040032008560a9006a
:10d65c004f0178004f00be00004006009560a90005
:10d66c008560a9004f0178004f00be000040060005
:10d67c00faff3700809fbe00a0cf80000000e800ba
:10d68c00a0cf8800b1cf8000810f5000070032007e
:10d69c0091cf8000614078000080fb002011880051
:10d6ac008580a9004f00be00004006009580a900af
:10d6bc008580a9004f00be0000400600fbff37002c
:10d6cc00c8e2a800c902a900c922a900c8c2a900c1
:10d6dc00cae2a900cb02a900cb22a900cac2a900a8
:10d6ec0000000600501680004700de00614060001c
:10d6fc000000060051d08000c208de00e1c06000ce
:10d70c00014178000204a200610161004911dd00b1
:10d71c00f0df2f004416800084016000830171004b
:10d72c0043168800e1806000c908dd00ca02b6001b
:10d73c000080700050168800400120009e7b040081
:10d74c0000000000cb22a900c922a9004001200042
:10d75c009e7b04000000000051d08000c208de0057
:10d76c00e1c06000014178000204a2006101610087
:10d77c004811dd00f0ef2f0044168000840160009a
:10d78c008301710043168800e1806000c808dd0049
:10d79c00ca02b600008070005016880040062000b7
:10d7ac009e7b040000000000cb02a900c902a90066
:10d7bc00400620009e7b040000000000889fbe00f5
:10d7cc00804478000904e000060032000044eb00bd
:10d7dc00e1ff0700f4ff07000844e80088cf54007d
:10d7ec00fbff3e004f04be0000000600881f7800bf
:10d7fc00d9ff0700581680004744de0061446400de
:10d80c00e9ff0700084078004f047800000006008c
:10d81c00881f78000004e00009003200b5ff070003
:10d82c00cdff0700581680004744de0061446400b9
:10d83c00ddff0700084078004f0478000000060068
:10d84c00c0ff0700c4ff0700581680004744de00e5
:10d85c0061446400d4ff0700084078004f0478004e
:10d86c0000000600f6ff3700889fbe008a1f780074
:10d87c00cdff0700a8a021009840780068c0600088
:10d88c0010003a0089c0b3000044eb000ac8b30092
:10d89c00b1ff07000884fb000804d100cae2ab000a
:10d8ac00010032000a444400bfff07008944e9002c
:10d8bc00f7ff3a00084078004f0578004f04be008f
:10d8cc000000060050d080004400de006140600083
:10d8dc00cfff07001834a10089c0b3000044eb004f
:10d8ec000ac8b300eaff3700889fbe008a9fbe00bb
:10d8fc008c1f780000447800abff0700a9a0210022
:10d90c009940780068c060003a003a008045eb000e
:10d91c000b4578000cc8b3000808a3002c003a0093
:10d92c0088ff07008cff07000884fb000804d10067
:10d93c008b85fb008b05d100cae2ab001c003a00c2
:10d94c0099ff0700a1a021001941780063406100f4
:10d95c00e24f5000080032000a45e800e84f55003d
:10d96c00edff3a000b4078004f0678004f05be00e3
:10d97c004f04be0000000600e64f5500f6ff3a00cb
:10d98c00114078000030a0000808a30022003a00e3
:10d99c000044a100804878000b4078004f067800c6
:10d9ac004f05be004f04be0000000600f2ff37001a
:10d9bc008cc545007cff0700a1a02100194178000f
:10d9cc0063406100e24f5000e3ff3a00eaff37008a
:10d9dc0048ff070060ff07000884fb000804d10023
:10d9ec008b85fb008b05d100cae2ab00d4ff320063
:10d9fc00efff370050d080004400de006140600033
:10da0c0083ff07001934a1008045eb000b4578001b
:10da1c000cc8b300c0ff37000044a0008048780059
:10da2c000b4078004f0678004f05be004f04be0037
:10da3c0000000600d0ff370051d08000c208de0085
:10da4c00e1c06000014178000204a20061016100a4
:10da5c004611dd00f0fb2f004416800084016000ad
:10da6c008301710043168800e1806000c608dd0068
:10da7c00ca02b600008070005016880040012000d9
:10da8c009e7b040000000000cac2a900c8c2a90005
:10da9c00400120009e7b040000000000e6ff070010
:10daac00a0c0b30045ff0700f7ff0700a0a02100ae
:10dabc00c1cfb30010c8600000000600881f7800ba
:10dacc0000447800e24f540016003200e34f54003b
:10dadc00080032000804e000020032004f04780015
:10daec0000000600edff07004f0478000000060060
:10dafc00fcff3700d0ff070010c0b3002fff07005a
:10db0c00e1ff070020c0b3002cff0700a0a02100fc
:10db1c009040780063c870004f0478000000060045
:10db2c00f0ff3700c4ff07000840780023ff070010
:10db3c00d5ff07000840780020ff0700a1a02100b6
:10db4c00114078000000a1000014a000804878006b
:10db5c004f04780000000600e2ff3700881f7800b1
:10db6c00a8a0210050d0800063006000e20f50009c
:10db7c000d003200e30f500012003200e10f500094
:10db8c0007003200c0ff070010c0b3000bff0700f6
:10db9c00184078000000a0000014a100004c780090
:10dbac004f04780000000600184078000038a300ed
:10dbbc00040032000048a3000d003200cdfe070027
:10dbcc001834a1009cff070020c0b300fbfe070027
:10dbdc00adff070010c0b300f8fe07001840780036
:10dbec000000a0000014a100004c7800ecff3700ee
:10dbfc00d4fe07001834a100f2ff37000200fa002f
:10dc0c00889fbe008a9fbe008c1f7800c8e2a800c7
:10dc1c00c902a900c922a900c8c2a900cae2a90068
:10dc2c00cb02a900cb22a900cac2a900a0a0210046
:10dc3c00104178000224a00071ceb30001486100ad
:10dc4c00eaa02100f8a021008005eb00990f20002c
:10dc5c00c66a020000000000004d7800e14f500041
:10dc6c0042003200e24f5000f9ff3a00a0bf9f0083
:10dc7c008aff07009ffe0700b8ff07002fb8970028
:10dc8c008eff070000c0eb00ccfe070000c0eb00cd
:10dc9c00cafe0700b1ff070030c0b30087ff0700c2
:10dcac006bd08800acfe07005c1680004766de0077
:10dcbc0061466600bcfe07000c04e00005003a005b
:10dccc0060d080000000e80060d08800890f500010
:10dcdc00f4ff3e00a1ff070070ff07009fff070045
:10dcec0030c0b30075ff07002000200061d0800019
:10dcfc000008dd00d46a020000000000004ceb00bc
:10dd0c0060d080000000e00012003200d6fe070058
:10dd1c00d46a020000000000d3fe0700d46a02009f
:10dd2c0000000000d0fe0700d46a020000000000d2
:10dd3c00cdfe0700d46a0200000000001840e80085
:10dd4c00004c78000080fb0061d08000810f5000f7
:10dd5c00eeff390081ff0700c66a020000000000d8
:10dd6c00004d7800e14f5000beff3a004bff07001a
:10dd7c007aff0700b6ff3700814f500007003200d2
:10dd8c0051002000b0bb20006e7c0200000000009f
:10dd9c0080a221001048e80000000600310020009d
:10ddac0080bb20006e7c040000000000881f7800ff
:10ddbc000044780041002000b0ba2000167c02001c
:10ddcc0000000000501680004900de006140600039
:10dddc0088407800e8ff070031002000f0ba2000ee
:10ddec00167c020000000000501680004800de0087
:10ddfc006140600088407800dfff07004100200090
:10de0c0020bb2000167c0200000000005016800091
:10de1c004700de006140600088407800d6ff0700b4
:10de2c002100200060bb2000167c020000000000d6
:10de3c00501680004600de0061406000884078008b
:10de4c00cdff07004f04780000000600889fbe003d
:10de5c008a1f78000004be000205780080c2b3005f
:10de6c00d46a02000000000008007800567a020014
:10de7c00000000000004780008007800926902009d
:10de8c000000000090c2b300d46a02000000000041
:10de9c000040eb00890f54000300360010c0b300a3
:10deac008a0f54000500310011c0b300b2ff070007
:10debc004f0578004f04be00000006000040eb0048
:10decc0011c0b300acff07004f0578004f04be0033
:10dedc0000000600f9ff3700889fbe008a9fbe0035
:10deec00004578008144780088a22100004ceb00aa
:10defc000a04e0008c003a0050cf80000080a000a3
:10df0c0050cf88004100200040b220006e7c0200ff
:10df1c0000000000cb42a800c942a900310020003b
:10df2c0080b22000167c0200000000005016800019
:10df3c004a00de006140600011c0b3008eff070094
:10df4c00cb42a900c942a800c222a800c022a90045
:10df5c0081002000b0b22000167c020000000000fe
:10df6c00c202d5006140600011c0b30082ff0700ff
:10df7c00c222a900c962a800cb62a90081002000be
:10df8c0030b32000167c0200000000005016800008
:10df9c004b00de006140600011c0b30076ff07004b
:10dfac00cb62a900c962a90081002000b0b3200097
:10dfbc00167c020000000000501680004b00de00b2
:10dfcc00614060008040eb006bff0700c002a900bd
:10dfdc00c202a80020002000cc7b02000000000040
:10dfec004100200030b42000167c0200000000002c
:10dffc00101680006140600011c0b3005eff070086
:10e00c00e100200070b420006e7c020000000000d3
:10e01c0021e3a8002100200050b52000167c02004e
:10e02c000000000072352000712b200090002000b1
:10e03c0086ff07000904e00095003a00410020002b
:10e04c00a0b52000167c0200000000000225200074
:10e05c00011b2000a00020007cff070021e3a90089
:10e06c008100200010b620006e7c02000000000031
:10e07c00fbc32f00802c20001088650060168000e8
:10e08c00003cb3006016880040062000cc7b0200e8
:10e09c000000000010c0b30044ff0700a1002000e6
:10e0ac0090b620006e7c020000000000c02c200006
:10e0bc001088650040062000cc7b020000000000a8
:10e0cc000040eb0039ff07000a04e00002003200b8
:10e0dc000904e000b0003a00147a020000000000cd
:10e0ec0061002000d0b92000167c02000000000066
:10e0fc0018407800946802000000000081002000a5
:10e10c0030ba20006e7c02000000000050cf80006e
:10e11c000080a10050cf8800184078004f05be0049
:10e12c004f04be00000006000904e00075ff320039
:10e13c00f103200050ae20006e7c020000000000b5
:10e14c0011012000a01921006e7c020000000000cb
:10e15c00c66a0200000000004100200040b220000e
:10e16c006e7c020000000000cb42a800c942a9004e
:10e17c003100200080b22000167c0200000000005c
:10e18c00501680004a00de006140600011c0b300f0
:10e19c00f9fe0700cb42a900c942a800c222a80080
:10e1ac00c022a90081002000b0b22000167c020021
:10e1bc0000000000c202d5006140600011c0b30035
:10e1cc00edfe0700c222a900c962a800cb62a9001b
:10e1dc008100200030b32000167c020000000000fb
:10e1ec00501680004b00de006140600011c0b3008f
:10e1fc00e1fe0700cb62a900c962a90081002000e2
:10e20c00b0b32000167c0200000000005016800005
:10e21c004b00de00614060008040eb00d6fe070042
:10e22c00c002a900c202a80020002000cc7b020082
:10e23c00000000004100200030b42000167c0200d9
:10e24c0000000000101680006140600011c0b30097
:10e25c00c9fe0700e100200070b420006e7c0200b3
:10e26c000000000021e3a8002100200050b5200090
:10e27c00167c02000000000072352000712b20007b
:10e28c0090002000f1fe07000904e0006bff320053
:10e29c003100200070b52000167c02000000000048
:10e2ac0072352000712b2000b0002000e7fe070023
:10e2bc0041002000a0b52000167c020000000000e8
:10e2cc0002252000011b2000a0002000dffe07001b
:10e2dc0031002000e0b52000167c02000000000098
:10e2ec0002252000011b2000c0002000d7fe0700e3
:10e2fc0021e3a9008100200010b620006e7c0200f2
:10e30c0000000000fbc32f00802c2000108865004b
:10e31c0060168000003cb3006016880040062000a8
:10e32c00cc7b02000000000010c0b3009ffe070071
:10e33c00a100200090b620006e7c020000000000be
:10e34c00c02c200010886500c962a800cb62a9000f
:10e35c0040062000cc7b0200000000000040eb00d7
:10e36c0092fe0700a100200030b720006e7c020056
:10e37c000000000040168000003cb30040168800ee
:10e38c0040062000cc7b02000000000010c0b3004f
:10e39c0086fe07004cff3700c002a900c202a8008d
:10e3ac00c422a80001022000d0b720006e7c02001d
:10e3bc0000000000f1002000b01821006e7c02006b
:10e3cc0000000000c66a020000000000c422a90080
:10e3dc00c002a900c202a900147a020000000000c9
:10e3ec0061002000d0b92000167c02000000000063
:10e3fc0018407800946802000000000081002000a2
:10e40c0030ba20006e7c02000000000050cf80006b
:10e41c000080a10050cf8800184078004f05be0046
:10e42c004f04be00000006003fff3700a0b92800d3
:10e43c00b265040000000000c66a04000000000081
:10e44c00881f7800004478000880fb004401de003f
:10e45c00610161004a11dd004116800001a0a1009c
:10e46c008100710041168800c600dd000120b20059
:10e47c00421680000290a1000281700042168800b2
:10e48c00c600dd000110b200421680000280a1001f
:10e49c000281700042168800c600dd000108b2003f
:10e4ac00421680000270a1000281700042168800a2
:10e4bc00610060004600dd00411680000160a10093
:10e4cc008100700041168800500020009e7b0200e5
:10e4dc000000000000ceb30000406400cb42ab0053
:10e4ec00010032000044a000cb22ab00010032003e
:10e4fc000034a000cb02ab00010032000024a000cd
:10e50c00cae2ab00010032000014a000cac2ab008a
:10e51c00010032000004a0004f0478000000060047
:10e52c00881f7800004478000880fb000068a30076
:10e53c003e003200c002a900c202a8000058a3008d
:10e54c0037003200c962a800cb62a9004401de008a
:10e55c00610161004a11dd005116800001a0a1008b
:10e56c008100710051168800c600dd000120b20048
:10e57c00521680000290a100028170005216880091
:10e58c00c600dd000110b200521680000280a1000e
:10e59c000281700052168800c600dd000108b2002e
:10e5ac00521680000270a100028170005216880081
:10e5bc00610060004600dd00511680000160a10082
:10e5cc008100700051168800500020009e7b0200d4
:10e5dc000000000000ceb30000406400cb42ab0052
:10e5ec00010032000044a000cb22ab00010032003d
:10e5fc000034a000cb02ab00010032000024a000cc
:10e60c00cae2ab00010032000014a000cac2ab0089
:10e61c00010032000004a0004f0478000000060046
:10e62c00cb62a900c962a900c8ff3700c002a900cb
:10e63c00c202a900c1ff370000c0eb0080ff070039
:10e64c000040eb00b6ff3700889fbe00804078008a
:10e65c000040eb00726f02000000000000447800e4
:10e66c000804e00001003200c222a8000840780033
:10e67c00d46a0200000000008084eb00146a0200df
:10e68c00000000000004e00007003200c66a02002f
:10e69c0000000000e14f400015003200084040002f
:10e6ac00d46a0200000000000804e000f3ff3a0006
:10e6bc00d0d080000000e00009003a00d9d08800da
:10e6cc00c202d5000080ea006100600080004000ba
:10e6dc00101680000010a100008070001016880039
:10e6ec00d0d080000000e900d0d08800e3ff3700d4
:10e6fc0010c0b300d46a0200000000004f04be003a
:10e70c0000000600889fbe008a9fbe00c222a8009f
:10e71c00c9ff0700a0b92800b26502000000000084
:10e72c00c8a1210009fe2f00c66a020000000000eb
:10e73c00004c78000004e0002a0035000004e000e2
:10e74c0030003200e14f50002a003200e24f5000fe
:10e75c0036003200e34f50003c003200e44f5000d2
:10e76c002c003200e54f500040003200e64f5000c4
:10e77c0046003200e74f500026003200ef4f5000a9
:10e78c004a003200f04f500054003200f14f50005c
:10e79c006a003200f24f50006b003200f34f500011
:10e7ac0091003200f44f500097003200f54f5000aa
:10e7bc004d003200f64f5000a00032000068a3005c
:10e7cc00420032001eff0700d46a02000000000065
:10e7dc00c66a020000000000004c78000004e00053
:10e7ec00d6ff3d004eff0700d46a02000000000077
:10e7fc00cdff370090ff07000c3f02000000000027
:10e80c008dff0700a0b92800b265020000000000cf
:10e81c00c5ff370088ff070087ff0700a0b9280055
:10e82c00b265020000000000bfff370082ff070046
:10e83c0086620200000000007fff0700a0b92800dc
:10e84c00b265020000000000b7ff37007aff070036
:10e85c005a4a02000000000077ff0700a0b9280008
:10e86c00b265020000000000afff370072ff070026
:10e87c005a570200000000006fff0700a0b92800e3
:10e88c00b265020000000000a7ff37006aff070016
:10e89c00067802000000000067ff0700a0b92800fe
:10e8ac00b2650200000000009fff370010c0b300eb
:10e8bc00d46a020000000000c222a900ce6a020045
:10e8cc00000000000000fe0097ff37000040eb0046
:10e8dc00d46a02000000000093ff37000040eb00f8
:10e8ec0059ff070090ff370021e3a800c00020006b
:10e8fc00567a02000000000000057800ce6a020083
:10e90c00000000004850de00d46a02000000000045
:10e91c000a407800d46a020000000000146a020069
:10e92c0000000000e14f5000f0ff3a00c66a020000
:10e93c000000000021e3a9007bff370010c0b300ea
:10e94c0041ff070078ff37001021ef001e21ef0078
:10e95c009c21ef0051368000018064006001b300ff
:10e96c0050368800c66a0200000000000080fb00e0
:10e97c000018a3000100320010a1a8000008a30099
:10e98c00010032001081a800c66a020000000000dd
:10e99c004805dd00c66a0200000000000080fb0094
:10e9ac000a057000da0c8800ca0c88006000200090
:10e9bc00e00c8800c66a0200000000004805dd007b
:10e9cc00c66a0200000000000080fb000a00700014
:10e9dc006008880011e1a80010c0b300d46a0200de
:10e9ec000000000050ff37001021ef009c21ef00c9
:10e9fc00a26c20001289640010c0b300d46a02001b
:10ea0c000000000048ff370021e3a800c0002000f0
:10ea1c00567a0200000000000005780021e3a900ee
:10ea2c004850de00d46a0200000000000a40780062
:10ea3c00d46a0200000000003bff3700504f020078
:10ea4c00000000000005be004858de00d46a020039
:10ea5c00000000000b007800d46a020000000000e7
:10ea6c004859dd004850de0000007100c858de0037
:10ea7c00d46a0200000000000a407800d46a020048
:10ea8c000000000028ff3700829f21000049780019
:10ea9c00e34f50001a00320000202000d0cf880035
:10eaac00e0cf8800e1cf50001b003200e1cf5000d6
:10eabc0009003900e2cf500021003200e09f210014
:10eacc000048eb000000e8000048eb000000e80004
:10eadc000048eb000000060041c1b300e09f21009c
:10eaec000148780041c6b3000000e80001487800f6
:10eafc0021c3b3000000e8000148780000000600c4
:10eb0c0000202000d0cf880000082000e0cf880033
:10eb1c00e1cf5000e5ff3a0021c0b300e09f210097
:10eb2c0001487800a1c0b3000000e800014878005b
:10eb3c0051c0b3000000e800014878000000060056
:10eb4c0012c0b300e09f21000248780052c0b3000d
:10eb5c000000e800024878000000e8000148780056
:10eb6c0000000600829c2100124178007041610077
:10eb7c0004003200c822b7000180fb009e7b040019
:10eb8c0000000000cc22b7000080ea00c822b600ca
:10eb9c000180fb009e7b040000000000f9ff3700a1
:10ebac000080ea00cc22b600c822b6000180fb002f
:10ebbc009e7b040000000000889fbe008a1f780026
:10ebcc00004578000a04e0000b0032000044eb0022
:10ebdc00f99f21009940780000102000e1ff070008
:10ebec009940780000102000edff07000844e80071
:10ebfc00884f5500f7ff3e004f0578004f04be00cc
:10ec0c0000000600881f7800f89f210098407800cb
:10ec1c0000302000e2ff0700984078000010200030
:10ec2c00d0ff07009840780000202000cdff07009f
:10ec3c000000eb004f04780000000600889fbe0027
:10ec4c00f89f21009840780000302000c5ff070095
:10ec5c0019002000cb02ab000400320059168000d2
:10ec6c000920b2008904e900cf4cde0098407800fe
:10ec7c0000202000caff07009840780000102000f8
:10ec8c00c7ff07009840780000202000b5ff070060
:10ec9c00090078004f04be00000006000000e000f0
:10ecac0011003200809c2100104078007040600000
:10ecbc000500320001007800c822b7000280fb007a
:10eccc009e7b04000000000001007800cc22b700fd
:10ecdc000180ea00c822b6000280fb009e7b040083
:10ecec0000000000f8ff37000180ea00cc22b600db
:10ecfc00c822b6000280fb009e7b040000000000ce
:10ed0c00f1ff37000080fb00e19f210011417800ea
:10ed1c0001042000e1ff37000080fb00e19f21008f
:10ed2c001141780001102000dcff37000080fb004f
:10ed3c00e19f210011417800d1cf8000d7ff37002f
:10ed4c00881f78000080fb00e19f210011417800b2
:10ed5c00d1cf8000d1ff0700f89f210098407800a8
:10ed6c00001020007fff0700984078000010200062
:10ed7c008bff07004f04780000000600889fbe0040
:10ed8c008a9fbe008c9fbe007b9b21009b4078001d
:10ed9c000186fb000c06e900120020000c16dd00b9
:10edac000104e00013003200000478008004eb0042
:10edbc00ed9f2100028546000c0064001d41780087
:10edcc0001202000b5ff07009a40780000102000b9
:10eddc0064ff07009a4078000010200070ff0700c5
:10edec00080444008904e8001b80fb00890f5000d4
:10edfc00f1ff3e004f06be004f05be004f04be00a3
:10ee0c0000000600c822b70000000000000000004f
:10ee1c0000000000ca02b60000f0a7000000ea00e3
:10ee2c000000ea004f00de0000000600e0cf80008a
:10ee3c00f4ff3700889fbe00c99f2100190078009d
:10ee4c00f0ff070063844400984078000010200015
:10ee5c0044ff070019007800eaff0700804478009f
:10ee6c0098407800001020004dff07000940780002
:10ee7c004f04be0000000600889fbe008a9fbe00a3
:10ee8c008c1f780000202000deff07007c9b2100f7
:10ee9c000004eb001c04e000130032008004eb00c3
:10eeac00fa9f21009a407800001020002dff0700e7
:10eebc0000202000d3ff0700804578009a4078009e
:10eecc000010200036ff0700080444000b04e0008b
:10eedc00010032000804e8008904e8001c80fb00f3
:10eeec00890f5000efff3e00080078004f067800b5
:10eefc004f05be004f04be0000000600e48747002b
:10ef0c00889fbe008a9fbe008c9fbe008e1f78001b
:10ef1c007c9b21009c4078008186fb008d06e900db
:10ef2c00120020008d16dd000004eb000104e0004f
:10ef3c001c003200800478000005eb00ee9f2100dd
:10ef4c00820547000d8064001e41780001202000de
:10ef5c0052ff07009b4078000010200001ff0700c3
:10ef6c0000082000a7ff0700004178009b407800b4
:10ef7c000010200082bf9f0009ff07008984440015
:10ef8c00080444000fb997000204e00001003200ad
:10ef9c000804e8000a05e8001c80fb008a0f5000fa
:10efac00e8ff3e00080078004f0778004f06be00cf
:10efbc004f05be004f04be004f00b100000006001c
:10efcc00889fbe008a1f7800010578000a00e000c7
:10efdc0008003200800478000004eb00394078000f
:10efec00d46a0200000000000804e800880f5500f5
:10effc00faff3e004f0578004f04be0000000600eb
:10f00c00889fbe008a9fbe008c1f7800f8ce8000bf
:10f01c001000200050d18800c0ba2800b265020050
:10f02c00000000000a00220049832000c66a02008a
:10f03c0000000000e34f500019003200e34f500075
:10f04c0038003e00e14f500098003200930036002b
:10f05c00c66a02000000000080457800c66a020003
:10f06c0000000000e4cf5500e0003200af00360095
:10f07c00e8cf5500d6003200f0cf5500ebff3a0038
:10f08c000004e000df003200c962a800cb62a900d6
:10f09c00c66a020000000000e34f5000e7ff3a0090
:10f0ac00004c780080c0b3001044980021e3a80005
:10f0bc00c0002000567a020000000000c800de00ec
:10f0cc002144980030449800b0002000567a020089
:10f0dc0000000000c800de00414498005044980035
:10f0ec00a0002000567a020000000000c800de00dc
:10f0fc00614498007044980090002000567a0200f9
:10f10c0000000000c800de00014c9800104c980074
:10f11c0021e3a900a100200008007800a8ff070047
:10f12c00c2ff3700e64f5000580032002e003e0060
:10f13c00e54f500007003200004ceb000040eb00a4
:10f14c001044980011002000080078009cff070074
:10f15c00b6ff3700c66a02000000000000467800c7
:10f16c00c66a0200000000008560a900c865dd00c9
:10f17c008080fb008b8570008a8f55000100360063
:10f18c000b00220051c0b300014c78001c449800c5
:10f19c0020449800310020000800780088ff070008
:10f1ac00f0ce800060cf8800e7804500c308de0009
:10f1bc008180400071cf88000001eb0082cf880075
:10f1cc008900400091cf8800a2cf8800b2cf880080
:10f1dc009560a80053d180000b0178004e8002008e
:10f1ec000000000091ff3700e74f50000c00320088
:10f1fc00e84f5000d0ff3a00c66a02000000000041
:10f20c0080457800c66a020000000000c85ddd0081
:10f21c000080fb008b0570005bd1880083ff3700fa
:10f22c00c66a02000000000080457800e1cf55005e
:10f23c004700320020c2b300e66a02000000000062
:10f24c00c66a02000000000000467800c66a020090
:10f25c0000000000a1cab300814f56002b00320001
:10f26c0020c2b300e66a0200000000008045eb00fb
:10f27c0070c0b300004c78001b44980021002000a3
:10f28c00080078004eff070068ff3700c0ba28005e
:10f29c00b26502000000000064ff37004f067800e2
:10f2ac004f05be004f04be0000000600c66a0200f7
:10f2bc0000000000cac2a900cb22a900cb02a90001
:10f2cc00cb42a900ca02a900e24f50002c00320028
:10f2dc00cac2a900cb02a900cb22a900cb42a9002b
:10f2ec00ca02a9000040e900e14f50002900360095
:10f2fc00c8c2a800c922a800c902a800c942a80017
:10f30c00c802a800c8e2a80048ff370051c5b300e6
:10f31c00814f5000d6ff320020c2b300e66a0200d3
:10f32c00000000008045eb00d1ff3700e1cf550015
:10f33c001f003200e2cf55003cff3a000004e00011
:10f34c0033003200c002a900c202a80037ff370008
:10f35c0030c0b300e66a020000000000c66a02007a
:10f36c000000000000467800c66a020000000000a1
:10f37c00a1cab300814f5600b9ff3a00e3ff370032
:10f38c00cac2a800cb02a800cb22a800cb42a8007e
:10f39c00ca02a800c8c2a900c922a900c902a900b2
:10f3ac00c942a900c802a900c8e2a8001fff370083
:10f3bc00c022a9006100600000004000111680000e
:10f3cc000110a100810070001116880017ff370092
:10f3dc00610060004a00dd005116800001a0a10010
:10f3ec00810070005116880010ff3700610060002a
:10f3fc00511680000100a100810070005116880098
:10f40c000aff3700cb62a900c962a90007ff3700c9
:10f41c00c002a900c202a90004ff3700c922a8003b
:10f42c00c902a800c8e2a800c8c2a800c942a80026
:10f43c00c222a900c022a90000fe2f00ca26b600d5
:10f44c008000eb0021cf8800809c210010417800c7
:10f45c00f20150008149780001ceb30001486100ef
:10f46c00cb62a900c962a900c002a900c202a9000e
:10f47c002d83a9002d43a9002d23a9002d63a900dc
:10f48c0000198000000eb300001988003023ef0033
:10f49c0020f02100201988002223ef000000060034
:10f4ac00401988002023a8002003a9002003ab00ea
:10f4bc00feff3200001880000000060021e3a800c7
:10f4cc00c0002000401988002023a8002003a900b8
:10f4dc002003ab00feff320000188000926902008e
:10f4ec000000000021e3a90000000600889fbe0078
:10f4fc00e1002000e03520006e7c020000000000de
:10f50c00f1002000b01821006e7c02000000000009
:10f51c00f1002000c0362000167c02000000000024
:10f52c000000eb00926902000000000011002000b6
:10f53c00b0372000167c020000000000c80020003c
:10f54c00146a0200000000000004e00016003a00fb
:10f55c0021e3a800481988002023a8002003a90053
:10f56c002003ab00feff32000918800021e3a90044
:10f57c0020b92800b26502000000000009007800e4
:10f58c00926902000000000011002000b03720003a
:10f59c00167c020000000000146a0200000000004b
:10f5ac000004e000eaff3200c66a0200000000001e
:10f5bc0080b92800d2650200000000004f04be0094
:10f5cc0000000600889fbe0000047800709b21009c
:10f5dc0010407800ef4f500005003e000080fb000b
:10f5ec006f001000f1ff27000088de0000046400ab
:10f5fc0010cf8000e10f50001b00320006003900d4
:10f60c00e20f500022003200e30f50000c003200d9
:10f61c004f04be0000000600809c210001c2b30014
:10f62c0010c060002a003200080078004069020017
:10f63c00000000004f04be0000000600f6ff37007b
:10f64c00809c210001c2b30010c0600031003a0060
:10f65c0008407800d46a0200000000004f04be008d
:10f66c0000000600ecff3700809c210001c2b300b3
:10f67c0010c060001000320008007800e86602003c
:10f68c00000000004f04be0000000600e2ff37003f
:10f69c00809c210001c2b30010c0600012003a002f
:10f6ac000840780006660200000000004f04be000f
:10f6bc0000000600d8ff370008407800946802006c
:10f6cc00000000004f04be0000000600d2ff37000f
:10f6dc000800780008690200000000004f04be001a
:10f6ec0000000600ccff3700884478000840780002
:10f6fc00066602000000000000c2b300d46a0200db
:10f70c0000000000094078000666020000000000be
:10f71c00e6ff37004840de00d46a0200000000001b
:10f72c0008407800d46a020000000000cbff3700cc
:10f73c000000e000140032008000eb00000000002c
:10f74c0000000000000000000000000000000000ad
:10f75c00000000000000000000000000000000009d
:10f76c00000000000000000000000000000000008d
:10f77c000000000000000000000000008100e80014
:10f78c00810f5000edff3e0000000600889fbe0078
:10f79c00800478000900e0000c0032000004eb004b
:10f7ac00a00f2000e2ff0700a00f2000e0ff0700e1
:10f7bc00a00f2000deff0700a00f2000dcff0700d9
:10f7cc000804e800888f5400f5ff3e004f04be008b
:10f7dc000000060000027800020120001100200049
:10f7ec000000eb000000400084816000010032004a
:10f7fc000000a000818040000201e900f9ff3a00fe
:10f80c00719b210091407800f0cf50000300320032
:10f81c008180fb00f08010000100de00000006007b
:10f82c00889fbe008a9fbe00008540008a0f500052
:10f83c0011003100000478008b8522003900200073
:10f84c00110009000984d800e18f50000d0032002e
:10f85c00e28f50001500320000004000008045008f
:10f86c001000ba00d46a0200000000000804e8008e
:10f87c008a0f5400f2ff39004f05be004f04be0042
:10f88c000000060000004000008045001000ba0097
:10f89c004800de00d46a0200000000000804e80002
:10f8ac008a0f5400e6ff3900f3ff370000004000d8
:10f8bc00008045001080ba00d46a020000000000ed
:10f8cc000804e8008a0f5400ddff3900eaff370016
:10f8dc00d3ff070020bb2800d26504000000000005
:10f8ec001102200040272100f9ff0700c10420006d
:10f8fc0050292100f6ff070061022000102e210084
:10f90c00f3ff07008102200070302100f0ff070098
:10f91c0051012000f0322100edff0700b101200061
:10f92c0040342100eaff070081022000f03521005d
:10f93c00e7ff0700b101200070382100e4ff070049
:10f94c00e1022000203a2100e1ff070051012000d4
:10f95c00003d2100deff070031022000503e210057
:10f96c00dbff0700e102200080402100d8ff0700e8
:10f97c00c101200060432100d5ff070011022000c7
:10f98c0020452100d2ff0700c10120003047210093
:10f99c00cfff070051022000f0482100ccff0700e8
:10f9ac0011022000404b2100c9ff070091012000eb
:10f9bc00504d2100c6ff0700f1012000e04e210050
:10f9cc00c3ff070091022000d0502100c0ff0700a8
:10f9dc005102200060532100bdff0700610320008d
:10f9ec00b0552100baff0700e10320001059210097
:10f9fc00b7ff3700881f7800e100200070912000cd
:10fa0c0087ff0700c66a020000000000004478006f
:10fa1c0008407800d46a02000000000020bb2800d7
:10fa2c00d265020000000000f80db2009885b2000b
:10fa3c000804e9004f40de004f0478000000060087
:10fa4c00c222a9006820ef006a20ef006020ef00be
:10fa5c006220ef001e21ef00f0ff2800ac20b60062
:10fa6c001c21ef0000642000d00888000000210059
:10fa7c0080d088000000eb0090d0880000000600c9
:10fa8c00a1d080000100e00007003a00e24f5000d6
:10fa9c00150032000b003e000004e00017003a0095
:10faac00e7ff0700100005000040eb00e28f50005c
:10fabc0001003600000006000000eb00a0d088001a
:10facc0000000600f14f50001d003200f34f5000b3
:10fadc001b003200e44f50001a00320010002000ce
:10faec00a0d088000000050041002000a0b628002e
:10fafc008a6502000000000000000500e14f500084
:10fb0c00f6ff3a00c222a8001e21ef001621ef00da
:10fb1c001421ef001e61a8008660a9009660a90060
:10fb2c006005800000c0a00000d0a10000e0a10092
:10fb3c00600588001000200090d0880000000500af
:10fb4c000000050051012000e0b628008a65020083
:10fb5c000000000000000500881f7800411680009e
:10fb6c00007c20000100700040168800b4ff0700e4
:10fb7c0020c0b300c2ff0700146a0200000000009e
:10fb8c000004e00025003a0090d08000e10f500006
:10fb9c00f9ff3a008660ab0002003a006200e20016
:10fbac00f5ff3a001fe1a8008780a90088d08000eb
:10fbbc000800e000220032000001eb0001002100ef
:10fbcc0053168000c619de00f0ce80000370790059
:10fbdc003304800003806000fdff32008780a900a1
:10fbec000201e800880f5100f5ff39006220ef0098
:10fbfc001e21ef00f0ce80000800400070f8970046
:10fc0c00d46a0200000000000804e900f9ff3a0081
:10fc1c008bff07004f04780000000600c66a020044
:10fc2c000000000096ff07000004e000f9ff3a0016
:10fc3c0090d08000e10f5000cfff3a00d5ff370085
:10fc4c006220ef001e21ef007dff0700f1ff37005f
:020000040000fa
:10fc5c00901900002600000000000000161a000099
:10fc6c000400000000000000ec1900000c00000073
:10fc7c00000000001a1a0000040000000000000040
:10fc8c00261a000002000000020000000300000021
:10fc9c00d01900000e00000000000000f819000050
:10fcac000a000000000000000a1a00000600000014
:10fcbc0000000000de1900000e0000000200000031
:10fccc000008000000000000000000000000000020
:10fcdc0000000000b61900001a000000000000002f
:10fcec0000080000001000000000000000180000d8
:10fcfc00d000000000000000281a000002000000e4
:10fd0c0000000000101a00000600000000000000b7
:10fd1c001e1a00000400000000000000221a00005f
:10fd2c000400000000000000021a0000080000009f
:10fd3c00000000002a1a0000020000000000000071
:10fd4c00d0180000c000000002000000288128002c
:10fd5c0081288100288118008108810028812800d1
:10fd6c00812881002881080081288100f880f80012
:10fd7c0080e88000ce80ce0080ce8000e080da006b
:10fd8c00804869005a000000000000000847080085
:10fd9c00471a47001a473c0043d6420028812800e6
:10fdac00812881002881080081288100f8802a00a0
:10fdbc00475a49001844860046044700b44742009d
:10fdcc00435541005254000000000000b25eb200e6
:10fddc005e265f00265f32005ece5d002881280023
:10fdec00812881002881080081288100f880f80092
:10fdfc0080506100a85f0a006026600036608000b9
:10fe0c005f49320043000000000000000a37e200a6
:10fe1c003632370032376a003756370028812800cf
:10fe2c00812881002881080081288100f880f80051
:10fe3c0080323d00fc37a2003ab23900ca39880042
:10fe4c003753500049000000000000008281800000
:020000040000fa
:10fe5c000400fa00881f7800f0ff2f00010020003a
:10fe6c00d0bf9f00e1bf9f004507a9002ca3ef0066
:10fe7c004227a9005fb89700efb8970061015000c6
:10fe8c00e0815800d2bf9f00e3bf9f00e00f5000fd
:10fe9c00e08f5800f7ff3a0000fe2f00233580005a
:10feac00830060005100b30021358800c406b60001
:10febc003000b3002036880088c0b300009e2100bb
:10fecc00084878000080e8000008eb00147a020073
:10fedc0000000000ec6902000000000068c0a800ef
:10feec0068e0a8008000eb00f00f2000d869020049
:10fefc000000000030cf880021002000f00f20000f
:10ff0c00d86902000000000040cf88005116800024
:10ff1c00c208de00e380600072ba2800a09e2100b7
:10ff2c0062c8780068c0a90068e0a90050cf8000c2
:10ff3c000080a10050cf8800709b210008487800f9
:10ff4c003260ef0060ba2800d265020000000000a9
:10ff5c00fc10020000000000f81502000000000078
:10ff6c000000eb004f0478000080fa00000006004f
:10ff7c00e1806000c908dd00f5df2f0076168000f7
:10ff8c0086826200858270007516880001fe2f0043
:10ff9c0035358000858060007100b30031358800f4
:10ffac00f50f2e004636800086826200015020003c
:10ffbc008580700041368800c01188003022ef0027
:10ffcc003062a800610161004410dd00f1fe2f00d9
:10ffdc00851180008580600081007000811188008f
:10ffec00e38161008381410090ff2f003002b60055
:10fffc00008071008011880061026200e0ff2f0018
:020000040001f9
:10000c003002b60000007200801188003222ef002e
:10001c004e11dd00f0ff2b003202b6000000710023
:10002c00901188000000060031e2a8003342a800bd
:10003c0087c0a900c922a9000000060031e2a9006e
:10004c003342a90030358000f001b3003035880010
:10005c00f00f2e00c826b600cf22a900c922a80096
:10006c00000006003322ab00feff3a00a01188000e
:10007c00000006003202ab00feff3200b01180001f
:10008c000000060090118000614060000000060036
:10009c00889fbe008a9fbe008c1f78008002eb00f8
:1000ac000203e9008003780001047800030678005d
:1000bc00a92c20009a0020006b00200070cf80003b
:1000cc00e48242000028e60005007800f019e30005
:1000dc00feff350037017800b70178000280fd0083
:1000ec0003026900f40fb200040169008481690005
:1000fc000280fd00f00020000030e60006007800d1
:10010c00800078000c800900000000001980a1001c
:10011c000281d3001950ad008381d3001958ad0072
:10012c000c800900000000001980a0001970a300c9
:10013c000482d3008100e900f2ff3100ef001000cf
:10014c000122de00041c78004300de000000e80001
:10015c00f639b4009580ab0006003200a0cf8000c9
:10016c00f619e30003003200f219b4001000780015
:10017c002011880070035300d0ff31004f06780027
:10018c004f05be004f04be00f66a040000000000dc
:10019c0081c0b300709b21000148780071004000c1
:1001ac001054a1000000060040bb2800d2650400da
:1001bc000000000001012000400621006e7c0400bc
:1001cc000000000011022000203f20006e7c020085
:1001dc000000000011c0b3004088210001487800e5
:1001ec000000060011022000203f20006e7c02005f
:1001fc000000000011c0b3004088210001487800c5
:10020c000000050011022000203f20006e7c02003f
:10021c000000000011c0b3004088210001487800a4
:10022c000000050011022000203f20006e7c02001f
:10023c000000000011c0b300408821000148780084
:10024c000010050011022000203f20006e7c0200ef
:10025c000000000011c0b300408821000148780064
:10026c00000006000080fb000038a3001c003200d8
:10027c00c002a900c202a8000028a3001500320089
:10028c00c962a800cb62a9000018a3000a003200c2
:10029c00c942a900cb42a8000008a3000a00320002
:1002ac00809c210010407800704060000f003200ec
:1002bc00c8c2a80000000600c942a900cb42a90090
:1002cc000008a300f6ff3a00ccc2a900c8c2a900de
:1002dc0000000600cb62a900c962a900eaff370042
:1002ec00c002a900c202a900e3ff3700ccc2a800db
:0802fc00c8c2a90000000600c1
:020000040000fa
:020000040001f9
:0403040000000000f5
:020000040000fa
:020000040001f9
:0457f800dff90000d5
:020000040000fa
:020000040001f9
:0457fc007f3f0000eb
:00000001FF
